:100000004808002015AC0108B9AF0008CDAF0008C2
:10001000E1AF0008F5AF000809B0000800000000DB
:100020000000000000000000000000001DB00008FB
:1000300031B00008000000009D740008F3CD0008F6
:1000400041AC010845AC010849AC0108BBD6000829
:100050004DAC0108E3B400088DB0000851AC0108B4
:100060003BB200081BB3000855AC010859AC0108AD
:100070005DAC010861AC010865AC010869AC010820
:100080006DAC010871AC010875AC010800000000FE
:1000900000000000000000000000000079AC010832
:1000A0007DAC01085184010881AC010885AC0108D0
:1000B00000000000000000000000000089AC010802
:1000C0008DAC010891AC010895AC010899AC010810
:1000D0009DAC0108A1AC0108A5AC0108000000001E
:1000E000A9AC0108F7B30008000000000000000000
:1000F000000000000000000000000000ADAC01089E
:100100000000000000000000B1AC01080000000089
:100110000000000000000000B5AC01080000000075
:10012000B9AC0108BDAC0108C1AC0108C5AC0108FF
:10013000C9AC010800000000000000000000000041
:1001400000000000000000000000000000000000AF
:10015000FB830108CDAC0108D1AC0108D5AC010886
:10016000000000000000000000000000000000008F
:10017000000000000000000000000000000000007F
:10018000D9AC0108DDAC010800000000000000004F
:1001900000000000E1AC01080000000000000000C9
:1001A000000000000000000000000000000000004F
:1001B000000000000000000000000000E5AC0108A5
:1001C000E9AC0108EDAC010870B500224FF41261F2
:1001D000DFF8140B02F002F9DFF8104B00221021B7
:1001E00004F11C0002F0FAF8DFF8045B0022182189
:1001F00005F10C0002F0F2F80022082104F12C00B5
:1002000002F0ECF80022082104F1340002F0E6F8D4
:100210000020E06320646064A0646862A862E86211
:10022000DFF8D06AB063F063E06428633064706420
:100230006863A863E863012028640020B064F06468
:100240004FF0FF306864A8640020E86430652065E2
:100250007065F06530667066B066F06202462C210B
:10026000304602F0BBF842F210707081B08100207D
:100270007060022030810020306002460C21204650
:1002800002F0ACF8DFF8700A6060DFF8700A2060F6
:10029000012020720020287028656880A880E880EE
:1002A0006065F0662881A06530636865A865606652
:1002B000A066E0667067306768662866E8650120BA
:1002C0002867E866A8660020E867A86768670620D0
:1002D000B0860020A082F067B0672067DFF8200AB0
:1002E000E065002020660120E082962068810620DB
:1002F000F0860C2020830020B06502464021DFF804
:100300005C0D02F06BF80022062104F10C00BDE840
:10031000704002F063B810B584B0DFF8D0490C2209
:10032000214600A802F098F8FFF74EFF0C2200A922
:10033000204602F091F81FBD2DE9F0472DED0C8B02
:1003400090B00024254600A821460A460B460EC060
:10035000302102F0B9F89FED9B8ADFF8906996EDA5
:100360001B0AD6ED140AC6ED1B0ADFF8887997ED53
:10037000149A86ED149ADFF8788998ED131AB8EE7E
:10038000411ADFED911AC1EE819AC7ED149AD8F89F
:100390004420D8F83490A9EB0200FA30FA21B0FBDF
:1003A000F1F1FA2303FB110080B2002800F0FE8374
:1003B0004C2880F28180D8F8401001297CD0D7F8F1
:1003C0004CA0BAF1040F21D3F4EE490AF1EE10FA71
:1003D0001CD5B4EE699AF1EE10FA17D59FED7B1A91
:1003E00020EE811AB4EE691AF1EE10FA0ED59FEDE7
:1003F000DB1AF4EE419AF1EE10FA07DB87ED149A5E
:10040000C6ED140A86ED1B0A00F009BC97ED0EAA92
:1004100087ED0FAAD7ED10AAC7ED11AA014600EE8D
:10042000101AB8EE400AD8ED0B8AC8EE800A98ED93
:100430000C1A81EE001A2146B963396420E0521C7F
:1004400092B2FA2A00D12246DFF89C3803EB8203ED
:10045000D3ED231A71EEE01AD3F8743402EE103A99
:1004600032EE412AD7ED0E2A41EEA12AC7ED0E2A1F
:10047000D7ED101A42EE021AC7ED101A491C89B2C4
:100480008142DCDBD7ED0E0A80EE80BA87ED0EBA32
:10049000D7ED100A80EE80CA87ED10CAD6ED1ABAE1
:1004A00098ED150AD8ED160A70EE60CAC6ED1ACAA4
:1004B00000F092FF012802D12046386376E3BAF1BA
:1004C000000F0BD1388E052802DB05462046388602
:1004D000788E052802DB4519204678861AFA85F0C1
:1004E000002824D1B6EE00DA3CEE2A0A20EE0D0AEE
:1004F000DFED9B0AB4EE600AF1EE10FA11D43BEE88
:100500000A0A20EE0D0ADFED970AB4EE600AF1EE5A
:1005100010FA06D4B3EE040AF4EE40CAF1EE10FA73
:1005200005D5388E401C3886C8F848903EE3388E92
:10053000002802D04519204638861AFA85F000288E
:1005400015D1B7EE000AF4EE409AF1EE10FA00F180
:100550002D839FED850AF4EE409AF1EE10FA03DB4D
:10056000788E401C788621E32046788603E0788EDA
:10057000451920467886284680B200F0C3FF01283E
:1005800008D187ED149AC7ED10AAC6ED1ABA87ED07
:100590000EAA0BE39FED750AF4EE409AF1EE10FA05
:1005A00002DBDFF8180C386520463886BAF1000FF8
:1005B0000ED1386D786586ED13BAC6ED19CA00F014
:1005C000A5FE3CE00000000000007A446666E63FBD
:1005D000B6EE00DA00F09AFE012816D197ED140A63
:1005E000F0EE000A20EE200A87ED140A6BEE0D0AE9
:1005F000C7ED0E0A2CEE0D1A87ED101AC7ED0F0A83
:1006000087ED111A86ED140A6D1C97ED140AD6EDCC
:10061000140A30EE200A20EE0D0A87ED150A97ED38
:100620000E0AD7ED0F0A30EE200A20EE0D0A86EDF5
:10063000130A3BEEAC0A20EE0D0A86ED190A98F873
:100640000100012840F0A782D8F80C00009000A813
:10065000D8F810104160D8F814108160214617E0D6
:1006600000AB03EB820393ED010A50F822C000EEC9
:1006700090CAB4EE600AF1EE10FA05D500EB820CD8
:100680008CED000AC3ED010A521C022AE8DB491C6A
:10069000022901DA2246F8E79DED000AB5EE400A8C
:1006A000F1EE10FA2AD5B5EE400AF1EE10FA01DCAF
:1006B000B1EE400AD0ED020A30EE800A80ED020A67
:1006C0009DED000AB5EE400AF1EE10FA01DCB1EE44
:1006D000400AD0ED010A30EE800A80ED010A9DED5E
:1006E000000AB5EE400AF1EE10FA01DCB1EE400A64
:1006F000DDED000A30EE800A8DED000A90ED010A72
:10070000D0ED020A30EEC01ADDED000A30EE600ACC
:10071000B4EE401AF1EE10FA05D5F0EE410AB0EE53
:10072000401AB0EE600AD6ED0B0AC6ED0C0A31EEA7
:10073000400A80EE010A9FED0E1A20EE010A86EDB6
:100740000B0A706BB063F4EE400AF1EE10FA11D5AB
:1007500070EE600AC6ED0D0A10E000BF01004040D7
:10076000000016430000A042666616400100A0404B
:100770000000C84270EEC00AC6ED0D0A386F796FEE
:10078000081800EBD070401002EE100A86ED0F2A18
:10079000C6ED108AD7ED100AC6ED110AD7ED141A6E
:1007A000DFF8300CC0EDC41A96ED121A31EE611A62
:1007B000D6ED122A72EEE12A21EE221A00F54471DA
:1007C00081ED011AC6ED121AD7ED1B1AC1ED021AFE
:1007D000D8F81810039103A9C1ED011AC1ED020A5E
:1007E000C1ED038AC1ED041AC1ED058AC1ED061AF7
:1007F000B8EEC22A81ED072AC1ED081A81ED090A77
:10080000C1ED0A1A81ED0B1ADDED032A9FEDD03AF6
:1008100062EE832A9FEDCF3A41EE832A9FEDCE3AD6
:1008200020EE833ADFEDCD3A08EEA33ADFEDCC3A85
:1008300061EEA33A9FEDCB4A48EE843A9FEDCA4A57
:1008400021EE844ADFEDC94A02EE244ADFEDC84AB0
:1008500061EEA44A9FEDC75A40EE054A9FEDC65A85
:1008600021EE855ADFEDC55A01EE255AF8EE085AF9
:10087000F4EE652AF1EE10FA00F18D81DFEDC05A39
:10088000B4EE653AF1EE10FA00F18581DFEDBD5A64
:10089000F4EE653AF1EE10FA00F17D81DFEDBA5A1F
:1008A000B4EE654AF1EE10FA00F175819FEDDF6A52
:1008B000F4EE464AF1EE10FA00F16D819FEDDC6A2C
:1008C000B4EE465AF1EE10FA00F16581DFEDD96A17
:1008D000F4EE662AF1EE10FAC0F25D81DFEDD62A61
:1008E000B4EE623AF1EE10FAC0F25581F4EE653AD8
:1008F000F1EE10FAC0F24F81B4EE464AF1EE10FA72
:10090000C0F24981F4EE654AF1EE10FAC0F243817B
:10091000DFEDCA2AB4EE625AF1EE10FAC0F23B8162
:10092000DFEDC72A9DED033AB4EE623AF1EE10FA1C
:1009300001D5CDED032ADDED032A9FEDD83AF4EE83
:10094000432AF1EE10FA02DBDFF8AC2B0392DFED65
:10095000D42AF4EE621AF1EE10FA01D5C1ED012AA3
:100960009FEDB83ADFEDB83A91ED014AB4EE634A33
:10097000F1EE10FA01DB81ED013A9FEDB44AF4EE9D
:10098000440AF1EE10FA01D581ED024AD1ED020AD6
:100990009FEDAF4AF4EE440AF1EE10FA02DBDFF805
:1009A0005C2B8A60DFEDBF0AF4EE608AF1EE10FA8C
:1009B00001D5C1ED030A9FEDBC4AD1ED034AF4EE27
:1009C000444AF1EE10FA02DBDFF8342BCA60F4EE91
:1009D000621AF1EE10FA01D5C1ED042AD1ED044AF4
:1009E000F4EE634AF1EE10FA01DB81ED043AF4EE25
:1009F000608AF1EE10FA01D5C1ED050AD1ED050AC4
:100A0000F4EE440AF1EE10FA02DBDFF8F42A4A6150
:100A1000F4EE621AF1EE10FA01D5C1ED062AD1ED1D
:100A2000060AF4EE630AF1EE10FA01DB81ED063AF4
:100A3000F1EE000AB4EE602AF1EE10FA02D54FF0A2
:100A40008142CA61D1ED070A9FEDA12AF4EE420A64
:100A5000F1EE10FA02DBDFF82C2CCA61F4EE621A18
:100A6000F1EE10FA01D5C1ED082AD1ED080AF4EE35
:100A7000630AF1EE10FA01DB81ED083ADFED950A29
:100A8000B4EE600AF1EE10FA01D5C1ED090A91ED5C
:100A9000090ADFED910AB4EE600AF1EE10FA02DB0A
:100AA000DFF8E42B4A62F4EE621AF1EE10FA01D597
:100AB000C1ED0A2A91ED0A0AB4EE630AF1EE10FACA
:100AC00001DB81ED0A3AB5EE401AF1EE10FA01D5DC
:100AD0002246CA6291ED0B0ADFED800AB4EE600A8D
:100AE000F1EE10FA02DBDFF8A42BCA62214612E015
:100AF0001B1FD3ED000A92ED031AF4EE410AF1EE4A
:100B000010FA01D59FED760AB8EEC00AD2ED020ABE
:100B100000EE208A491C312938DA9FED720A0B0158
:100B20001A18D2F804C0BCF1010F0DF10C0C1B58BF
:100B30000CEB8303DCD11B1FD3ED000A92ED031AEB
:100B4000F4EE410AF1EE10FADEDB9FED650ADBE719
:100B5000168733BDB0568DBD03275BB9E23C9CB907
:100B6000983115BEBF49D3B97061FDBD55C128BCD0
:100B700036CB05BE3D7FDABBDDED0ABEE4BE353EB9
:100B80006666A6BF3333F3BFCDCC4CBFB5EE408A0B
:100B9000F1EE10FA0ADC97ED150A284680B200F053
:100BA000B1F800F057F80446C8F84890C8F84490E7
:100BB0000020C8F84C00C8F82C00C8F83000C8F86D
:100BC00040000246102106F11C0001F007FC002243
:100BD0000C2108F10C0001F07FFC4948F065002071
:100BE0003066F88800281AD1F86F00280CD0B86C4D
:100BF0003969401AB98EB0EB510F02DB0020388101
:100C00000DE0012038810AE0388E798E11FA80F0EB
:100C1000032802DB0120388101E0022038812046D0
:100C200010B0BDEC0C8BBDE8F08700BFCDCC8CBF05
:100C3000333333BFCDCC0CC09A9919BFCDCC4CBE49
:100C40005017C93F15E6684016E668407D90A341FD
:100C5000A2F2924438B50025DFF8BC4B0120E067D2
:100C600000F0F0FC2060E06CA18E884214D3A06CF0
:100C70002061A08DA080E08DE080A06DA061E06D7E
:100C8000E061206E2062606E6062A06EA062012052
:100C9000A0672846E0670125284632BDC9AC454219
:100CA000A9F56E3EBA9F17443564EC4411480169BA
:100CB00081640021C1644160022101810021C1627F
:100CC000016A0166816A81660021C1677047000080
:100CD000010058427B4D4F3D47FFC742BEBA984185
:100CE00001000000FFFFFFFFBC250020341D002095
:100CF000341C0020B41C002000002F430000704270
:100D000000007A442DE9F84F2DED048B82B0834624
:100D1000F0EE400A00239E461846DFF8FC4AE56CD8
:100D200005F10F0101F00F01EA1D02F00702009228
:100D3000CA4A02EB8106C6ED000ABBF1000F15D0CE
:100D4000064611E04F1EBF1B10374FEAE70C07EBBA
:100D50001C7C4FEA2C1CB7EB0C1703D402EB870763
:100D6000C7ED000A761C36B25E45EBDB102D02D2D1
:100D7000294609B200E00F219FEDB68A9FEDB51A12
:100D8000DFEDB51A06461BE052F8217000EE107A2E
:100D9000B5EE400AF1EE10FA10DD38EE008AB4EE3E
:100DA000401AF1EE10FA01D5B0EE401AB4EE610A25
:100DB000F1EE10FA01D5F0EE401A761C491E09B288
:100DC0000029E1D536B2314603290BDB38EE410A62
:100DD00030EE610A891E01EE101AB8EEC11A80EEDB
:100DE000018A07E0012905DB00EE106AB8EEC00AAF
:100DF00088EE008AB5EE408AF1EE10FA01D0002E9E
:100E000001D1B0EE608A84ED168A9FED950AB4EEAA
:100E1000408AF1EE10FA02D5B0EE408A08E09FED6C
:100E2000910AB4EE408AF1EE10FA01DBB1EE028ACB
:100E3000B0EE040AB4EE408AF1EE10FA08D494ED54
:100E40001B0AF0EE080AB4EE600AF1EE10FA02D5C1
:100E50000321A18501E00421A185A66C06F0070805
:100E6000DFF8BC7908EB070CA18D8CF8B818BBF142
:100E7000000F0AD0721E02F00702D21906F007090D
:100E8000B94499F8B89882F8B89808220EE0B9F1F8
:100E9000040F00D1401CA8F101080FFA88F8B8F13E
:100EA000000F01D508F10808521E12B2012A16DB04
:100EB0000FFA88F808EB070999F9B898B9F1030F08
:100EC00002D10EF1010E03E0B9F1040F00D15B1C59
:100ED000062AE0DBB9F1030FD9D1401EDBE7E28D32
:100EE0009BB21FFA8EFE734507D39E4502D20420A3
:100EF000E0850DE000B2002802D50320E08507E080
:100F0000012802DB0420E08502E09CF9B808E085B6
:100F1000B4F82E80B8F1040F01D1184600E07046F5
:100F2000424509D000202081E088002820D1042DEE
:100F30001ED3012020811BE013FA8EF2012A15DB5B
:100F4000052A10DB00EE102AB8EEC00AF6EE080AF9
:100F500020EE200A00EE900AF8EE600AF4EE400A55
:100F6000F1EE10FA02D50120208101E0022020815B
:100F7000DFF8B09849B2B0EE480A484600F020F9D0
:100F8000DFED8D0AB4EE600AF1EE10FA01D5B0EE95
:100F9000600A84ED170A584600F1010A00EE90AA93
:100FA000F8EEE08AD4ED180A48EE800AC4ED180A7B
:100FB0009FEDCB9A20EE080A20EE090A009907EB74
:100FC000810101F65C0181ED000ABBF1000F16D032
:100FD000002212E00099491E891A08318B1001EB9A
:100FE0005373DB10B1EBC30105D407EB810101F6AC
:100FF0005C0181ED000A521C12B28242EADB082D2C
:1010000002D2284600B203E0072001E0401E00B2F1
:101010000028FBD584ED190A414649B2484600F044
:1010200047F968EE090AB7EE001AC1EE200A20EE71
:10103000800AD4ED1A0A48EE800AC4ED1A0A0AEBB7
:101040000600A0640AEB0500E06402B0BDEC048B6E
:10105000BDE8F18F000000000000C842E86E0020EB
:101060006666A63F0100904049B2032944D1DFEDF6
:101070009D0AB4EE600AF1EE10FA01DBB0EE600AF0
:101080009FED991ADFED990A40EE010A90ED011AE1
:101090009FED970AB4EE401AF1EE10FA43DADFED55
:1010A000951AB4EE611AF1EE10FA74DBB4EE401A40
:1010B000F1EE10FA6FD59FED900A31EE000ADFEDE8
:1010C0008F1A60EE211A9FED8E0A9FED8E2A01EE97
:1010D000002A22EE200A20EE210A9FEDB72ADFED3A
:1010E000B72A41EE022A62EEA00AB7EE001A31EEEC
:1010F000611A00EE810A56E0DFED830A60EE200AF5
:1011000060EE800A9FEDAE1A40EE410A9FEDAD0AF7
:1011100070EE800A90ED011A9FED750AB4EE401A48
:10112000F1EE10FA0ADB90ED010A9FED751ADFED82
:10113000751A40EE011A21EEA00A34E0DFED6D1AB7
:10114000B4EE611AF1EE10FA25DBB4EE401AF1EEBE
:1011500010FA20D59FED680A31EE000ADFED671A1C
:1011600060EE211A9FED660A9FED662A01EE002AC5
:1011700022EE200A20EE210A9FED8F2ADFED8F2A32
:1011800041EE022A62EEA00AB7EE001A31EE611AB1
:1011900000EE810A07E090ED010A20EE800ADFED03
:1011A0008A0A20EE200A007A022803D1DFEDCA0A5B
:1011B00020EE200A70470000CDCC4C3E0000A0403D
:1011C00010B52DED028BB0EE408A0C46DFED7F8A24
:1011D00049B2FFF749FF64B2042C31D1DFED7C0A3C
:1011E000B4EE608AF1EE10FA16DBB1EE021AB4EE3C
:1011F000418AF1EE10FA0FD5DFEDB80A78EE200A39
:10120000B1EE041A60EE810AFCEEE00A10EE900ADC
:10121000C01D08EE900A3DE0B4EE608AF1EE10FACF
:1012200003D5072008EE900A34E0F1EE020AB4EE8E
:10123000608AF1EE10FA2DDB122008EE900A29E008
:10124000F7EE080AB4EE608AF1EE10FA11DBDFED7A
:10125000A40AB4EE608AF1EE10FA0AD5FFEE080A8D
:1012600078EE200AB1EE041A60EE810AFCEEE08A04
:1012700010E0F7EE080AB4EE608AF1EE10FA09D435
:10128000DFED970AB4EE608AF1EE10FA02DB062079
:1012900008EE900ADFF8580D18EE901A00EB810066
:1012A000D0ED000A20EE200ABDEC028B10BD00003C
:1012B000F0EE0C0A49B2042904D19FED8A1A40EEDF
:1012C000010A03E09FED881A40EE010A9FEDDB0A58
:1012D00020EE800AD0ED000A20EE200A70470000C0
:1012E000000070429A9919406ADEF13D8638163F37
:1012F00000002A4300001643000016C3CDCC4C3D2D
:101300004260E53A6666263F2575C23E0020DFF85A
:10131000081591ED140AF7EE040AB4EE600AF1EE36
:1013200010FA47DADFF8CC2CD288042A42DAD1ED61
:10133000150A9FED6E1A60EE810AB4EE600AF1EEB6
:1013400010FA03D5022A01DB012012E0DFF8D414E1
:1013500091ED0A0ADFED660AB4EE600AF1EE10FACA
:1013600007DBDFED640AB4EE600AF1EE10FA00D597
:10137000012001281ED1DFF8AC1491ED170AD1ED40
:10138000180A70EEC00A9FEDAE1AF4EE410AF1EEB3
:1013900010FA07DBF7EE080AB4EE600AF1EE10FA75
:1013A00000D50020DFEDB30AB4EE600AF1EE10FACA
:1013B00000D500207047000052491D3BB81E053F74
:1013C0007593E83F24975340C1C0C03B0000000024
:1013D00066660640481800200021DFF83C24D38DC3
:1013E000032B1BDA92ED140ADFEDA30AB4EE600AB8
:1013F000F1EE10FA12DB92ED0E0AF2EE040AB4EEF0
:10140000600AF1EE10FA09D592ED100ADFED9B0AA1
:10141000B4EE600AF1EE10FA00D5012192ED100A47
:10142000F6EE000A92ED111A30EE011A21EE201AA2
:10143000F3EE0E1AB4EE611AF1EE10FA1CD492ED2E
:101440000E1AD2ED0F1A71EE211A61EEA01AB2EE49
:10145000042AF4EE421AF1EE10FA0DD4F3EE041A57
:10146000B4EE610AF1EE10FA06D4B1EE040AB4EE5D
:10147000401AF1EE10FA00D5012192ED140A9FED09
:10148000801AB4EE410AF1EE10FA23DBDFF8942360
:1014900092ED090A92ED0A1A80EE010A9FEDA51A53
:1014A000B4EE410AF1EE10FA14DB00EE100AB8EEC9
:1014B000400A20EE200AD2ED070AF4EE400AF1EECF
:1014C00010FA07D5D2ED080AF4EE400AF1EE10FA50
:1014D00000D50121084670473333733F666606C066
:1014E0009A993940CDCC4C3ECDCCCC3D3333333FB3
:1014F000010020420000C842C8AC4542A1F292441B
:101500003464EC440021C44AD36C13FA80F00228FE
:1015100016D392ED140ADFED880AB4EE600AF1EEFC
:1015200010FA0DDB92ED110AD2ED100A80EE200ABE
:10153000DFED820AB4EE600AF1EE10FA00DB012161
:10154000022818D39FED7E0AD2ED110A92ED101AEF
:10155000C0EE810AF4EE400AF1EE10FA0BDBD2ED98
:101560000F0A92ED0E1AC0EE810AF4EE400AF1EE77
:1015700010FA00DB012100280ED0AA4890ED190ACC
:10158000DFED9E0A20EE200AD0ED1A0AF4EE400AA2
:10159000F1EE10FA00D5012192ED140ADFED980A60
:1015A000B4EE600AF1EE10FA08DA92ED150ADFEDFA
:1015B000950AB4EE600AF1EE10FA1ADB92ED100A09
:1015C000DFED910AB4EE600AF1EE10FA0DD492ED5F
:1015D0000E0ADFED8E0AB4EE600AF1EE10FA04D4C2
:1015E000DFF8100AC088022803DBD08D032800DB57
:1015F00001218C4890ED130ADFED830AB4EE600AF6
:10160000F1EE10FA08D492ED1B0AF1EE040AB4EEE2
:10161000600AF1EE10FA0ED5106F526F101800EE3E
:10162000100ABAEEEF0ADFED7A0AB4EE600AF1EEC4
:1016300010FA00DB01210846704700000AD7A33BDF
:101640000100C03F002074498A6C12F10A0F0FD2CA
:101650009FED700AD1ED180AF4EE400AF1EE10FA8F
:1016600006DAD1ED1A0AF4EE400AF1EE10FA00DBC8
:101670000120704785EB113F01000040000020422F
:10168000010040400000584246FFC742BDBA9841A1
:1016900010B401460020634A614BD3F8144900EEB0
:1016A000104AD1ED000AB4EE600AF1EE10FA08D14A
:1016B000147B641C1473E4B2FE2C04DB3224147318
:1016C00001E00446147303F6141393ED010AD1EDFF
:1016D000010AB4EE600AF1EE10FA08D1547B641CE2
:1016E0005473E4B2FE2C04DB3224547301E004464C
:1016F000547393ED020AD1ED020AB4EE600AF1EEE2
:1017000010FA08D1917B491C9173C9B2FE2904DB00
:101710003221917301E001469173117B322905DA80
:10172000517B322902DA917B322900DB012010BC87
:10173000704700003433333F010060400100A04097
:10174000010070410146002091ED000AB5EE400A0B
:10175000F1EE10FA01DCB1EE400A324ADFED2F0A59
:10176000B4EE600AF1EE10FA08DBD37B5B1CD37396
:10177000DBB2FE2B04DB3223D37301E00346D373C9
:1017800091ED010AB5EE400AF1EE10FA01DCB1EE7E
:10179000400AB4EE600AF1EE10FA08DB137C5B1C21
:1017A0001374DBB2FE2B04DB3223137401E0034617
:1017B000137491ED020AB5EE400AF1EE10FA01DC65
:1017C000B1EE400AB4EE600AF1EE10FA08DB517C8B
:1017D000491C5174C9B2FE2904DB3221517401E065
:1017E00001465174D17B322905DA117C322902DAA3
:1017F000517C322900DB0120704700009A99993E04
:1018000001009040010080400000C84300001643E2
:1018100001005C428096184BB41C002035336B41AC
:10182000BC250020341D00202DE9F24F2DED048B46
:1018300084B004469FEDE58ADFEDE48A9FEDE39AEC
:10184000DFF8405BE888ADF80800A888ADF8020032
:1018500028898DF8000000273E462046FFF718FF34
:1018600001902046FFF76EFF8246DFF888873046FA
:10187000C8F85400C8F85800D8F86800DFF8089B8A
:10188000D9F8141900EE101AD4ED000A30EEC01A7F
:1018900001EE900AF8EEE11A21EE211AB5EE401A97
:1018A000F1EE10FA1ED598ED1D1A70EE411AF5EE04
:1018B000401AF1EE10FA01DC71EE401A9FEDC41AE5
:1018C000F4EE411AF1EE10FA07DB296F491C296783
:1018D000D8F85C10491CC8F85C1088ED1D0A40421D
:1018E000C8F8680009F6141090ED010AD8F86C10D9
:1018F00094ED011A31EE401A01EE901AF8EEE11A59
:1019000021EE211AB5EE401AF1EE10FA1ED598ED2F
:101910001E1A70EE411AF5EE401AF1EE10FA01DCD3
:1019200071EE401A9FEDAA1AF4EE411AF1EE10FA88
:1019300007DB2A6F521C2A67D8F86020521CC8F8AF
:10194000602088ED1E0A4942C8F86C1090ED020A2A
:10195000D8F8700094ED021A31EE401A01EE900AA8
:10196000F8EEE11A21EE211AB5EE401AF1EE10FA66
:101970001ED598ED1F1A70EE411AF5EE401AF1EEE1
:1019800010FA01DC71EE401A9FED911AF4EE411A43
:10199000F1EE10FA07DB296F491C2967D8F86410AB
:1019A000491CC8F8641088ED1F0A4042C8F870004E
:1019B00098F80000052809D10120C8F840003046F9
:1019C00088F80000A8F80200A8F80400D8F84C0035
:1019D00008990818C8F84C00D8F83400D8F8441012
:1019E000884202D10120C8F84000D8F8380000EB46
:1019F000400109EB810B0BF6C000C0ED000A6168E5
:101A00004160A16881600899204600F029FA686168
:101A10000198012802D0BAF1010F32D19FED6B0A73
:101A2000DBF8C00800EE900A60EEA00ADBF8C408FC
:101A300001EE100A21EE011ADBF8C80801EE900A47
:101A400061EEA11ADFF84409017B322904DAC17B77
:101A5000322901DA30EE800A417B322904DA017C36
:101A6000322901DA30EE010A817B322904DA407C26
:101A7000322801DA30EE210A00F094FCF0EE409AB0
:101A800037E00BF50C60D0ED020A90ED011ADBF89F
:101A9000C00800EE100A20EE000A01EE010A00EE76
:101AA000A00A00F07FFCF0EE409AD4ED010A94ED1C
:101AB000000A20EE000A00EEA00A00F073FCB0EE6F
:101AC000408AD4ED020A94ED010A20EE000A00EEED
:101AD000A00A00F067FCF0EE408AD4ED020A94ED13
:101AE000000A20EE000A00EEA00A00F05BFCB0EE57
:101AF000409AD8F83C0000282ED130460CE009EB83
:101B00008001C1ED159A09EB800282ED008AC1EDDA
:101B1000078A81ED0E9A401C0728F0DBB1EE0C0A13
:101B200069EE800AC8ED090AD8F80C00C8F8180058
:101B3000D8F81000C8F81C00D8F81400C8F8200025
:101B400068EE000AC8ED030A68EE800AC8ED040AD0
:101B500029EE000A88ED050AD8F8380009EB800163
:101B600091ED150A39EEC00AD8ED090A30EE200AC7
:101B700088ED090AC1ED159AD8F8340009EB800008
:101B800080ED230AD8ED0B0A70EE800AC8ED0B0A2F
:101B9000D8F80C20C8F81820D8F81020C8F81C2055
:101BA000D8F81420C8F82020D8F8382009EB820291
:101BB00082ED008AC1ED078A81ED0E9A3246DFED93
:101BC000030A9FED021ADFED011A12E00000000087
:101BD000CECC4C3E09EB820393ED002A70EE820AD4
:101BE00093ED072A31EE021A93ED0E2A71EE821A56
:101BF000521C072AEEDBC8ED030A88ED041AC8ED73
:101C0000051AD1ED1C0A70EE600A00F27442C2EDB2
:101C1000000A81ED1C0A98ED0C0AD0F8741400EE4D
:101C2000901A30EE200A88ED0C0A09F6141194EC93
:101C3000030A81EC030ADFF85417096F01290AD15E
:101C40000120C8F84000304688F80000A8F80200DB
:101C5000A8F804007EE0D8F85010491CC8F85010CD
:101C600098F80020012A01D0032A3AD102292BD268
:101C7000EA8D042A28DAE96C00296BD198ED0A0A6A
:101C8000DFEDDA0AB4EE600AF1EE10FA08D5D0F80A
:101C9000741401EE101AB4EE601AF1EE10FA0FDAB5
:101CA000F9EE0C0AB4EE600AF1EE10FA52DBD0F84D
:101CB000740400EE100AB4EE600AF1EE10FA49D591
:101CC0000120C8F8400045E027290AD3B8F80220CF
:101CD000002A03D011FA82F14B2902D30121C8F85E
:101CE0004010D0F8740400EE900A98ED0A0A00F053
:101CF00083F998F8000001282CD1B8F802000028D8
:101D000028D0B8F80410002924D0032211FA80F05A
:101D10003D2802DB0120C8F84000E88D042800DBE4
:101D20000222B8F80600824202D20120C8F8400020
:101D30003046C8F86400C8F86000C8F85C00FEF7D8
:101D4000FBFA0746286F686730462867A8F8040042
:101D5000A8F80600D8F83400D8F84810401AFA302D
:101D6000FA242146B0FBF1F104FB1100B8F80A1087
:101D7000884201D100F031FAD8F83400D8F8481080
:101D8000401AFA302146B0FBF1F104FB110064283F
:101D900001D100F063FAE888BDF80810814204D14F
:101DA000BDF80210AA88914200D00126002814D064
:101DB000D8F83400D8F84810401AFA302146B0FB61
:101DC000F1F104FB1101322902D10120288116E032
:101DD0004B2914D10020288111E0A88800280ED0BA
:101DE000D8F83400D8F84810401AFA302146B0FB31
:101DF000F1F104FB11007D2801D1012028819DF81B
:101E000000002989884200D00126D8F8340009EB67
:101E10008001D1F87414C8F82810401CC8F83400A8
:101E2000FA2802D10020C8F83400D8F83800401C45
:101E3000C8F83800072802D10020C8F83800D8F8C0
:101E40003C00401CC8F83C0047EA0600401E8041A8
:101E5000C043C00F04B0BDEC048BBDE8F28F00009E
:101E600030B4DFF8243590ED000AD3F8142900EEE1
:101E7000902A30EE600A03F61412D0ED010A92EDBA
:101E8000011A70EEC10A90ED021AD2ED021A31EE7B
:101E9000611AB5EE400AF1EE10FA02DDF0EE401ADA
:101EA00001E0F1EE401AF5EE400AF1EE10FA02DD23
:101EB000B0EE602A01E0B1EE602AB5EE401AF1EE14
:101EC00010FA02DDF0EE412A01E0F1EE412A71EE56
:101ED000821A71EEA21AB5EE400AF1EE10FA01DC98
:101EE000B1EE400ADFF8A40490ED072A32EE000AB2
:101EF00080ED070AF5EE400AF1EE10FA01DCF1EE92
:101F0000600A90ED080A30EE200A80ED080AB5EE6E
:101F1000401AF1EE10FA01DCB1EE411A90ED090A17
:101F200030EE010A80ED090A90ED0A0A30EE210A2E
:101F300080ED0A0A2F4AD46B002C12D1002406E04F
:101F400003EB850505F67C05C5ED001A641CA4B2FB
:101F500025460F2DF4DBB2EE0E0A21EE800A80ED4D
:101F6000150A148903EB8403D3F87C5800EE105A49
:101F700031EEC00AD0ED150A30EE200A80ED150AC8
:101F800003F67C03C3ED001AF2EE0E0A80EE200A7F
:101F9000DFF8F03383ED1B0AD0ED170AB4EE600AC8
:101FA000F1EE10FA01D580ED170AD0ED180AF4EE23
:101FB000400AF1EE10FA01D580ED180ADFEDA50A0E
:101FC000B4EE600AF1EE10FA03D5836DC91881658D
:101FD00001E000218165611C118189B20F2901D1C5
:101FE00000211181806D30BC704700000100E0408D
:101FF000681E0020341C00209FED971ADFF8840330
:10200000C08D042801DBB0EE001ADFF88403B5EEC2
:10201000400AF1EE10FA07DBF5EE400AF1EE10FA95
:1020200002D5C188491CC1800178002905D0022948
:1020300060D02DD3032976D0B0E0F1EE0C1A31EE4A
:10204000211AB4EE401AF1EE10FA0BDBB4EE601A6E
:10205000F1EE10FA06D5016D1029C0F08F80002135
:1020600001658BE0416BDFF8202302EB8101D1F8A1
:10207000741401EE901ADFF81C1391ED010AF4EECE
:10208000401AF1EE10FA40F18980C1ED011A85E0A5
:10209000416BDFF8F42202EB8101D1F8741401EEF8
:1020A000901ADFF8F01291ED002AB4EE612AF1EEF9
:1020B00010FA01D5C1ED001AF7EE001AB4EE610A6C
:1020C000F1EE10FA6ADBB7EE000AF4EE400AF1EE28
:1020D00010FA63D5016D418000210165B9EE0C0A4B
:1020E00030EE410AF4EE400AF1EE10FA10D402216B
:1020F000017053E0F9EE0C1A31EEC11AB4EE410A48
:10210000F1EE10FA4ADBF4EE410AF1EE10FA45D591
:10211000032101709C49426B01EB8201D1F87414D8
:102120009C4A51603AE0416B974A02EB8101D1F839
:10213000741401EE901A974991ED012AF4EE421AB7
:10214000F1EE10FA01D5C1ED011ADFED7B1AB4EE04
:10215000610AF1EE10FA21D5F4EE610AF1EE10FAFF
:102160001CDB016D818000210165B1EE0C0A31EEAE
:10217000000AB4EE600AF1EE10FA0ED501210170EA
:1021800084490A6842654A6882657F4A436B02EB6C
:102190008302D2F874240A6000E00170007870476E
:1021A000002803D077492C2200F056B97047002848
:1021B00006D0764942684A6002680A60007A08726E
:1021C000704780B5002801D1002002BD542201468D
:1021D000714800F041F9012002BD10B5694CE08D55
:1021E000A18D002904D0002802D00020208106E023
:1021F000084302D00120208101E00220208100203C
:10220000E0646062A061A080A08520636065A06535
:1022100002464021614800F0E1F8E06F012801D159
:10222000FEF744FD5948818A002909D0E28E8A428E
:1022300001D2A18600E0A286002181820846A06723
:10224000A06F012801D1E08EA0860020A06710BDFC
:1022500000000000EC51383E0000000010B5494C71
:10226000E08DA18D002904D0002802D0002020811B
:1022700006E0084302D00120208101E002202081F5
:1022800000206062A061E085E080024608214448A9
:1022900000F0A4F800202063E06F012801D1FEF7D0
:1022A00005FDA06F012801D1E08EA08610BD80B58C
:1022B000012036490867FFF7D1FFFFF78EFFBDE821
:1022C000014003E000203149086770472F48008B28
:1022D0002C49898E814200D200E070472949CA6C9E
:1022E0008B8E9A4203D288860020886770472749E0
:1022F000888270472348C16C002904D1018E408E2A
:1023000010FA81F070470020704701460020002934
:1023100002D0012901D0704702E01A48C06C704712
:102320001848818EC26C891A028E891A408E081A4A
:1023300000D5002070470000FEFF7FBF38B504467F
:102340001348124D0F49012C06D10622CA860C22D1
:102350002A839622428105E00722CA860F222A8319
:1023600064224281E88AA04209D0888E082803DAD4
:10237000C88EFFF7B3FF02E0288BFFF7AFFFEC82B8
:1023800031BD0000B41C0020BC250020341D0020FD
:10239000341C0020AC700020681E0020E86E002075
:1023A000742E002081B08DED000A0098401000F1DD
:1023B000FE500090DDED000AC0EE200A9DED001AEF
:1023C00070EE810ACDED000AB5EE001ADDED001ABF
:1023D00080EE210A00EE810A01B0704762F30F22FD
:1023E00062F31F4200B500BF1300964694461039B1
:1023F00028BFA0E80C50FAD85FEA417C28BF0CC087
:1024000048BF40F8042BC90728BF20F8022B48BF5B
:1024100000F8012B00BD50F8041B61B150F8042BEB
:10242000D30744BFA9F101039A180023091F42F8FA
:10243000043BFAD1EFE7704762B38B0708D0521E16
:1024400011F8013B00F8013B00F024808B07F6D126
:10245000830740F0208000BF103A07D330B4B1E8C2
:102460003810103AA0E83810F9D230BC530724BF16
:10247000B1E80810A0E8081044BF51F8043B40F848
:10248000043BD20724BF31F8022B20F8022B44BFB3
:102490000B7803707047083A07D3B1E80810083A80
:1024A00040F8043B40F804CBF7D25307E4E78268D6
:1024B000521C8260426832B10268531C0360117082
:1024C0004168491E416070470022FFF78BBF0268D8
:1024D000531C03601170704762F30F2262F31F42B6
:1024E000401810F0030308D0C91A1FD3DB0748BFF8
:1024F00000F8012D28BF20F8022D130030B4144637
:102500001546103928BF20E93C00FAD8490728BFF2
:1025100020E90C0048BF40F8042D890028BF20F8AE
:10252000022D48BF00F8012D30BC7047C91818BFF4
:1025300000F8012DCB0728BF00F8012D70470000DF
:1025400010B5DFF8344D04F1AC01012001F0A2FB1D
:10255000002805D00FF2480002F0CAF8032010BD91
:102560000FF2500002F0C4F8002060732087E0648E
:1025700002464421DFF8040DFFF730FF01223C2121
:10258000AA2002F09EFA00202074A073E063A065E8
:10259000A4F84000A07400F0B7FD002010BD0000BA
:1025A00050443A204641494C20524547494C494203
:1025B0005648000050443A20537461727450656468
:1025C0006F2D30383232000080B5DFF8481D012011
:1025D00001F0A1FB002801D0032002BD002002BDB4
:1025E000F0B587B003A80FF24C1191EC030A80EC10
:1025F000030A0FF24C100068029003A9012001F0B9
:1026000013FD02A9062001F00FFD02F046FE441E54
:10261000A441E40F02F03BFE012801D1012000E0BB
:102620000020DFF8F45C6978A14200D06C70297852
:10263000814200D02870DFF8406C06200020C046A0
:10264000002816D1DFF8D40C02900020F063B6F811
:102650004000401CA6F8400080B240F2EF218842C2
:102660004BDB0FF2E00002F043F80020A6F8400038
:1026700043E096F90800022838D19DED020AD6ED14
:10268000160AB4EE600AF1EE10FA03D1B08F401CC6
:10269000B08701E00020B0879DED020ADFED890AD6
:1026A000B4EE600AF1EE10FA06D4DFED870AB4EE5C
:1026B000600AF1EE10FA03DBF08F401CF08701E0B6
:1026C0000020F087F78FB48F972C01DA972F0FDB5C
:1026D000029802F011FFCDE900013A4621460FF2BF
:1026E000780002F005F80020F06301E00020F063BC
:1026F0000020A6F840000298B065706C006AC468BB
:1027000002F06DF930722046DDED021A03A991EC5A
:10271000030A02F095F8B06C2018B06495F9010036
:1027200000F03AFB002801D000F0D0F8002007B0FC
:10273000F0BD0000000000000000000000000000EC
:102740000000000050443A204261726F4469736196
:10275000626C65640000000050443A204241524FD0
:1027600020256420256420256600000010B5DFF8D0
:10277000084B94F9000000283AD494F90A0094F91F
:102780000110814228D1217B0818A07240B23D2857
:1027900001DB3C38A07294F90A100FF2700001F0CE
:1027A000A7FF0020A064DFF8780C90F9010010F179
:1027B000010F01D1012010BD94F90110081A02F097
:1027C000C3FE21F0004102F0D7FE40B2012801DB38
:1027D000012010BD002010BDDFF8D80C90F90120B9
:1027E000914203D0D4E90023C0E90023002010BDAA
:1027F000A06CDFF8541D884205DB0FF21C0001F0CD
:1028000077FF012010BD002010BD000050443A2089
:102810004E5420256400000050443A204E6F546905
:102820006D6500002DE9F8430026DFF84C4A02E010
:10283000207B4019A07294F90A50002E1DD46078B4
:10284000461B76B2012EF3DA002E16D094F90C70E6
:10285000304602F079FE21F0004102460B469046D8
:102860009946384602F070FE42464B4602F0B0FEF2
:10287000E1D2E81BA0720026DDE73C2D02DBA5F1CA
:102880003C00A072BDE8F18380B5DFF8EC090021BF
:10289000817301210172002141724FF0FF310170FB
:1028A0000F21C17214210173002141730187C1649A
:1028B0004174016541650A4624211430FFF78EFDFD
:1028C000002002BD0000FA430180BB4430B5A5B032
:1028D0000AA85821FFF7F8FD00A82821FFF7F4FD0A
:1028E00020A81421FFF7F0FD0AA800F035FEDFF85C
:1028F0005C4C9DF8290020709DF829000146C029F4
:1029000006D113A9C88DA4F85E00086B2066E9E023
:10291000E02953D100203FE00AA901EB8001D1F862
:102920000220130223F0FF13120A02F0FF121A43CF
:10293000C1F802204FEA3242C1F80220D1F8062045
:10294000130223F0FF13120A02F0FF121A43C1F818
:1029500006204FEA3242C1F80620D1F80A201302BD
:1029600023F0FF13120A02F0FF121A43C1F80A20E3
:102970004FEA3242C1F80A20D1F80E20130223F0A8
:10298000FF13120A02F0FF121A43C1F80E204FEA99
:102990003242C1F80E20001D1428BDDB50210FF279
:1029A0007C1001F0A5FE50220DF12A01601CFFF7FA
:1029B00043FD5120A4F85E00246693E0000633D462
:1029C0009DF82A008DF8800020A89DF82B104170FA
:1029D000002181709DF82C10C170BDF833100A0AD7
:1029E000027141710DF133018A788271C978C17128
:1029F0009DF8371001729DF8381041729DF82D1026
:102A000081729DF82E10C1729DF82F1001739DF8F0
:102A1000301041730E2220A9601CFFF70DFD0F201E
:102A2000A4F85E0024665DE0DDF82A10080C8DF83D
:102A3000000000A80A0A42708170DDF82E100A0C0E
:102A4000C2700A0A02714171DDF832100A0C8271FB
:102A50000A0AC2710172DDF836100A0C42720A0AC3
:102A60008272C17213990A0C02730A0A427381734B
:102A700013A90A79C2734A790274CA88130A8DF8B5
:102A800011308274097A8DF81310DDF83A100A0CAF
:102A900002750A0A8DF815208175DDF83E100A0CC2
:102AA0008DF817200A0A8DF818208DF81910DDF816
:102AB00042100A0C82760A0A8DF81B208DF81C1031
:102AC000DDF846100A0C8DF81D200A0A82778DF871
:102AD0001F10202200A9601CFFF7AEFC2120A4F8E3
:102AE0005E002466DFF89007406CB4F85E20D11CCD
:102AF000418200218182C182DFF8585A012028706A
:102B000068700320A870216EE81CFFF795FC294629
:102B1000262001F0B5F925B030BD00005044205307
:102B2000462053656E7425640000000038B5DFF858
:102B300048374FF46164C1EB0115AD0014FB00543C
:102B400014194FF47A756C43DC611B7C00931346B7
:102B50000A4601460FF2080001F0CAFD31BD00002F
:102B600050443A20425420256420256420256420C6
:102B700025640000F8B52DED028BA0B0DFF8FC66EF
:102B8000314684B068464422FFF766FC0FBC00F073
:102B900093FC10EE100A02F0AFFC41EC100B9FED1D
:102BA0007C8BDFF8D446256A53EC102B51EC180BC4
:102BB00002F026FD02F0E0FC15FA80F020624FF6EC
:102BC000FF75A84200D32562314684B0684644228E
:102BD000FFF742FC0FBC00F025FC10EE100A02F0DB
:102BE0008BFC41EC100B676A53EC102B51EC180B6B
:102BF00002F006FD02F0C0FC17FA80F06062A84205
:102C000000D3656200200E9002200D90314684B002
:102C100068464422FFF720FC0FBC00F08BFAE18AE3
:102C20004018E08280B2FF2801DBFF20E082002014
:102C30000E9003200D90314684B068464422FFF781
:102C40000BFC0FBC00F076FAA16A4018A062A84203
:102C500000D3A56200200E9006200D90314684B06E
:102C600068464422FFF7F8FB0FBC00F063FA218BA3
:102C70004018208380B2FF2801DBFF202083002042
:102C80000E9007200D90314684B068464422FFF72D
:102C9000E3FB0FBC00F04EFA618B4018608380B2FA
:102CA000FF2801DBFF20608300200E9008200D909C
:102CB000314684B068464422FFF7CEFB0FBC00F0DB
:102CC00039FAE16A4018E062A84200D3E5620020C8
:102CD0000E9009200D90314684B068464422FFF7DB
:102CE000BBFB0FBC00F026FA216B40182063A84202
:102CF00000D325630FA801F076FE276D1E9802F021
:102D0000FBFB0022DFF8003D02F07AFC02F034FC0D
:102D100057FA80F02065616D491C6165B0FBF1F0E8
:102D2000207500200E9001200D90314684B0684639
:102D30004422FFF791FB0FBC00F0FCF9616B4018D7
:102D40006063A84200D36563E07B00F0E9FA20B03D
:102D5000BDEC028BF1BDDFF82005C18A002914D13A
:102D6000816A002911D1018B00290ED1418B0029E4
:102D70000BD1C16A002908D1016B002905D1406B34
:102D8000401E8041C043C00F7047012070470000C3
:102D900000000000000059402DE9F04FA1B00646A8
:102DA0000025B246DFF8D044A07B3146884205D0EA
:102DB000BAF1010F78D1284602F0BAF90FA801F054
:102DC00012FEDFF8B89428460E9001200D90494677
:102DD00084B068464422FFF73FFB0FBC00F0AAF91D
:102DE00007469DED1E0AD9ED0F0A30EE600A10EE7F
:102DF000100A02F081FB2A46DFF80C3C02F000FCCE
:102E000002F0BAFB80461FFA88F8B9F80200BDF854
:102E10003E10A1EB000B5FFA8BFBD9F81020139B3F
:102E20009A4207D1884205D1B9F80A00BDF8461088
:102E3000884210D00FF27022D2E90001CDE90001E2
:102E4000139800901398D9F81010401A019000A917
:102E5000472001F015F8002E36D1002F02D15BEA91
:102E6000080000D001250020A0644FF0FF30207042
:102E7000D4E90001DFF83C26C2E90001DFF8782C34
:102E8000C2E90001DFF89825C2E90001E07AA072EA
:102E9000A07B002851D00020A073207C00284CD0BB
:102EA00001206074054648E0002E07D10FF2002093
:102EB00001F01EFC012002F03BF97FE70FF2FC104D
:102EC00001F016FC2846EBE00FF20C22D2E90001DB
:102ED000CDE9000100A802F0F6F900F0B7F90028EA
:102EE00017D0DDE90001C4E9000128466072D4E989
:102EF0000001DFF8C025C2E9000194F9023094F91D
:102F0000012094F900100FF2D81001F0F1FBFFF747
:102F100089FCDDE90001C4E90001FFF727FC002876
:102F20000BD0D4E90001DFF8F824C2E90001207CCD
:102F3000002801D0012060740125BAF1010F06D1EB
:102F4000A07B3146884202D000F057FAA673BAF14E
:102F5000010F56D1002F54D0DFF89C6BE07B217C11
:102F600008430AD101202074D4E90001C6E9020116
:102F7000A27861782078FFF7D9FD94F9010096F9DD
:102F80000910401A411E222901D2012005E010F14A
:102F9000230F01DA012000E0002001282AD1FFF7E9
:102FA000DAFE002826D0E07B401CE073C0B2152872
:102FB00009D10FF2441001F09BFB01206074142032
:102FC000E073012516E0002020656065024624219B
:102FD00004F11400FFF702FA207C401C2074A27850
:102FE00061782078FFF7A2FD0622214606F108004D
:102FF000FFF732FAFFF7BEFD44220FA94846FFF75C
:103000002BFA607B012834D1208F002805D10FF6E0
:10301000443001F06DFB012523E0E16C814218D2C0
:10302000002F02D15BEA080000D00125DFF8C86A52
:1030300096F9020094F90220904212D0491CE164F2
:103040000FF6243001F054FBD4E90001C6E9000179
:1030500007E0002060732087E0640FF61C3001F069
:1030600047FBBAF1010F04D1207C002801D00120D8
:1030700060742846012801D10021A164616C496A6D
:10308000002906D10021A164012801D100F0B5F981
:103090000025002D03D1A07C012800D10125284660
:1030A00021B0BDE8F08F000000000000000000002B
:1030B00050443A206C63646F6E00000050443A2024
:1030C0006249734150536C656570696E6720777211
:1030D0006F6E672025640000000000000000000003
:1030E00050443A2054696D654E6F74692025642000
:1030F000256420256400000050443A2042542042B8
:10310000462046554C4C000080B500205A49886442
:1031100000F002F8002002BD00B591B000A801F057
:1031200062FC442200A95548FFF796F9012011B02E
:1031300000BD00000FB410B592B000249DF99800B6
:1031400001280BD101F038FD1899884202D3441AA6
:10315000E4B271E08038441AE4B26DE000A801F0F6
:1031600042FC9DF99400401E082865D8DFE800F075
:103170002905111D2935414D590005981999884295
:1031800001D3441A58E0DFF878291018401A441C7B
:1031900052E006981A99884201D3441A4CE0DFF8AD
:1031A00060291018401A441C46E007981B99884271
:1031B00001D3441A40E0DFF848291018401A441C93
:1031C0003AE004981899884201D3441A34E0DFF8B1
:1031D00030291018401A441C2EE008981C99884287
:1031E00001D3441A28E0DFF818291018401A441CAB
:1031F00022E009981D99884201D3441A1CE0DFF8A7
:1032000000291018401A441C16E00A981E9988429A
:1032100001D3441A10E0DFF8E8281018401A441CC3
:103220000AE00B981F99884201D3441A04E0DFF8A2
:10323000D0281018401A441C204612B010BC5DF86B
:1032400014FB0120DFF8BC18487270470A48407A26
:10325000704701F0D2BB0146DFF8A828792902DBCC
:103260007820108700E01087012050730FF61C10A3
:1032700001F03EBA00000000641B0020A46E002094
:1032800010B5040001D1012402E0072C00DB062464
:1032900021460FF60C1001F02BFA641E052C2DD8D8
:1032A000DFE804F0030A11181F26DFF85808372159
:1032B000C1723C21017321E0DFF848081921C17275
:1032C0001E2101731AE0DFF83C080F21C17214219E
:1032D000017313E0DFF82C080A21C1720F2101737A
:1032E0000CE0DFF820080721C1720C21017305E012
:1032F000DFF810080521C1720A210173DFF8040804
:10330000C17A8172BDE81040FFF78CBADFF8F80788
:1033100070470000101C00200071002000007A445B
:1033200000EB80018800821CDFF8DC07DFF8D4178F
:10333000CB691B0E92B21354521CCB691B0C92B278
:103340001354521CCB691B0A92B21354521CCB6902
:1033500092B21354521C0B6A1B0A92B21354521CA1
:103360000B6A92B21354521C4B6A1B0A92B213544A
:10337000521C4B6A92B21354521CCB8A92B2135411
:10338000521C8B6A1B0A92B21354521C8B6A92B263
:103390001354521C0B8B92B21354521C4B8B92B28F
:1033A0001354521CCB6A1B0A92B21354521CCB6AA0
:1033B00092B21354521C0B6B1B0A92B21354521C40
:1033C0000B6B92B21354521C0B7D92B21354521CCD
:1033D0004B6B1B0A92B21354521C4B6B92B2135498
:1033E000501C4887704710B5DFF81847618F0FF2FF
:1033F000BC7001F07DF9608F10BD10B5DFF8044797
:103400000022242104F11400FEF7E8FF0020E073FD
:1034100001206087002020742065606510BD0000D9
:10342000A47000200FB400B591B000A801F0DBFA41
:103430009DED0C0ADDED1E0AB4EE600AF1EE10FA05
:1034400002DB30EE600A05E09FED411A71EE600A82
:1034500030EE800A10EE100A02F04EF8DFF8AC26CB
:10346000DFF8AC3602F09EF902F010FA02F044F8F0
:103470000022DFF8A03602F0C3F802F07DF800EE7B
:10348000100AB8EEC00A10EE100A02F035F8DFF8A4
:103490007C26DFF8843602F0B3F8DFF88026DFF808
:1034A000803602F07FF902F0F1F900EE100A11B057
:1034B0005DF814FB9C7000200FB400B591B000A81B
:1034C00001F091FA9DED0E0ADDED200AB4EE600ADE
:1034D000F1EE10FA02DB30EE600A05E09FED1C1AF7
:1034E00071EE600A30EE800A10EE100A02F004F865
:1034F000DFF81826DFF8183602F054F902F0C6F9A2
:1035000001F0FAFF0022DFF80C3602F079F802F041
:1035100033F800EE100AB8EEC00A10EE100A01F0FF
:10352000EBFFDFF8E825DFF8F03502F069F8DFF8A7
:10353000EC25DFF8EC3502F035F902F0A7F900EEE2
:10354000100A11B05DF814FB40771B008C6D002051
:10355000002474494C63002070B52DED068BA0B09B
:1035600004460FA801F03FFADFF89855687B012860
:1035700004D1288F002801D100206873A87C01287D
:103580000AD1E0206070502205F15C01A01CFEF71A
:1035900053FF0020A874C2E1687C012816D1287C62
:1035A000002813D0C0216170DFF85C15C0220A70BA
:1035B000487004F12406FFF716FFF085FFF7A6FE1A
:1035C0003063FFF71AFF00206874A8E19FEDD68BE7
:1035D0009FEDD79BDFF84C5500200E9001200D90F9
:1035E000294684B068464422FEF736FF0FBCFFF739
:1035F000A1FD0A2880F0BE80002060700E9002209D
:103600000D90294684B068464422FEF725FF0FBC82
:10361000FFF790FD61780843607000200E90032052
:103620000D90294684B068464422FEF715FF0FBC72
:10363000FFF780FDA07000200E9004200D90294619
:1036400084B068464422FEF707FF0FBCFFF772FD07
:10365000E07000200E9005200D90294684B0684649
:103660004422FEF7F9FE0FBCFFF764FD20712946E6
:1036700084B068464422FEF7EFFE0FBCFFF71CFF44
:1036800010EE100A01F038FF41EC100B53EC102B38
:1036900051EC190B01F0B4FF01F06EFFA4F80B0020
:1036A00004F10B061E9801F027FF53EC182B01F0D4
:1036B000A7FF01F061FFB070BDF83E00F070294631
:1036C00084B068464422FEF7C7FE0FBCFFF7AAFE8F
:1036D00010EE100A01F010FF41EC1A0B53EC1A2BFC
:1036E00051EC190B01F08CFF01F046FFE0731F98BD
:1036F00001F002FF53EC182B01F082FF01F03CFFB8
:10370000207400200E9006200D90294684B0684653
:103710004422FEF7A1FE0FBCFFF70CFD60710020F4
:103720000E9007200D90294684B068464422FEF78B
:1037300093FE0FBCFFF7FEFCA07100200E90082046
:103740000D90294684B068464422FEF785FE0FBCE2
:10375000FFF7F0FCE07100200E9009200D90294643
:1037600084B068464422FEF777FE0FBCFFF7E2FC08
:103770002072D2E08020607000200E9002200D9018
:10378000294684B068464422FEF766FE0FBCFFF768
:10379000D1FCC4F8020000200E9003200D902946B1
:1037A00084B068464422FEF757FE0FBCFFF7C2FC08
:1037B000C4F8060000200E9004200D90294684B025
:1037C00068464422FEF748FE0FBCFFF7B3FCC4F87E
:1037D0000A0000200E9005200D90294684B068460E
:1037E0004422FEF739FE0FBCFFF7A4FCC4F80E001C
:1037F000294684B068464422FEF72EFE0FBCFFF730
:103800005BFE10EE100A01F077FE41EC100B53EC5A
:10381000102B51EC190B01F0F3FE01F0C3FE6062B6
:1038200004F124061E9801F067FE53EC182B01F0FA
:10383000E7FE01F0A1FE3071BDF83E00707129462F
:1038400084B068464422FEF707FE0FBCFFF7EAFD8E
:1038500010EE100A01F050FE41EC1A0BDFF8C822FE
:10386000DFF8C83202F05AF808D8DFF8C422DFF8CF
:10387000C43201F0ADFE01D29FED64AB53EC1A2BC4
:1038800051EC180B01F0BCFE01F076FEF0801F98A1
:1038900001F032FE53EC182B01F0B2FE01F06CFE89
:1038A000307200200E9006200D90294684B06846A4
:1038B0004422FEF7D1FD0FBCFFF73CFCC4F8120018
:1038C00000200E9007200D90294684B068464422BF
:1038D000FEF7C2FD0FBCFFF72DFCC4F81600002058
:1038E0000E9008200D90294684B068464422FEF7C9
:1038F000B3FD0FBCFFF71EFCC4F81A0000200E90A9
:1039000009200D90294684B068464422FEF7A4FDA4
:103910000FBCFFF70FFCC4F81E00FFF7FDFB20B043
:10392000BDEC068B70BD00000000000000002440CC
:10393000000000000000594070B582B0044600202D
:10394000002C05D10FF2782000F0D2FE002076BDC9
:1039500004F150014978012948D10FF2782000F094
:10396000C7FE0020ADF80000734D664E17E0BDF8AD
:10397000000006EB8000C26500EE102AB8EE400A97
:10398000DFED5E0A20EE200ABDF8000005EB8000A6
:1039900080ED000ABDF80000401CADF80000BDF845
:1039A000000014281CDABDF8000054F82020A2F50D
:1039B0002F70B0F5167FDAD9BDF800100FF2202075
:1039C00000F096FEBDF800004FF07E5145F8201043
:1039D0004FF47A70BDF8001006EB8101C865D9E795
:1039E00001202865284601F0A5FB0BE0022909D13A
:1039F00094F850100FF2FC1000F07AFE94F850008A
:103A00000120C046C0B276BD000024409A99999921
:103A10009999B93F80B5112802D11078FFF71BFCA6
:103A2000002002BD30B595B0144610281FD01428D0
:103A30000AD015280DD0162810D0172813D0292801
:103A400043D1FFF7FEFB40E021780020FFF701FCA7
:103A50003BE021780120FFF7FCFB36E021780220D3
:103A6000FFF7F7FB31E02078FFF70AFC2DE000A814
:103A70005421FEF729FD217814AD69700FF2C000C2
:103A800000F036FE6878012817D100200FE004EB23
:103A900080014A788B781B0403EB0262CB7802EB3F
:103AA00003220979511800AA42F82010401C14285A
:103AB000EDDB00A8FFF740FF07E0022805D16078A2
:103AC0008DF8500000A8FFF737FF002015B030BD7B
:103AD0000C494864B831C16126210170142181600C
:103AE000012101730182002141828182C182134937
:103AF00081610020704700004C7000206F12833AF3
:103B000080969800641B0020886100207B14AE47DB
:103B1000E17A743F00005940E17A843F2D431CEB69
:103B2000E2361A3FA46E0020B81E85EB51B89E3FC6
:103B30009A9999999999B93F141E00204C630020D5
:103B400050443A2050726F70657274792053462049
:103B50002564000050443A20526571205065646F1E
:103B6000496E666F3100000050443A207574696DEB
:103B7000657220256400000050443A20526571208F
:103B80005065646F496E666F3200000050443A2001
:103B900053746172742044617461202564000000D4
:103BA00050443A20555420256400000050443A20E7
:103BB0004241544C454E47544820256400000000C3
:103BC00050443A2053462050545233206E756C6C4A
:103BD0000000000050443A20534620534554310021
:103BE00050443A205346204552525B25645D2025BF
:103BF0006400000050443A2053462053455432207C
:103C00002564000070B5002420E02C2001F09EFE09
:103C1000054600222C21FEF7E1FB28460FF2007139
:103C200051F826108847DFF8A066287846F820501B
:103C30000020E96909688847002806D00020297813
:103C400046F82100284601F099FE641CE4B226469D
:103C5000182EDADB002070BD10B46FF0004108466A
:103C6000002210E0DFF8603653F82230002B09D034
:103C70001C6A002C06D0DB78002B03D1E368984245
:103C800000DD1846521C622AECDB884200D100207D
:103C900010BC7047F8B506460F4600F0E4F8040083
:103CA00001D10320F2BD251D6868002801D0B8604D
:103CB0007860786801F044FB7860B968002902D028
:103CC000084601F03DFBB860394604F1200001F0E0
:103CD0005DFF94F82800012807D10020A9694968F0
:103CE000884701F0E3FF606008E0E078012805D133
:103CF0003878002802D1304602F052F800221146EE
:103D00002E20AB691B699847DFF8C015022002F02E
:103D100071F80020F2BD70B50D4600F0A4F8060061
:103D200007D006F11C04287800280AD1A0680028D2
:103D300001D1032070BDC0686860A0680069A860F8
:103D400007E0686801F0FCFA6860A86801F0F8FA1A
:103D5000A860294606F1200001F038FFF369207BB6
:103D6000002803D10020D968884704E000221146CA
:103D70002E201B699847DFF85415022002F03AF80C
:103D8000002070BD38B50C4600F06DF8054660683F
:103D900001F0D6FA6060A168002902D0084601F05F
:103DA000CFFAA060002D02D0686A002801D103205C
:103DB00032BDC1686268914205D10169A268914231
:103DC00001D1002032BD00F1080105F1200001F011
:103DD000FDFE002811D1214605F1200001F0D6FE9C
:103DE000002211462E20EB691B699847DFF8DC148E
:103DF000022001F0FFFF002032BD032032BDF8B5E4
:103E000004460D4616461F4600F02DF8002801D145
:103E10000120F2BD3A4631462846DFF8AC3453F86B
:103E20002430DB691B6998470020F2BDF8B50446D1
:103E30000D4616461F46192D03D1012102F00CF83C
:103E40000FE000F010F8002801D10120F2BD3A4641
:103E500031462846DFF8703453F82430DB695B695B
:103E600098470020F2BD0146622901DA002801D1FD
:103E700000207047DFF8500450F821007047000020
:103E800070B52DED028B0C46DFF83C1451F8205034
:103E9000012812D0042849D005286DD0082800F048
:103EA00097801D2800F0B280222879D0442800F0A5
:103EB000A580472800F0AF8021E09FED750ADFF86C
:103EC0001064B4F9000000EE900AF8EEE00A60EE2B
:103ED000800AC6ED000AB4F9020000EE900AF8EE7E
:103EE000E00A60EE800AC6ED010AB4F9040000EEB3
:103EF000900AF8EEE00A20EE800A86ED020A002D14
:103F000011D0686A00280ED04069DFF8C413C96D6B
:103F1000401A012807DA214605F1100001F0FEFFE2
:103F200001F0C4F96860BDEC028B70BD9FED598B48
:103F3000DFF89C63B4F9000001F006FB53EC182B8A
:103F400001F05EFB01F0A2FCF060B4F9020001F0A8
:103F5000FBFA53EC182B01F053FB01F097FC306196
:103F6000B4F9040001F0F0FA53EC182B01F048FB0F
:103F700001F08CFC7061C2E7D54E20687062606809
:103F8000B0622089B0856089F085A0893086E0899B
:103F90007086207C86F83400607C86F83500AEE7B9
:103FA000CB4E2068B0636068F0632089A6F84000BB
:103FB0006089A6F84200A089A6F84400E089A6F826
:103FC0004600207C86F84800607C86F8490096E729
:103FD000BF4E207886F84C00607886F84D00E08867
:103FE000A6F84E00686A00289DD0214605F1100011
:103FF00001F094FF01F05AF9686094E7B44E20682C
:10400000B0616068F061A068306278E72078B049FC
:1040100081F8500073E708222146AE48BDEC028BC0
:10402000BDE87040FEF708BA02460846012A0ED0E5
:10403000042A10D0052A12D0082A18D01D2A1ED012
:10404000222A10D0442A16D0472A1CD070470C22AE
:104050009F49FEF7F1B90C229F49FEF7EDB91422F2
:104060009E49FEF7E9B914229D49FEF7E5B90422FD
:104070009C49FEF7E1B90C229B49FEF7DDB901220C
:104080009A49FEF7D9B908229249FEF7D5B900003E
:10409000FDF61C3B0597A11D4F04443F10B50828B1
:1040A00002D010281FD010BD0120FFF7DCFE034610
:1040B000002211462F20DB691B6998472B20FFF750
:1040C000D2FE90F82800002801D002F03CFA11201E
:1040D000FFF7C9FE044694F82800002827D0BDE861
:1040E000104002F064BB0820FFF7BDFE044601F05B
:1040F000DDF86168401AE16989688847002816D1AF
:10410000606A002807D0C1680069814203D100219C
:10411000082001F0A1FE5B20FFF7A5FE044694F8FD
:104120002800002803D0BDE8104002F09DBC10BD5F
:104130002DE9F04385B0044601A80FF244212CC9B3
:104140002CC001F0B3F8054601F09BF8012801D11D
:10415000012600E000265E48C4650027DFF868817C
:1041600029E0622F20DADFF888910120BDF80710DE
:1041700001F80900022200A9BDF807004844401CCC
:10418000FEF75AF958F8270000F11001BDF80700B2
:104190004844C01C01F0EDFEBDF80700BDF800105A
:1041A000C91C0818ADF80700214658F82700203030
:1041B00001F029FD7F1C622F79DA58F827000028CA
:1041C000F8D090F828100029F4D0C1780029F1D156
:1041D000011DCA695269121B012A05DA4068281AB2
:1041E000401C89698968884758F82700416A002976
:1041F000DAD08969091B0129D6DA002E02D0017BA9
:104200000029D1D0103001F000FFADF8000058F8BF
:104210002700103001F01AFFADF80200BDF80000D1
:104220000028C1D0BDF802000028BDD0BDF80700AD
:10423000BDF8001011FA80F2101DB0F5007F0CDD02
:104240000FF2B0010FF2C00000F052FA284901A8A5
:1042500002F011FF0020ADF80700232FBFF681AF59
:10426000DFF88C903720BDF8071001F80900BDF881
:1042700007004844477002220DF10201BDF8070013
:104280004844801CFEF7D8F858F8270000F11001C8
:10429000BDF807004844001D01F06BFEBDF80700A3
:1042A000BDF80010091D0818ADF807007CE7BDF83F
:1042B0000700002803D00E4901A802F0DCFE002010
:1042C00005B0BDE8F083000010650020183700201D
:1042D000F06D0020446E0020FC6D0020146E002064
:1042E000286E00203C6E0020086E0020406E0020EA
:1042F000045A0020636F6C6C6563745F73656E7342
:104300006F725F646174610025733A2074785F6432
:104310006174612069732066756C6C2825642900BE
:1043200045A70108519A01081DA80108BB9D010875
:104330005DAA0108136F000827970108DBA8010890
:10434000798001087F65000863A50108D13A00085B
:104350001968000887A1010853A6010811990108EE
:10436000BBA201087B9401084F8D01086F7B0108F7
:104370002B920108A9A90108D5AA0108FB9F0108F1
:10438000050000000000000000000000EFF30380C3
:1043900070474FF0AC3000787047F8B507460C46D0
:1043A0000025DFF830646FF01E01401A27D008386E
:1043B00025D0001F10D0001F1AD0083818D0001FB9
:1043C00024D104F120003062EFF3148040F00200A9
:1043D000F062306AB06219E004F164003062EFF319
:1043E000148040F00200F062306AB06201250DE0F6
:1043F00004F120003062EFF31480F06206E004F173
:1044000064003062EFF31480F0620125EFF308805E
:104410007062EFF31080F063EFF311803064EFF31C
:1044200013807064F1EE100AB064EFF3058030631E
:10443000EFF300807063FFF7A9FFB063F76400201B
:1044400004E054F8201046F82010401C0828F8D347
:10445000012D0AD1002006E004EB8001096A06EB79
:1044600080021165401C1128F6D3F1BDDFF8680306
:10447000DFF868130A6802604A6842608A688260EE
:10448000CA68C2600A6902614A6942610A7E826141
:10449000097F8161DFF848130A7882614A684262C5
:1044A0008A688262CA68C2620A6902634A694263B0
:1044B0008A698263CA69C2638A6EC0F88820DFF89D
:1044C00024239369C0F89830D368C0F88C301369FE
:1044D000C0F890305369C0F894300B6FC0F89C302E
:1044E0004B6FC0F8A0308B6FC0F8A430C96FC0F814
:1044F000A810DFF8F4120968C0F8AC10DFF8EC126D
:104500000B68C0F8CC304B68C0F8D0308B68C0F86E
:10451000D430CB68C0F8D8300969C0F8DC105168D5
:10452000C0F8E8101168C0F8E410704710B582B008
:10453000044640F20240ADF8000005202070002043
:104540006070A070022200A9E01CFDF775FFDD205D
:10455000607113BD02F02ABFA0F10060B0F5003F0A
:1045600001D80120704700207047F8B505460E4677
:1045700014461F462868FFF7EFFF002801D10020EE
:10458000F2BD2868400840000090042030600246D8
:1045900000A938880019FDF74FFF0120F2BD2DE971
:1045A000F04182B080460C4615461E46002738462C
:1045B0000090B8F1000F19D0002C01D116E07F1C3B
:1045C0000C2F12D233462A4600A94046FFF7CDFFF2
:1045D000002803D0308800990818308030881428CB
:1045E00003DA08F104084445E9D20120BDE8F68168
:1045F000F8B50C46154610F1030F02D010F1130F59
:1046000009D17B4EB06802F0D9FE0746B06802F0CF
:10461000E1FEC11905E002F0EBFE064602F0EAFEFB
:1046200081192B4622466B48806AFFF7B8FF0120AC
:10463000F2BD80B50021ADF8001000AA0146654822
:10464000C06CFFF7D5FF01BD10B582B0044616203F
:10465000ADF800000520207000206070A0700222DC
:1046600000A9E01CFDF7E8FE0F2060711420A07186
:1046700013BD70B588B0724601461046FFF78DFE37
:10468000FFF7F4FE00A81C21FDF71EFF00A8FFF7AE
:10469000DBFF0DF10700FFF7CCFF1B2100A802F0A4
:1046A000FEFD0024534D2846FFF740FF40F2074629
:1046B0000CE0AC710A46A00200F10051E81DFDF7C4
:1046C000BBFE3146284602F0EAFD641C4FF48061CF
:1046D000202CEED30022E81DFDF7FEFEDD20A871A0
:1046E0003146284602F0DBFDFFF734FF08B070BD0D
:1046F0000EB470B5C1B0044600A84FF48071FDF748
:10470000E3FE45AB22464FF4807100A802F07AFE2A
:1047100000A802F095FE441C002000A9611801F8D1
:10472000010C334D2878401C28706878F02108422D
:1047300002D0992002F0A0FE02F014FF6878401C1D
:1047400068702D4E317808462218FA2A0DDA2B4A65
:104750008018002902D00A2100F8011C224600A975
:10476000FDF76AFE3078201830706878F021084232
:1047700002D0992002F080FE6878401E6870C0B2B6
:10478000002801D102F0E8FE03F0D6F941B070BC78
:104790005DF810FB18480078002801D0801C00E06C
:1047A0000020C0B2704738B5134C2278002A10D0D0
:1047B00000280ED0032101704270104D2946801C44
:1047C000FDF73AFE0022FA212846FDF707FE0020F9
:1047D000207031BD086C0020C068002000ED00E0B2
:1047E00020ED00E004E000E0A0ED00E034EF00E0A8
:1047F000081F0020A052002003710020C467002081
:10480000DFF81809C17B00EB810181ED050AC17B4E
:1048100000EB8101C1ED090AC17B00EB810181ED53
:104820000D1A017C042901DA491C0174C17B491C61
:10483000C173C9B2042901DB0021C17370470000B4
:10484000F8B52DED068B88B0B0EE408AF0EE608AA8
:10485000B0EE419AF0EE619A04468DED040AB0EE96
:1048600068AA8DED05AAF0EE49AACDED06AA0A26A2
:10487000DFF8A858B5F9660010FB06F0B5F9681026
:10488000471A05F1440003F07BFA95F8440010FB49
:1048900006F095F845104618B6B22A2E0FD13FB251
:1048A000002F0CD56868002806D10120FDF72DFDEA
:1048B000FDF7FDFC012068600120286015E06868B4
:1048C000012807D1FDF7FEFC002068600FF66800A4
:1048D000FFF70EFF2868282E3BDA012803D10FF6D8
:1048E0008400FFF705FF0020286095ED150AF0EE23
:1048F000480AB4EE600AF1EE10FA37D195ED160AC7
:10490000B4EE4A0AF1EE10FA30D195ED170AB4EE82
:104910006A0AF1EE10FA29D1DFF804683068401C09
:10492000306015282CD3E86D00F0E6FDCDE90201DA
:10493000A86D00F0E1FDCDE90001686D00F0DCFD3F
:1049400002460B460FF62800FFF7D2FE002030602B
:1049500016E0002805D1002231460FF2E870FFF77B
:10496000C7FE01202860FDF7B1FCBEE7049868652A
:104970000598A8650698E8650020DFF8A417086088
:1049800004A890EC030AFFF73BFF204680B2B0EE8C
:10499000690A03F00DFA214604A8FCF745FF05F16A
:1049A0006000FDF7FDFB286E012811D1FBF7B3FC79
:1049B00005F16000FDF7F4FB2C2205F1600105F123
:1049C0008C00FDF749FD0FF2BC70FFF791FE01E08E
:1049D00000F000F9002008B0BDEC068BF2BDDFF856
:1049E0003C07807B7047002806D0DFF83017D1F8ED
:1049F000B8104422FDF730BD704710B500281CD117
:104A0000DFF81847483400EE101AB8EE400A84ED7B
:104A1000010A2046FDF7CBFB94ED010AF2EE0A0AEB
:104A200020EE200A10EE100A00F066FD02460B464A
:104A30000FF25870FFF75CFE2FE001281CD1DFF861
:104A4000DC4600EE101AB8EE400A84ED120A04F1BA
:104A50004800FDF7ACFB94ED120AF2EE0A0A20EED4
:104A6000200A10EE100A00F047FD02460B460FF236
:104A70002870FFF73DFE10E002280ED1DFF89C46BB
:104A8000483421722046FDF792FB207A0D2111FB5C
:104A900000F10FF21070FFF72BFE0FF21470FFF70A
:104AA00027FE42F26A7001460FF21070FFF720FEF7
:104AB00040F2EE7001460FF21070BDE81040FFF7B3
:104AC00017BE2DE9F0412DED028B84B006460F464E
:104AD00090460FF2DC60FFF70BFE42F26A7001466F
:104AE0000FF2D860FFF704FE40F2EE7001460FF2BD
:104AF000D860FFF7FDFDDFF8244600224FF4E67191
:104B00002046FDF76BFC04F58075C4F8B85000EE44
:104B1000106AB8EE408A84ED138A00EE107AB8EE7F
:104B2000400A84ED120A84F85080F2EE0A8A404668
:104B30000D2111FB00F0029020EE280A10EE100A61
:104B400000F0DAFCCDE9000128EE280A10EE100A88
:104B500000F0D2FC02460B460FF27C60FFF7C8FD66
:104B6000FBF732FB04F14800FDF721FB42F2107025
:104B7000A4F8C200A4F8C4000020A4F8BC00A4F863
:104B8000BE000220A4F8C6002C2204F1BC01284675
:104B9000FDF762FC0220A07303F0FCF801206073B3
:104BA00004F1440003F0ECF800206060206004B0E1
:104BB000BDEC028BBDE8F08110B592B0FDF79AFB19
:104BC000044600A8FFF70FFF0498001912B010BDAB
:104BD000000000002DE9F0412DED028BDFF83C458F
:104BE00004F17005E86A216F814205D1B4F86620AE
:104BF0006B8C9A4200F08880B1EB000802D5DFF898
:104C00002405804495ED060AD5ED110A70EE608A00
:104C1000F5EE408AF1EE10FA03D59FED950A78EE95
:104C2000808A95ED040AD5ED0F0A30EE608AB5EE64
:104C3000408AF1EE10FA03D59FED8D0A38EE008A16
:104C4000B4F86600C0B295ED050A03F0ADF9B0EE18
:104C5000401A04F10C067078012802D002282BD0EB
:104C600033E004F5A27739469FED821AF0EE480A48
:104C7000B0EE680A404600F057F8207B40442073AD
:104C8000C0B2062821DB04F5AA7004F1BC019FED37
:104C9000791AD0ED0A0A90ED080AD4F8540100F010
:104CA00043F8207B401C2073002244213846FDF746
:104CB00095FB0220707008E004F1BC01F0EE480A98
:104CC000B0EE680A404600F02FF8B4F866000028FD
:104CD00009D10022442104F5A270FDF77FFB0020DA
:104CE0002073012070702C2204F1600104F18C000B
:104CF000FDF7B2FB04F1BC01A96404F580764422FF
:104D00003046FDF7A9FBAE6404F166004088B4F8B4
:104D10000A11884203D0A4F8C600A4F80A01BDEC29
:104D2000028BBDE8F08100002DE9F0412DED048BF0
:104D30008AB0B0EE409AB0EE608AF0EE418A0C463E
:104D4000DFF8D87307F164056E88B7F86480A68031
:104D5000B0EE680A00F0BDF8B868002819D194EDEB
:104D60000C0A30EE090A84ED0C0A00F0AFF984ED6C
:104D70000C0A6680A4F80080A869606394ED0E0AAE
:104D800030EE080A84ED0E0A00F094F984ED0E0A64
:104D90004AE007F1480007AA0AC80AC2036813607C
:104DA00007F1600184B068462C22FDF755FB0FBC6B
:104DB000B0EE680A00F030F9D4ED0C0A30EE800A4B
:104DC00084ED0C0A00F082F984ED0C0AF5EE408ABD
:104DD000F1EE10FA0BDD032E03D106206080208057
:104DE00010E0042E0ED10820608020800AE0032EFF
:104DF00003D107206080208004E0042E02D1092026
:104E000060802080F6EE000A95ED060A20EE200A6A
:104E100084ED0D0A94ED0E0A08EE200A84ED0E0AC8
:104E200000F048F984ED0E0A95ED080ADFEDB00AAE
:104E300020EE200A84ED0F0ADFEDAE0AB4EE600A20
:104E4000F1EE10FA01DBB848E0636869206460881D
:104E5000002801D1002020642869E0602889208191
:104E6000A88860810AB0BDEC048BBDE8F081000029
:104E7000002474490000000010B50C46A1880329E5
:104E800012D1B5EE400AF1EE10FA06DD216A4018A3
:104E9000206200F027F9206210BD616A401860624C
:104EA00000F020F9606210BD042911D1B5EE400A6E
:104EB000F1EE10FA06DDA16A4018A06200F012F9C6
:104EC000A06210BDE16A4018E06200F00BF9E062F8
:104ED00010BDF8B52DED028B0546B0EE408A0C46AC
:104EE00020692818206100F0FDF82061B5EE408AA5
:104EF000F1EE10FA02DDB0EE480A01E0B1EE480A28
:104F0000B5EE400AF1EE10FA43DD844EB068002899
:104F100030D106F5CE77B86806280ED2618804290C
:104F200003D179686918796004E0D6F89C11691892
:104F3000C6F89C112818B86051E0E1694018E0619A
:104F400000F0D0F8E0612146B0EE480AB868FFF7FB
:104F500093FFE0692818E06100F0C4F8E0612146A1
:104F6000B0EE480A2846FFF787FF00F03BF8012023
:104F7000B06034E0E0692818E06100F0B3F8E06167
:104F80002146B0EE480A2846BDEC028BBDE8F4404D
:104F900072E76088032802D0042807D00DE060691A
:104FA0002818606100F09EF860610CE0A069281884
:104FB000A06100F097F8A06105E0606928186061C1
:104FC00000F090F86061554E06F5CE7080680028BC
:104FD00001D000F010F800F005F80020B060BDEC42
:104FE000028BF1BD4D480021C0F89C1100F5CE7038
:104FF0004160816070474948D0F8D010D0F89C21BA
:105000005118C0F8D01000F1D0014A68D0F8A001C2
:1050100080184860704700000FB4DFED370A9FED3D
:10502000361AF0EE0C1A9DED092ABDF80600042888
:105030000FD1DFED322A42EE221AB5EE400AF1EE30
:1050400010FA15D49FED2E1A22EE011A21EE001A45
:105050000EE0DFED2C2A42EE221AB5EE400AF1EE08
:1050600010FA05D49FED281A22EE011A21EE001A3B
:10507000B5EE402AF1EE10FA0ED09DED060AB5EE1F
:10508000400AF1EE10FA07D0DFED200A20EE200AE8
:10509000F7EE000AC0EE800A31EE810A9FED1C1A7D
:1050A00020EE010A9DED0B1A20EE010A20EE200AE7
:1050B00004B07047DFED170AB4EE600AF1EE10FAA3
:1050C00003DBDFED150A30EE200A7047DFED110A31
:1050D000B4EE600AF1EE10FA03DBDFED0F0A30EEFA
:1050E000200A70470F49884201D3104908187047B9
:1050F0008FC2753D0100C84100000000CDCC4C3E80
:105100006666663FCDCCCC3D6666E63F00007042E9
:105110000AD7A33B01247449002474C9BC5F002052
:10512000D8700020819698000000C841806967FF10
:10513000FDF704B9FDF745B850443A2042505F4F9F
:105140004646000050443A2053746570436E7455CF
:10515000702056482825642920435943282564296E
:105160000000000050443A20455849542056480059
:1051700050443A204E41432025662025662025666E
:105180000000000050443A204F46520050443A205C
:10519000312025660000000050443A203220256668
:1051A0000000000050443A20332025640000000035
:1051B00050443A20303246454231350050443A207E
:1051C0004D50445F7625640050443A205052495077
:1051D000445F76256400000050443A203120256663
:1051E00020322025662033202564000051480068C5
:1051F00070471FB5044601A800210A460B460EC0A1
:10520000FFF7F4FF00900522214601A8FDF714F9ED
:105210000420ADF8070000A901A801F02CFF1FBD74
:10522000F0B587B0044602A800210A460B460EC01E
:105230000846CDE90001012510E02846FEF713FEDF
:1052400000280AD0DDE90067012000212A4603F08A
:105250007BF830433943CDE900016D1C232DECDB95
:105260000522214602A8FDF7E7F80820ADF80B005B
:1052700000A902A801F0FFFE07B0F0BD2E4908709A
:1052800070472D48007870472B49487070472A486E
:105290004078704728498870704727488078704761
:1052A0002549C87070472449C86070472248C068C3
:1052B0007047214902780A7142784A718078887172
:1052C00000200881704706221C49FDF7B5B81A4A2C
:1052D0001369002B01D0CB1A00E00346B3F57A7FA7
:1052E00000D3034610891818108100B2B0F57A7FF8
:1052F00005DBA0F57A7010819079401C907192F9CD
:1053000006003C2804DB3C3890715079401C5071F9
:1053100092F905003C2804DB3C3850711079401CA0
:10532000107192F90400182801DB0020107111613E
:1053300070470000B825002014700020187000206D
:10534000B0F5A07F02DB4FF4A0707047A02801DB0E
:10535000A0207047502801DB50207047282801DB2F
:1053600028207047142801DB142070470A2801DB2D
:105370000A2070470520704710B586B002A80FF2CA
:1053800060111CC91CC000A800210A4606C002F01A
:10539000F6FF01788DF8001000A9C2784A704279B2
:1053A0008DF802208079C87001208DF80400052056
:1053B000ADF80B0002A801F05EFE06B010BD30B5DE
:1053C0009DB003A86421FDF77FF800A80FF21C111F
:1053D0001CC91CC00024FF226421FCF7FFFF01252B
:1053E00017E02846C0B2FEF73EFD002810D029463F
:1053F000491E012906D9C91E022903D9091F01D056
:105400001A3905D103A964B26554408A401C0419B5
:105410006D1C092DE5DB64B2ADF8034003A900A8BB
:1054200001F029FE00201DB030BD10B50446A07863
:105430000146491E01290FD9091F012914D9891EC6
:10544000012919D9891E01291ED9203923D1D4F85F
:105450000500FFF72EFF1EE0012801D1002000E02B
:105460000120FFF70BFF16E0052801D1012000E025
:105470000020FFF70FFF0EE0072801D1012000E018
:105480000020FFF70DFF06E0092801D1002000E011
:105490000120FFF7F9FEA0781438032801D9153848
:1054A0000ED12620FEF7DFFC030009D0D4F805203A
:1054B000B4F80310A078DB691B69BDE810401847F9
:1054C00010BD81780C2906D0182906D01B2903D0DD
:1054D0002C2903D070478CE6A2E64DE76FE7000069
:1054E00004FF1800000000000000000004FF2C0072
:1054F00000000000000000005FF0FF0C1CEAD0512B
:1055000014BF614506E0C110400721F0E04101F100
:105510006051704779B900F0004100020AD0B0FA3A
:1055200080FC00FA0CF001F16051A1EB0C5101EB91
:10553000D0214005704741020CBF40F4E0016FF0FC
:105540000001002070470000010040F10980F4468E
:10555000404200F005F851F000416047010000BFF3
:1055600009D0B0FA80F18840C91CC1F584610905F1
:1055700001EBD02140057047F446400D40EAC120C0
:10558000490006D200F014F8004248BF6FF0004016
:10559000604700F00DF84FF0004188428CBF08468C
:1055A00040426047400D40EAC120490080F00D8034
:1055B00040F00040490DA1F58061491C05D4D1F1AE
:1055C0001F0154BFC840C01770474FF0000070471C
:1055D0004FF4001C1CEB410F94BF1CEB430F09E080
:1055E00041EA030C50EA4C0C52EA0C0C03D29942EB
:1055F00008BF9042704714BF8B4282427047000040
:10560000B0B581EA030C0CF0004C40F2FF7515EACE
:1056100011541DBF15EA1357AC42AF4239E0E419EB
:1056200023EA455343F48013C90241F0004141EAA3
:10563000505EC7021100A7FB020200284FF00000D5
:10564000EEFB01204FF00001E3FB072118BF42F001
:105650000102401800214941E3FB0E01A4F58064DA
:105660000F0302D252004041494154F101046CDD64
:10567000470872F1004250F1000051EB0451A1F5CE
:1056800080115CBF41EA0C01B0BD4CEA055100201D
:10569000B0BD05EA1357AC4214BFAF4241E050EA37
:1056A000410E1CBF52EA430E02E061460020B0BD2D
:1056B00024423C441BD15FEA070EF6D0090302BF27
:1056C00001460020AEF1140EB1FA81F7AEEB0704EB
:1056D00001FA07FE0C37C7F1200100FA07F7C840AE
:1056E0004EEA000E23EA455343F48013A2E733F059
:1056F0000043B3FA83F704BFB2FA82FE77440B3F4C
:10570000E41BB7F1200E2FBF02FA0EF3BB40C7F126
:10571000200E22FA0EFE38BF43EA0E03BA40641C84
:1057200082E750EA410E14BF52EA430E6FF00001C7
:105730004FF4001717EB430F8ABF194617EB410FC1
:10574000B5E74CEA05510020B0BDD4F10104B4F135
:1057500020070FDAC4F12007520828BF42F00102E7
:1057600010FA07F501FA07F7E1BF2A43E040384392
:10577000E1400FE0352C98DCC7F1200452EA4002EA
:1057800020FA07F218BF42F0010231FA07F0A140F7
:105790000A43002172F1004250F1000051EB0C016C
:1057A000B0BD000070B44FF0004591EA030C44BF57
:1057B0006B4002F087BE00BF841A71EB030603D270
:1057C000001BB141121973414FF4001C1CEB410F37
:1057D00034BF7CEB430443E00C0DA4EB1356352E91
:1057E00050DC45EAC323DB0A45EAC121C912B6F100
:1057F00020050DDD63FA05F6EB4086EA030512424B
:1058000018BF45F00105C01851F100010CD213E09A
:1058100062FA06F5F2405540F3415A40B340F34076
:105820005A408018594107D349085FEA30005FEABF
:10583000350528BF45F0010501F58011420875F1D5
:10584000004250F1000041EB045170BC4FF4001CC9
:105850001CEB410F38BF70470020090D0905704748
:105860001CEB410F10D252EA43060BD0BCEB410FA8
:1058700005D80C0DAB43661E342EB5DD02E0AB43FC
:105880008018594170BC704770BC70474FEAF17C7A
:10589000BCF1E04C2CBFBCF5001F11E05FEA4C0CE2
:1058A00034BFBCF17F5F2EE05FEA9C0C4FEA0C1C1A
:1058B0004FEA3C0CC10071F100414CEB5070704755
:1058C000C90241EA5051C00218BF41F0010141F044
:1058D00000414FEA6C50C0F10900212810D240EA83
:1058E000CC7CCCF1200C11FA0CF070F10040CCF122
:1058F000200C21FA0CF00CF0004C40EB0C0070472F
:105900004FEACC707047490011F5001F04D84FEAE8
:10591000CC10FF30C0057047C81770474FF4001C0B
:105920001CEB410F94BF1CEB430F09E041EA030C51
:1059300050EA4C0C52EA0C0C03D28B4208BF824254
:10594000704714BF994290427047000010B50400A0
:1059500010480078002805D10F4802F08EFE0D484F
:10596000012101700C4802F0C2FE200003F0BFFDCF
:105970000400094802F0EFFE200010BD10B504003D
:10598000054802F0B4FE200003F011FF024802F0C7
:10599000E2FE10BD0D7100202870002038B50446CD
:1059A000002500E06468002C0CD0207A0A78904230
:1059B000F8D1E0684A689042F4D120698A68904240
:1059C000F0D101252A460FF2C8210FF2D020FEF7B0
:1059D0008FFE002D00D10024204632BD38B504468C
:1059E0002020FFF7B3FF054600222021FCF7F6FC3C
:1059F0000C22214605F10800FCF72EFD6068686165
:105A0000A068A86101202877284632BD2DE9F84317
:105A100005460E460027B84606F108099B4C20783B
:105A2000401C20706078F021084202D0992001F0DB
:105A300023FD01F097FD6078401C60702868D9F85C
:105A4000041001E080464068002803D0C2689142FB
:105A5000F8DA0127002F0AD0016831607060016810
:105A6000002901D04E6000E02E60066008E0B8F129
:105A7000000F04D0C8F80460C6F8008000E02E6073
:105A80006078F021084202D0992001F0F5FC60789E
:105A9000401E6070C0B2002801D101F05DFD02F02F
:105AA0004BF80020BDE8F28370B506460D46774CF2
:105AB0002078401C20706078F021084202D09920A4
:105AC00001F0DAFC01F04EFD6078401C60706868FF
:105AD0002968002901D0486000E03060686800282B
:105AE00001D0296801602846FFF748FF6078F0215F
:105AF000084202D0992001F0BFFC6078401E60701F
:105B0000C0B2002801D101F027FD02F015F80020F5
:105B100070BD70B505462E68002E00D16E68002E4F
:105B200033D05A4C2078401C20706078F021084215
:105B300002D0992001F0A0FC01F014FD6078401C17
:105B40006070F0687169401AE9680A1A90FBF1F315
:105B500001FB0321696129690A1A90FBF1F001FB3D
:105B60000020A8616078F021084202D0992001F05D
:105B700083FC6078401E6070C0B2002801D101F043
:105B8000EBFCBDE8704001F0D7BF70BD70B50446B6
:105B90000D462068FFF702FF06000BD12846FFF7ED
:105BA0001DFF064631462046FFF730FF3046FFF71F
:105BB000B0FF02E0307F401C3077207A401C20721A
:105BC000307A002800D16660002070BD10B5044610
:105BD0002068FFF7E3FE002801D1032010BD017FFC
:105BE000491E0177217A491E2172017A002901D1CB
:105BF00000216160017F002903D101462046FFF7A3
:105C000053FF002010BD70B506460D461F4C20788E
:105C1000401C20706078F021084202D0992001F0E9
:105C20002BFC01F09FFC6078401C6070306801E044
:105C300081614068002815D041694A1B8169491B70
:105C4000012A05DAC368D61892FBF3F203FB12624D
:105C500042610129ECDA02698B1891FBF2F102FB37
:105C60001131E5E76078F021084202D0992001F077
:105C700003FC6078401E6070C0B2002801D101F0C2
:105C80006BFC01F059FF002070BD0000081F0020D0
:105C900066696E645F636C69656E740025733A2093
:105CA00066696E6428256429000000002DE9F04D26
:105CB0008EB0394E7078F021084202D0992001F060
:105CC000DBFB01F04FFC7078401C707004F0DEF8D4
:105CD000074601A9002004F02FF900A9002004F0D4
:105CE000B0F8DFF8B880D8F80800B84203D2811CB9
:105CF000B94200D307469DF8020002909DF80100CA
:105D000003909DF8000004909DF8060005909DF812
:105D10000500401E06909DF80700463007900020C1
:105D20000A90DFF870A0834602A804F0F9F9AAFBF4
:105D3000004543F6FF70C01B4EF66B614843594661
:105D40004FF47A720B4604F075FA24184D41D8E9E5
:105D500000018D4206D801D3844203D214EB0A0419
:105D600045EB0B05C8E90045C8F808707078F021CC
:105D7000084202D0992001F07FFB7078401E7070BD
:105D8000C0B2002801D101F0E7FB204629460EB041
:105D9000BDE8F08D40420F00081F00207870002001
:105DA0007FB50446FEF75FF801A9114A68CA68C1C9
:105DB000458A0120ADF80000281DFFF7C7FD064603
:105DC000372030707470022200A9B01CFCF734FB3D
:105DD000311D2046FEF728F9281DADF80700314691
:105DE00001A801F048F93046FFF7C8FD7FBD00BFAC
:105DF000FCAB010838B505000C0094F8500064288D
:105E000002D0802001F038FB01F02DFE802080F3CD
:105E1000118800BF00BFA0692843A061207C10F05A
:105E2000F800082806D1E069A169084202D02000E4
:105E300001F0C2FE07484078F021084202D09920C4
:105E400001F01AFB03484078002802D1002080F3BB
:105E5000118831BD081F00202DE9FF4104460D4681
:105E6000FEF701F8064600A829498CC98CC006F146
:105E7000100000F0CAF8074606F1100000F0E6F83E
:105E8000ADF80C00002F01D1002D3FD0002D01D026
:105E9000032000E00020002F01D0391D00E0002188
:105EA0000818FFF753FD8046002F13D0372088F8DD
:105EB000000088F80140022203A908F10200FCF763
:105EC000BBFA06F1100108F1040000F052F8381D89
:105ED000ADF80300002D12D00520BDF8031001F825
:105EE00008000120BDF8031041444870BDF80300CC
:105EF00040448470BDF80300C01CADF80300414667
:105F000000A801F0B8F84046FFF738FDBDE8FF8172
:105F100008AC010800218180C180704738B5044673
:105F2000E088401C2288A38890FBF2F502FB150054
:105F300093FBF2F502FB1535A84205D1581C90FBE6
:105F4000F2F302FB1300A080E088401C90FBF2F308
:105F500002FB1300E08060880246A368E58800FB2E
:105F60000530FCF769FA2088012801D10120E08082
:105F700031BDF8B504460D0046D0002C44D0A988A8
:105F800008462B88012B01D1002604E0421C92FB1D
:105F9000F3F603FB1626EA88571C97FBF3FC03FB7A
:105FA0001C7C90FBF3FE03FB1E0EF44518D1022B64
:105FB00016DB8A4208D26E8806FB07F2A968181A17
:105FC00006FB0040FCF738FA6888A9882A88521A2C
:105FD0004243AB6800FB01312046FCF72DFA10E08C
:105FE000284600F012F800280BD0284600F00DF8E3
:105FF0000246A868B6B2698801FB06012046FCF794
:106000001BFA0020A880E880F1BD70B481880A46A0
:10601000C3881C46A51A01D5C91A00E0591A631C89
:106020000488254693FBF5F605FB163392FBF5F63F
:1060300005FB1622934202D1022D00DB2146C9B294
:10604000408811FB00F080B270BC704730B481888A
:106050000A46C3881C46A51A01D5C91A00E0591A78
:10606000631C0088044693FBF4F504FB153392FB94
:10607000F4F504FB1522934202D1022C00DB014609
:10608000C9B2084630BC70470020704710B5DFF831
:1060900014450020A08104F114010120FDF7FAFD50
:1060A000002803D00FF21050FEF722FB0120A07150
:1060B0000020E071207020816070E0811E206071FE
:1060C00000202061A070E070207110BD80B501211A
:1060D0008DF800108DF8011008218DF802108DF850
:1060E000030000A92B20FDF7CBFE01BD70B52DEDFF
:1060F000048B84B0002400A90120FDF795FFDFF890
:10610000A45495F90160002E05D0022E37D00FD38C
:10611000032E5DD086E09DED000AB0EE408A9DED35
:10612000010AF0EE408A9DED020AB0EE409A79E055
:106130009DED010AF0EE408ADDED020AB0EE609AB4
:106140009FEDCC1A00EE401A00EEE01AB5EE401AB0
:10615000F1EE10FA10DD11EE100AFFF7CDF941EC67
:10616000100B04F0DFF851EC100BFFF78FFB00EE83
:10617000100AB0EE408A55E09FEDD08A52E09DEDC6
:10618000000AB0EE408ADDED020AB0EE609ADDED65
:10619000001A9FEDB81A00EE611A00EEE01AB5EE93
:1061A000401AF1EE10FA10DD11EE100AFFF7A4F913
:1061B00041EC100B04F0B6F851EC100BFFF766FB46
:1061C00000EE100AF0EE408A2CE0DFEDBC8A29E0F8
:1061D0009DED000AB0EE408A9DED010AF0EE408A86
:1061E0009FEDA41A00EE401A9DED000ADDED000AB5
:1061F00000EE601AB5EE401AF1EE10FA10DD11EE65
:10620000100AFFF779F941EC100B04F08BF851EC10
:10621000100BFFF73BFB00EE100AB0EE409A01E0D6
:106220009FEDA69AB5F90C00012801D101201DE1CE
:1062300095F90000002860D16889411C698195F9B1
:106240000500421C09B28A4233DB0098FFF754F97B
:1062500021F000414FF02042D34BFFF75FFB03D802
:10626000A878401CA87001E02046A8700198FFF7AC
:1062700043F921F000414FF02042CB4BFFF74EFB9A
:1062800003D8E878401CE87001E02046E8700298E6
:10629000FFF732F921F000414FF02042C24BFFF7E7
:1062A0003DFB03D82879401C2871DEE02046287188
:1062B000DBE095F90210814202DB012068700FE0FB
:1062C00095F90310814202DB0220687008E095F91D
:1062D0000410814202DB0320687001E020466870F0
:1062E00095F901100FF2DC20FEF702FA0120287068
:1062F0002046688104F096F8B7E0012864D1288927
:10630000401C28813046B0EE491AF0EE680AB0EE23
:10631000480A04F08BF8002847D0F0EE680AB0EE87
:10632000480A20EE000A00EEA00A09EE090A04F06D
:106330003FF989EE000A10EE100AFFF7DDF841EC94
:10634000100B04F0D5F953EC102B98489849FFF73F
:1063500057F9FFF711F9286195F90100002821D1BB
:10636000A879012809D105F114010120FDF7D3FC1A
:10637000002800D003240020A871E87900280AD161
:1063800005F120011C20FDF785FC002801D0032029
:106390006CE00120E8710FF23C20FEF7A9F9022021
:1063A000287062E0032028705FE0B5F908006428D7
:1063B0005BDB2046288100F0A5F8052028700FF24D
:1063C0002820FEF795F950E003284ED1F0EE680A38
:1063D000B0EE480A20EE000A00EEA00A09EE090A13
:1063E00004F0E6F889EE000A10EE100AFFF784F8D0
:1063F00041EC100B04F07CF953EC102B6B486C490A
:10640000FFF7FEF8FFF7B8F82969081A04F078F9E1
:10641000002E19D16989491C698109B2652908DAF8
:10642000242803DBE889401CE88115E02046E88148
:1064300012E020466881012028702046E8810FF292
:10644000B410FEF755F910E0242803DBE889401C5E
:10645000E88101E02046E881B5F90E00052804DB5B
:10646000042028700120FFF731FE204604B0BDEC67
:10647000048B70BD3D57C04210B54A4C00202070BF
:10648000A081E079012808D104F120011C20FDF74A
:1064900042FC00280BD10020E071A07901280AD12C
:1064A00004F114010120FDF736FC002801D003207F
:1064B00010BD0020A071002010BD000000000000F1
:1064C000002070470020704710B5364CE079012855
:1064D00008D104F120011C20FDF71DFC00280BD180
:1064E0000020E071A07900280AD104F114010120F4
:1064F000FDF7D0FB002801D0032010BD0120A071C2
:10650000002010BD10B5274C002060812081A079AB
:10651000012808D104F114010120FDF7FCFB00283B
:106520000BD10020A071E07901280AD104F12001EB
:106530001C20FDF7F0FB002801D0032010BD002037
:10654000E071002010BD10B50FF2DC00FEF7D0F8AE
:10655000144C94F9000002280FD1FFF7B5FF03286F
:1065600005D10FF2D000FEF7C3F8032010BD0320C1
:1065700020700FF2CC00FEF7BBF8002010BD0D49D3
:106580000A1DC2612B220270142282600122027352
:1065900002820422428200228282C28281611046EB
:1065A00070470000142100209999274046DF617E42
:1065B000DCA54C40F4230020736D2041434320664A
:1065C00061696C0053535020534D41204D6F6465F9
:1065D0002025640053535020534D41204144442012
:1065E000414343494E54000053535020534D4120E2
:1065F0004E46000053535020534D4120556E736159
:1066000074697366696564204D6F76696E672041B1
:106610006E676C6520647572696E6720322D7365D4
:10662000632021212100000053535020534D41206D
:10663000494E5400534D20414420464C0000000078
:1066400053535020534D4120494E56205341490049
:1066500080B58DF8000000A91120FDF711FC01BDE7
:106660000020704710B5754C04F108010120FDF7BA
:1066700011FB002801D0032010BD04F045F80020D4
:106680002070012060700020A07060600120E07028
:10669000002010BD3EB500A90120FDF7C5FC674CE8
:1066A0002078012818D16078012808D104F1080168
:1066B0000120FDF730FB00281BD100206070A0787E
:1066C00001284FD104F114011C20FDF724FB002800
:1066D0000FD10020A07045E0E078002824D1607838
:1066E00001280AD104F108010120FDF714FB00285C
:1066F00001D003203EBD00206070A078002831D179
:1067000004F114011C20FDF7C5FA002805D00FF292
:106710003410FDF7EDFF03203EBD0120A0700FF205
:106720003810FDF7E5FF1DE000A890EC030A04F027
:106730000DF8054604F083F9002803D16068401C79
:10674000606001E0002060606068332803DB0020A7
:10675000E07003F0D9FF012D04D10120FFF778FF8D
:106760000120207000203EBD10B5344C6078012817
:1067700008D104F108010120FDF7CDFA00280BD162
:1067800000206070A07801280AD104F114011C20B7
:10679000FDF7C1FA002801D0032010BD0020A07031
:1067A0000020207010BD002070470020704710B5F9
:1067B0000FF2B400FDF79CFF204CE078002829D1AF
:1067C000A07801280ED104F114011C20FDF7A3FAD2
:1067D000002805D00FF29C00FDF78AFF032010BDB2
:1067E0000020A070607800280ED104F1080101207B
:1067F000FDF750FA002805D00FF29400FDF778FF5E
:10680000032010BD012060700120E0700FF29400A1
:10681000FDF76EFF002010BD09490A1DC26111225B
:1068200002701422826001220273028242820022DC
:106830008282C28281611046704700005C23002082
:10684000D823002053535020534D4420494E542008
:106850004641494C0000000053535020534D442002
:10686000494E54204144440053535020534D44203A
:10687000494E540053535020534D4420414343202C
:10688000494E542052656D6F7665204661696C00F3
:1068900053535020534D4420414343204F6E2046D4
:1068A00061696C0053535020534D4420494E54208D
:1068B0004F4343000020704710B5DFF8804604F1D5
:1068C00038010120FDF7E6F9002805D00FF28060BD
:1068D000FDF70EFF032010BD04F138010520FDF780
:1068E000D9F9002805D00FF27860FDF701FF0320E9
:1068F00010BD00F081F9002010BD1CB50446012038
:106900008DF800008DF8010038208DF8020001207C
:106910008DF803008DF804008DF805108DF8062021
:1069200000A95B20FDF7ACFA204600F04EF813BD3D
:1069300080B500F0F0F8DFF80406C07A052813D817
:10694000DFE800F003060C09120F00F0A1F90EE0D9
:1069500000F0DAF90BE000F010FA08E000F047FA76
:1069600005E000F082FA02E0012000F0F8F800F003
:1069700067F900F01AF9002002BD10B500F0B7F871
:10698000DFF8B84504F138010120FDF7C4F900280B
:1069900001D0032010BD04F138010520FDF7BBF93B
:1069A000002801D0032010BD002010BD80B51128A3
:1069B00001D100F081F8002002BD80B5102802D17D
:1069C000104600F01EF8002002BD012811D1DFF8AA
:1069D0006C054179017100210172C171417902296F
:1069E0000DD18179082901D0092908D10021C1627E
:1069F00005E0022803D1DFF844054178C170012089
:106A0000704738B5017803292CD144788178C07853
:106A100010EB0125ADB22A4621460FF25450FDF786
:106A200067FE012C06D01DD3032C0ED006D3042CF8
:106A300012D017E0DFF80805857713E04FF47A707D
:106A40006843DFF8FC1488600CE04FF47A70684308
:106A5000DFF8E814486105E04FF47A706843DFF826
:106A6000E0144860012032BD70B582B000A9082052
:106A7000FDF7DAFA9DF80050BDF90260DFF8BC447A
:106A8000B4F93030324629460FF2F440FDF730FEBB
:106A9000B4F93000864200DA2686002D04D1B4F91C
:106AA0003000301A322802DB0120A07202E0002000
:106AB000A0722062002076BD0120DFF880140872E9
:106AC000704710B5DFF87444607A002801D00020C8
:106AD00010BD04F138010820FDF7DCF8002801D0D2
:106AE000032010BD012060720020206210BD10B58F
:106AF000DFF84844607A002801D1002010BD04F17D
:106B000038010820FDF707F9002801D0032010BD47
:106B10000020607210BD00B589B000A90120FDF70A
:106B200083FA03A90520FDF77FFA039900A803F073
:106B3000A9FFDFF80804417A002907D090F90A106C
:106B4000012903D1016A826A51180162816AC26A0D
:106B50008A18C262426A8918416209B000BD38B51C
:106B60000446DFF8D8532246E97A0FF24040FDF799
:106B7000BFFDEC7200206862BDE83140B7E770B538
:106B800004460D46164633462A4621460FF230404B
:106B9000FDF7AEFDDFF8A403047021464171857155
:106BA000002E01D00121C17170BD10B5DFF88C43FA
:106BB000207A002806D021786171A2790120BDE8F1
:106BC00010409AE6E07900280BD061792079814263
:106BD00004D0A2790120BDE810408EE60020E071CB
:106BE00010BD207B002806D0A27861780220FFF734
:106BF00084FE0020207310BD10B503F033FFCF4C8E
:106C0000002234212046FBF7E9FB5020A06200203F
:106C1000E07240F6B830206147F230516161A06106
:106C200001206073E1614FF4FA60E062012020709E
:106C30006071A07147F6FF7020866420E07010BD7F
:106C400038B5BE4C94F8320001280ED104F056F944
:106C500000280AD0022084F83200651C0120E87266
:106C6000032060700B20687031BD94F83200032857
:106C70000DD1651CE87A002809D104F0E1F8A97863
:106C8000814204D00121E97260700C20687031BD2E
:106C900080B503F06FFF00280AD0002201210846CA
:106CA000FFF76DFF0120FFF75AFF0120A34948734A
:106CB00001BD000038B5A14C606BA16A0818606383
:106CC0000025FFF7FEFEA069616B88421AD200EE34
:106CD000100AB8EE400ADFED980A20EE200ABCEE5A
:106CE000C00A10EE100A216A884206D20225E17A13
:106CF0000FF2E820FDF7FCFC00E0012500206063B6
:106D0000FFF7F5FE284632BD10B58C4C00F01DF89B
:106D1000002805D00320FFF722FF0120607310BD7B
:106D2000606900F021F800280ED0FFF7C3FF0228A9
:106D300005D1002060730220BDE810400FE7012854
:106D400002D100206073606210BD80B504F04FF87E
:106D5000002807D07948006903F012FF022801D10A
:106D6000012002BD002002BD74494A6A904201D24E
:106D70000120487391F90D00704710B56F4C00F079
:106D800023F800280AD0012202211046FFF7F7FE5F
:106D90000120FFF7E4FE0120607310BD607B002836
:106DA00011D0FFF787FF022807D100220821022017
:106DB000FFF7E5FE0020607310BD012803D100201D
:106DC00060730520A07110BD10B55C4CE06AB0F591
:106DD000FA6F0AD304F017F8002806D0E16A0FF220
:106DE0001020FDF785FC012010BD002010BD70B5FE
:106DF0000026524C534DFFF7A8FF002807D030461D
:106E00002870012060730320FFF7A9FE18E0E069F5
:106E1000FFF7AAFF002813D0FFF74CFF02280CD180
:106E20002878411C2970304660626073E27AC9B2EA
:106E30000FF2D010FDF75CFC02E0012800D1012622
:106E40002878032807DB012209210220FFF797FE9B
:106E500003F0F2FE0526002E06D000202870607395
:106E60003046BDE870407AE670BD3448C06AB0F57F
:106E7000FA6F00D2704780B500F010F8002803D1F7
:106E800000F01AF8002808D0012204211046FFF76C
:106E900076FE0120BDE8024061E601BD00B585B087
:106EA00000A90520FDF7C0F8009815288041C043CF
:106EB000C00F40B205B000BD38B50024224D95F991
:106EC0000000002805D103F0C3FE002801D00120F6
:106ED000287095F90000002819D0FFF7F2FD174837
:106EE0006968826A51186960B1F5967F0FDB90F985
:106EF0000A00002804D10FF22410FDF7F9FB012449
:106F0000002068602870FFF7F2FD03F095FE204630
:106F100032BD0E4901F10802C2615B2202705022AB
:106F20008260012202730282072242820022828250
:106F3000C282816110467047CDCCCC3E501F0020EC
:106F4000641F00200471002084700020FC220020B7
:106F50004450434D20414343206661696C0000006A
:106F60004450434D204C49474854206661696C00A9
:106F70004450434D2053657420256420256400004F
:106F80004450434D2050726F7820537461746520D3
:106F90005B25645D206F6666736574205B25645DA8
:106FA000206D696E205B25645D0000004450434DF8
:106FB000205354205B25645D2D3E5B25645D0000FD
:106FC0004450434D2053455420524554205B256482
:106FD0005D5B25645D5B25645D0000004450434DAE
:106FE00020434C4F534544205B25645D0000000066
:106FF0004450434D20484F4C442054494D45202592
:10700000640000004450434D204F464620434E54F8
:10701000205B25645D5B25645D0000004450434DAA
:107020002050726F7869204F70656E0010B5864CE5
:1070300086488089C0464021854804F005F8002034
:1070400001F014FA4FF48051824804F0F5FB002857
:1070500010D12046441E0128F4DA00217E4804F0B5
:10706000C5FC00217D4804F0C1FC0120BDE81040B2
:1070700001F0FCB910BDF8B504460E46784D2878ED
:10708000401C28706878F021084202D0992000F056
:10709000F3F900F067FA6878401C687020780528DA
:1070A00003D1FDF777FB074600E00027B4F80300A3
:1070B00017FA80F0FEF74AFCC4F80500002812D148
:1070C0006878F021084202D0992000F0D5F968785C
:1070D000401E6870C0B2002801D100F03DFABDE842
:1070E000F14000F029BDB4F803203146FBF7A4F9C4
:1070F000002F0BD0D4F80500B4F803100818FDF7E2
:1071000052FBB4F803003818A4F803006878F021A3
:10711000084202D0992000F0AFF96878401E6870EC
:10712000C0B2002801D100F017FA00F005FD4D4D66
:10713000214605F2144004F019FD29460420BDE85B
:10714000F440FEF757BE38B50446B4F80300401DBE
:10715000FEF7FCFB050016D005222146FBF76CF973
:10716000B4F80320D4F80510681DFBF765F9B4F8EE
:107170000300411D89B2284600F091F8002D02D08D
:107180002846FEF7FBFBD4F80500002804D0FEF7E4
:10719000F5FB0020C4F8050031BD10B584B0012016
:1071A000ADF8030005208DF80000BDF80300FEF7E0
:1071B000CDFBCDF8050000280FD0072101700FF29C
:1071C000B000FDF795FA274C00A904F2144004F032
:1071D000CDFC21460420FEF70DFE1FBD10B584B086
:1071E00000A800210A460B460EC0FFF7D6FF062076
:1071F00004F0F2FC0446A00701D5FFF717FF600773
:10720000F5D500A9184804F02DFD00A8FFF79BFF55
:10721000EDE710B584B0134C04F586630422092110
:1072200004F2144004F052FD022002904FF47070FA
:10723000019004F1540000900C4B64220FF23801CD
:10724000204604F097FD1FBD404B4C00003001402C
:10725000646E002000040240586402401064024042
:10726000081F0020404A0020544E0020DD71000815
:107270005245534554000000636F6D6D5F74617338
:107280006B000000BFF34F8F4248016801F4E061DA
:10729000414A11430160BFF34F8F00BFFDE7F0B5D6
:1072A00083B00E4600210091032101913B4CA16C5B
:1072B000C90706D5A16C49084900A164A16CC9079A
:1072C000FCD4374D00220146284604F0A5FB4FF0C0
:1072D000C051284604F0BDFB314628464160C046F7
:1072E0000121284604F082FB2E4E0096002001F07A
:1072F000BBF80FF2BC070DE00096012001F0B4F8D6
:10730000052001F071F801993846FDF7F1F90020E8
:1073100001F0AAF84FF0C051284604F087FB00287E
:1073200016D10098411E00910128F3DA0198401E01
:107330000190E1D50021284604F058FB00212046A9
:1073400004F054FB01993846FDF7D2F9FFF79AFF94
:1073500049F640400090144C0221204604F028FEDB
:10736000002804D10098411E00910128F4DA42F26D
:10737000107000908021204604F01AFE012804D1EC
:107380000098411E00910128F4DA0120BDE8FE407A
:1073900001F06AB80CED00E00400FA051064024048
:1073A0005864024080841E00003001406AE70000FB
:1073B000547852657472792025640000002801D148
:1073C0000A48806890F85010642901D0002000E03D
:1073D000C06A7047002801D10448806890F85010B6
:1073E000642901D0002000E0806A7047081F002057
:1073F0000248704702480149401A7047480000207F
:107400004808002008B584B00023029311B9009306
:10741000019302E00090481E019004AB00A90748C8
:107420007844183004F0CCFD009911B1009A002185
:107430001170002858BF029805B000BD73B0FFFF5F
:1074400000F10103810704D010F8011B89B1810705
:10745000FAD10268B2F10131914311F0803F04BFCB
:1074600050F8042FF6E710F8011B11B110F8011BBA
:10747000FBE7C01A7047000000B585B002460FF266
:10748000140100A805F072FC00A8FCF782FF05B00B
:1074900000BD00004F4525640000000034488168AD
:1074A000002904BF08B008E0EFF30982A2F1280226
:1074B000036882E8F84F83685A6000F056F98168E3
:1074C00059B14A6892E8F84F036002F1280282F34A
:1074D000098813F47F4F3FD0704726482649096832
:1074E000401A80F308884FF08071C161234981619F
:1074F0007FF0060E704701BC2046DFF884E000BD37
:10750000FEE7204800681C490968401A203820F02E
:10751000070080F308884FF000011548417081F39F
:10752000118862B600F014F8FEE703680CB44FF05F
:10753000000141704FF0000181F311881249134A94
:107540000A604FF0800181F311880CBC0360704722
:107550000D490E4A0A6070474FF0000181F311880F
:10756000704700BF4FF0800181F31188704700BF62
:10757000081F00202808002038AC0108CDCE0008E4
:10758000017500080000000804ED00E00000001094
:1075900010B4802080F3118800BF00BFDFF8C0075F
:1075A0008068DFF8BC1700220A71002181F311887E
:1075B00000282ED0016800292BD042690168496952
:1075C000914226D1016800E019000B68002B02D01F
:1075D0005C699442F8D0802282F3118800BF00BF1A
:1075E000DFF87C271269824203D1DFF87427036831
:1075F0001361026A036813601A6201620B68036018
:107600000268002A00D01862086091F8450081F8ED
:107610004400002080F3118810BC7047802080F364
:10762000118800BF00BFDFF83C070068DFF83017A3
:10763000096A401A01283ADADFF82407006A05E0EF
:10764000DFF81C170862002181F31188DFF8181792
:107650000978C90726D5802181F3118800BF00BFB2
:10766000DFF8041709788907EAD5DFF8FC160978EE
:1076700011F0FD01DFF8F0261170002181F311886F
:10768000DFF8DC16096A8842FAD0DFF8D4160862FF
:10769000DFF8D0060068401CDFF8C8160860DFF885
:1076A000C0164862802080F3118800BF00BF704779
:1076B00010B5DFF8AC0600214171DFF8A406006ABE
:1076C00010F18040DFF898164862DFF89406C06930
:1076D000002805D0DFF88806DFF88416C9698847D6
:1076E000002080F31188DFF87806C4680EE0E068B7
:1076F000DFF86C16496A401A002803D5DFF86006E7
:10770000E1684162002080F311882468002C26D0B3
:10771000802080F3118800BF00BFDFF844060069B5
:10772000002806D06069DFF838160969496988427F
:107730001AD3207C4007E5D5E068DFF82416096AF3
:10774000401A0128D3DA200000F036FA802080F3B6
:10775000118800BF00BF207C0028C8D104E0802031
:1077600080F3118800BF00BF10BD38B5DFF8F00509
:1077700000214170DFF8E80501210170DFF8E00524
:10778000C06B002818D0802080F3118800BF00BF94
:10779000DFF8CC05C06B8047002080F31188DFF84C
:1077A000C0050021C163DFF8B80500214163DFF89F
:1077B000B005002180F83810FFF71AFE0078C0B23B
:1077C000CD2802D07D20FFF757FEDFF894058068B2
:1077D000002812D0DFF888058068806C00280CD063
:1077E000DFF87C058068806C01680800002804D000
:1077F000DFF86C05806840688847DFF8640590F81A
:10780000310000280FD0DFF858058068DFF85015E8
:1078100091F8301080F84410DFF844050079002812
:1078200001D0FFF7B5FEDFF8380590F840000028DA
:107830003DD0DFF82C0590F84000C00718D5DFF8E0
:107840002C050068DFF81815096A401A00280FD5C2
:10785000DFF80C0590F8400010F0FE00DFF800158E
:1078600081F84000DFF8F80490F8400000281ED0AE
:10787000802080F3118800BF00BF05F035FB002198
:1078800081F31188DFF8D814896800290CD0DFF85B
:10789000D0148968896B4118DFF8D4241268891ADA
:1078A000DFF8BC2492689163DFF8C4140860DFF845
:1078B000B004806800280ED0DFF8A4048068007C43
:1078C000002808D1DFF898048068406B401CDFF87E
:1078D000901489684863DFF888040069002839D06B
:1078E00006E0DFF87C0421680161002080F3118844
:1078F000802080F3118800BF00BFDFF864040469B2
:10790000002C2FD0257CEDB2002D2BD0680716D58A
:10791000E068DFF84C14096A411A012906DA2000F0
:1079200000F04AF9207C002809D113E0DFF8301478
:10793000496A411A002902D5DFF824144862EDB2E1
:1079400015F0FB001028CCD1A06880684068007C4E
:107950000028C6D1802080F3118800BF00BF01E05D
:10796000FFF7A6FEDFF8F80340790028F8D1DFF82A
:10797000F8030078C00701D5FFF750FEDFF8E003F9
:1079800000214171DFF8D8030069002853D0DFF8E7
:10799000D0030069007C002809D0DFF8C403006927
:1079A00080688068DFF8B8134068886005E0DFF819
:1079B000B003DFF8AC1309698160DFF8A4038068C5
:1079C00090F85000642802D08020FFF755FDDFF8C2
:1079D00090038068C06A0078CD2802D07820FFF735
:1079E0004BFDDFF87C038068806C00280CD0DFF84A
:1079F00070038068806C41680800002804D0DFF8BC
:107A00006003806840688847DFF85403806890F816
:107A10004400DFF84C1381F83000DFF8441381F89C
:107A20003100DFF83C038068006B401CDFF8301346
:107A30008968086314E0DFF82803002180F831101A
:107A4000DFF81C03002180F83010DFF81403002158
:107A50008160DFF80C0300210170002080F31188A1
:107A6000DFF8FC0232BD80B505F078FADFF80413C8
:107A70000978002806D0022810D009D3042815D090
:107A800010D314E0002902D0A320FFF7F5FC11E089
:107A9000002902D1A420FFF7EFFC0BE0A620FFF79E
:107AA000EBFC07E0A720FFF7E7FC03E002E0A820DB
:107AB000FFF7E2FC01BD10B505F050FA0400DFF855
:107AC000B4020078002802D0A020FFF7D5FC002CDB
:107AD00005D0022C08D003D3032C09D00CE00EE013
:107AE000A420FFF7C9FC0AE0A620FFF7C5FC06E0CA
:107AF000A720FFF7C1FC02E0A820FFF7BDFC10BDE6
:107B000080B505F02BFA002805D0022808D006D34E
:107B1000032809D00CE0A320FFF7AEFC0BE00AE03D
:107B2000A620FFF7A9FC06E0A720FFF7A5FC02E0CE
:107B3000A820FFF7A1FC01BD80B5DFF82402007882
:107B4000002802D19720FFF797FCDFF81402007895
:107B5000401EDFF80C120870C0B200282BD1DFF8ED
:107B600000024068002826D0802080F3118800BFE2
:107B700000BFDFF8EC01406800280BD0DFF8E0011F
:107B800001210170DFF8D801FFF7CFFCDFF8D00149
:107B900000210170DFF8C8014078F021084202D0CE
:107BA0009920FFF769FCDFF8B8014078002802D17E
:107BB000002080F3118801BD10B5816800290CD028
:107BC000DFF89C11096AC16081680A684968002A67
:107BD00000D051600A6000218160017C11F0030136
:107BE0000174C9B2002943D1DFF874110969002971
:107BF0002AD1DFF86C110861DFF8640100780028F1
:107C00000CD1DFF85C0101210170DFF85401FFF7AE
:107C10008CFCDFF84C010021017003E0DFF840012B
:107C200001214171DFF838014078F021084202D08B
:107C30009920FFF721FCDFF828014078002802D1C5
:107C4000002080F3118813E042694B699342D0D33E
:107C50008142D1D04B699A420AD10300FFE71B68E9
:107C6000002BDFD05C69A242DCD18B42F7D1C0E7A8
:107C700010BD10B504006069002802D1CB20FFF7C9
:107C8000FBFB626936480078401C354908703A4869
:107C900000E008000168002902D04B699A42F8D33D
:107CA000216020620460002909D00C62486990427A
:107CB00002D194F8450000E0002084F84400207CC4
:107CC000002816D1802080F3118800BF00BF20005B
:107CD000FFF772FF22484078F021084202D0992035
:107CE000FFF7CAFB1E484078002802D1002080F32D
:107CF0001188FFF721FF10BD10B519480478184806
:107D00000078401C164908701548FFF70EFC14480F
:107D1000047013484078F021084202D09920FFF700
:107D2000ABFB0F484078002802D1002080F3118877
:107D300010BD10B505F018F9094801210170FFF7D1
:107D400057FB04006846C046021B203A012A03DBA9
:107D5000CD21200005F02CF908480121017010BD4B
:107D6000081F0020DC7000200A710020F470002041
:107D7000E070002009710020141F00200C71002009
:107D8000002803D00249B1F89A170180704700001B
:107D90006C37002010B5DFF8A84500224FF4F071D1
:107DA0002046FAF71BFBDFF89C05606410BD00005D
:107DB00010B5DFF88C45A1894118A181E2898018AE
:107DC000E081207A192803DA401C207284ED110A20
:107DD000DFED700AB4EE600AF1EE10FAC0F29580A1
:107DE00094ED111AB4EE601AF1EE10FAC0F28D8023
:107DF000207A1928C0F2898089B2C329C0F285800F
:107E0000207904EB800080ED280A84ED110AE079E6
:107E1000002804D184ED120A84ED130A17E0D4ED92
:107E2000120A9FED5D1A60EE810A9FED5C1A40EE2A
:107E3000010AC4ED120A94ED130A9FED591A20EEBF
:107E4000010A9FED581A00EE810A84ED130AE089B9
:107E5000B0F57A7F14DDA07904EB8000E16CC0F806
:107E60004011A079401CA071C0B2142801D100209B
:107E7000A071607A142801DA401C60720020E08151
:107E80002279E17914290DD1501C142800D1002049
:107E900094ED0F0A04EB8000D0ED3C0A30EE600A4E
:107EA00084ED0F0A04F1A00000F086F9207904EBBC
:107EB000800080ED3C0AD4ED0F0A30EE800A84ED9C
:107EC0000F0A207904EB8000E16C0165207904EB56
:107ED0004000A1890182E079142801DA401CE07198
:107EE000E07900EE100AB8EE400AD4ED0F0A80EEF9
:107EF000800A84ED100A2079401C2071C0B2142839
:107F000001D1002020710020A08110BDDFF83004D5
:107F100081794A1E00D51432891F00D5143100EB37
:107F2000810191ED500A00EB8200D0ED500A91EDF5
:107F3000501A70EEC10AF5EE400AF1EE10FAD0EDDB
:107F4000500A02DD30EEC00A704730EE600A70471A
:107F5000DFF8EC0381794A1E00D51432891F00D561
:107F6000143100EB810191ED3C0A00EB8200D0ED71
:107F70003C0A91ED3C1A70EEC10AF5EE400AF1EEB2
:107F800010FAD0ED3C0A02DD30EEC00A704730EE48
:107F9000600A70470100FA436666663FD0CCCC3D6C
:107FA000CDCC4C3FCCCC4C3E2DE9F84F2DED088B81
:107FB000F0EE409A074688464FF000094C469FED88
:107FC000798ADFED788A9FED779A9FED76AAA246AF
:107FD000FFB2042F04D1DFED74AA9FED74BA03E061
:107FE000DFED73AA9FED73BADFF8545395F807B02D
:107FF0005E46142E40F0CF80687A0728C0F2CB800E
:10800000F5EE409AF1EE10FA40F3C580FFF77EFFDF
:10801000F0EE40BAFFF79CFFF4EE6BAAF1EE10FA17
:1080200034D5D5ED100AF5EE400AF1EE10FA02DD76
:10803000B0EE601A01E0B1EE601AB4EE41BAF1EEB2
:1080400010FA23D5F5EE400AF1EE10FA01DCF1EE5C
:10805000600A9FED7B1AF4EE410AF1EE10FA15D595
:10806000DFED780AB4EE600AF1EE10FA0ED528685A
:10807000002802D0A86BA8EB000A3B46524659469E
:108080002879401E00F0E4F8814602E0204628608E
:10809000A863B9F1000F7BD02868002803D1C5F888
:1080A000388001202860204605E005EB4101098A5F
:1080B0000C19A4B2401C80B201461429F5DB00EE75
:1080C000104AB8EE400ADFED970A20EE200ADFEDF5
:1080D0005F0A69EEA00A20EE200A2879411E00D529
:1080E0001431801B00D5143005EB8101D1ED140A49
:1080F00005EB800090ED141A70EEC10A9FED521A44
:10810000C0EE819AF4EE409AF1EE10FA02DBDFED58
:10811000259A07E020EE000A09EEE90AFAF742F98B
:10812000B0EE408AB5EE408AF1EE10FA01D0C9EE09
:10813000888A687905EB8000C0ED648A6879401C04
:108140006871C0B2142801D100206871A87A14287F
:1081500001DA401CA872002006E005EB800191EDD9
:10816000640A39EE009A401CA97A0A4680B290420D
:10817000F3D3B2EE040A29EE000A00EE901AF8EEEC
:10818000600A80EE200ADFED680A20EE20AA02E0F5
:1081900020466871A872B0EE4A0ABDEC088BBDE8B3
:1081A000F18F000000000000CDCC4C3EA69B443B6C
:1081B000CDCC4C3D6F12033B10B49FED5C0ADFED5C
:1081C0005B0A9FED5A1ADFED591A00231AE0142CAE
:1081D00000DB143C02EE103AB8EEC22A32EE000A7E
:1081E00050F8244002EE904A70EEA20A02EE221AE3
:1081F00013FB03F402EE104AB8EEC22A72EE211A03
:108200005B1CDBB20C46A34205DA141B1C19641C70
:10821000DDD51434DEE702EE101AB8EE422A22EE63
:10822000011A00EE601A62EE210A40EE400A9FED4C
:10823000400A30EE800A81EE000A10BC7047000050
:108240000AD7233C0AD7A33C8FC2F5BD3B89883CA3
:10825000F0B51C460023002801D5143002E0142894
:1082600000DB14381D461E46042C04D19FED310A54
:10827000DFED310A03E09FED2B0ADFED300A1C46EB
:108280000CE0B4EE410AF1EE10FA06D5B4EE601A35
:10829000F1EE10FA01D5761CB6B2641C0F46E4B2BA
:1082A000A446A7F1010EF4452EDAC71B67447F1CD4
:1082B00001D5143702E0142F00DB143F07F1010C45
:1082C000BCF1140F01DBACF1140CDFF874E00EEB21
:1082D0008C0C9CED141A0EEB8707D7ED141A31EEB7
:1082E000611AFFEE001A20EE212AB4EE421AF1EED6
:1082F00010FAC6D560EEA11AF4EE411AF1EE10FAAA
:10830000BFD56D1CADB2C8E7072A01D20C2000E032
:108310000A20B04201D2012302E0A84200D2022387
:108320001846F0BD6F12833ACDCCCC3D0000000062
:10833000BD3786356F12033B8FC2F53C8FC2753C4B
:10834000045C002000407E44D2B2203A22BF00FAF2
:1083500002F1002070475242D041D2F120029140F8
:108360004140D040904041407047000010B5344C2F
:10837000002208212046FAF731F8204610BD304887
:10838000704710B504462F4804F043FF2E4804F010
:1083900040FF0120607110BD10B5044604F079FF64
:1083A0000120A07110BD38B50446012505F027F85D
:1083B000012804D12846E0700020A0700AE00228BD
:1083C00004D10020E0702846A07003E00020E07097
:1083D000A0700546284632BD10B50446E07905F088
:1083E000D7FA0121217010BD18490A6A0B6A00BF33
:1083F00000BF00BF00BF00BF9B1A8342F6DB70477F
:1084000005F0B8B905F0BAB970B504460025E679AB
:10841000E171FFF7E1FF00280BD00D48007800283C
:1084200002D02046FFF7ADFF2046FFF7B5FF01253C
:1084300003E0E6712046FFF7CFFF284670BD00003D
:108440008C7000200058004000540040081F00209D
:108450000771002005F047BD05F0A9BD05F054BD2A
:1084600005F00EBE05F016BE04F0D0BD04F0DABD76
:1084700005F01ABE10B5FFF779FF044604F001FEBF
:108480000B212046FFF7C0FF05F049F82046FFF713
:10849000E1FF2046FFF787FF002201210846FFF792
:1084A000E7FF0120FFF7E0FF0120BDE81040DDE716
:1084B00070B44FF0004591EA030F44BF6B40FDF7E5
:1084C0007BB900BF841A71EB030604D26E40001B17
:1084D000B141121973414FF4001C1CEB410F34BF22
:1084E0007CEB430684E00C0DA4EB1356362E7DDCAA
:1084F000012E43DC45EAC32343EA525312BFD202A2
:1085000092025B08240545EAC12141EA5051D2EBB1
:10851000C020994125D407D1B0FA80F610FA06F1AF
:1085200064D00020203608E0B1FA81F6B140C6F1EF
:10853000200220FA02F21143B0404FEAF474B4EB87
:10854000465434F001064FEA74040AD8D6F50016F2
:10855000760D04F00044F04061FA06F25040F1401C
:108560004840C00A40EA415021F0004128BF5FEA7C
:10857000500550F1000044EBD12137E045EAC32318
:10858000DB0A45EAC121C90AB6F120050EDD42EA3F
:108590000242120CC5F1200603FA06F6EB4042EA4D
:1085A00006056D42984161F100010DE062FA06F5A1
:1085B000F240554063FA06FC82EA0C02F3405A404E
:1085C0006D42904161EB030111F4801F05D1641EDF
:1085D000620502D06D004041494121F480114308F9
:1085E00075F1004350F1000041EB045170BC70473D
:1085F0001CEB410F15D223F0004352EA43060BD087
:108600004FEA4C0CBCEB410F04D80C0D661E342E07
:10861000B7DDEBE7801A994150EA410608BF002117
:10862000E4E708BF1CEB430F28BF6FF00001DDE754
:1086300080B55A490978491C584A1170017A491E77
:108640000172C9B2002901D105F098FDFFF774FA53
:1086500001BD38B50400524805680BE0287A0028AF
:1086600007D06868A04204D1012028722800FFF7D3
:10867000DFFFED68002DF1D131BD38B50400494868
:108680000078002802D0A120FEF7F6FEFFF713FACB
:108690004348056805E0A54202D1AF20FEF7ECFE95
:1086A000ED68002DF7D140484049016014220021B7
:1086B000200004F07DFC69202074802080F3118864
:1086C00000BF00BF36480068E060354804603348AA
:1086D0004078F021084202D09920FEF7CDFE2F48C5
:1086E0004078002802D1002080F3118831BD38B5D0
:1086F00004002C480078002802D0A120FEF7BCFE20
:10870000FFF7D9F9207C692802D08520FEF7B4FE56
:1087100022480078401C21490870207A002804D1A2
:108720001E4880686060012510E060681B49896808
:10873000884209D01021200005F042FD207A00284F
:10874000F8D1164880686060207A451C2572FFF7D2
:10875000F3F9280032BD10B5040012480078002853
:1087600002D0A120FEF788FEFFF7A5F9207C69283A
:1087700002D08520FEF780FE207A002802D19620C4
:10878000FEF77AFE606805498968884202D09C201D
:10879000FEF772FE2000FFF74BFF10BD081F002000
:1087A000E47000200B710020F87000205386000850
:1087B00000F5E0700268914203D343689A18914231
:1087C00002D380680028F5D17047DFF860070168A0
:1087D00091B94FF4803181604FF4805141604FF086
:1087E000FF31C16001610421DFF844274161C2F813
:1087F000BC11DFF8401701600120704701F1080348
:1088000013F0070305D001F10803C3F1080303F0D7
:1088100007035918D21A8161C26042F001034B600C
:10882000511828234B60DFF804170969C1617047AC
:108830002DE9F04F064601F1080010F0070083B063
:1088400008BF884607D001F10800C0F1080000F019
:10885000070000EB010802F1080010F0070006D045
:1088600002F10800C0F1080000F007008218154668
:10887000A5EB0800A0EB030943F0030003EB080B92
:10888000C8F80400AB4528BF05F0BEFC2879C00736
:1088900058BF05F0B9FCB9F1100F38BF05F0B4FCB2
:1088A000B069854209D1F0684844F060C6F818B054
:1088B00040F00100CBF804006DE1706985420BD1F6
:1088C000B0684844B060C6F814B040F00101CBF87D
:1088D000041040F80B005EE1686800F00301012914
:1088E00040F0AD80C008C0000190C00820283AD2F6
:1088F000D5F808A0EF680090BD4208BF05F084FCE1
:10890000554508BF05F080FC68680099C008C000A4
:10891000B0EBC10F18BF05F077FC009806EBC00064
:1089200000F128018A4507D031698A45C0F082806C
:10893000DAF80C10A9427DD1574506D1009A30686B
:10894000012191408843306076E02830874205D08D
:10895000306987426ED3B868A8426BD1CAF80C70F0
:10896000C7F808A068E0EF68D5F818A0AF420CD0AF
:10897000A8683169884223D3C168A94204BFB96895
:10898000A9421DD1C760B8601CE005F1140007685A
:1089900037B905F110000768A7B101E0084607687C
:1089A00007F114010A68002A02BF07F110010A68E2
:1089B000002AF3D13169884202D30021016001E02D
:1089C00005F022FCBAF1000F36D0E86906EB800012
:1089D00000F5987001688D4208D10760A7B9EA696F
:1089E0007068012191408843706025E030698245BC
:1089F00008D3DAF81000A84214BFCAF81470CAF8F5
:108A0000107001E005F000FCB7B13069874211D366
:108A1000C7F818A0296929B1814226BF39618F6141
:108A200005F0F2FB686938B13169884202D3786198
:108A3000876101E005F0E8FB019845198144686809
:108A40004008400068604FEAD90549F00100CBF8C2
:108A5000040049F80B90202D23D206EBC50000F14D
:108A60002807B9F1100F38BF05F0CEFB306820FAA7
:108A700005F1C907BA4604D40121A9400843306072
:108A800006E0B868316988422CBF824605F0BCFB1D
:108A9000C7F808B0CAF80CB0CBF808A0CBF80C7037
:108AA00079E05FEA192108BF002023D0B1F5803FAB
:108AB00028BF1F201ED2A1F58070000C00F0080016
:108AC0008140A1F58052120C02F004029140A1F500
:108AD00080431B0CC0F10E0003F00203801AC01A81
:108AE000994000EBD130C11D29FA01F202F00101D9
:108AF00001EB4000CBF81C000022CBF81420CBF88F
:108B0000102006EB8001726822FA00F3DB0701F502
:108B1000987107D4012303FA00F010437060C1F884
:108B200000B01DE01F2809680EBF00204008C0F1FA
:108B3000190009FA00F000E011464A68D208D20094
:108B40004A4514D0C20F01EB820202F1100340002B
:108B50001A68002AF0D1306983421AD3C3F800B0F2
:108B6000CBF81810CBF80CB0CBF808B013E0326992
:108B70008868914228BF90420BD3C0F80CB0C1F86E
:108B800008B0CBF80800CBF80C100020CBF8180088
:108B900001E005F039FB08F1080000F005BE2DE901
:108BA000FA4D0546DFF88403006884B008B9FFF782
:108BB0000CFEDFF878030499806841182F31401EBD
:108BC00021EA00000499814280F0AB8105F5D87656
:108BD000B16841B1D5F8B0218018824280F0A181FE
:108BE0008142C0F09E8105F013FB00281EBF0446A1
:108BF000D0F8008014F1010F00F09381D5F8B00196
:108C00004044C5F8B0017168814238BF01467160C7
:108C1000A86980BB286908B1844200D22C61346104
:108C2000C6F814800020F06105F12801BF480068F3
:108C300068624FF0FF3028620020C960896001F14E
:108C40000802801C1031D26020289260F5D3B84809
:108C5000854203D1A8F12802214629E055F8040CE9
:108C6000C00805EBC000A0F1080108EB0400401AA1
:108C7000A0F128021CE005F5E071084600E08068DC
:108C8000D0B1026843689A189442F8D1027B120767
:108C900012D4AA6903689A420ED347683B449A42A9
:108CA0000AD208EB07014160E868A96908EB0002F5
:108CB0002846FFF7A3FD1EE128698442084638BF15
:108CC0002C6108EB040100E0806880B102688A42F0
:108CD000FAD1017B09070AD404604168414441602C
:108CE0002146049B284606B0BDE8F04DA0E5AF69DB
:108CF00039462846FFF75CFD01684068401802903D
:108D00002F3800F1080111F0070105D000F108012A
:108D1000C1F1080101F00701081807F110018842AC
:108D200034BF0097009000980830019004F10801CA
:108D3000009800F1180A11F007014FF0000BA8F19C
:108D4000280005D004F10801C1F1080101F0070174
:108D50000A19401AAA61E86040F0010151608018C8
:108D60002821416071480069E861019810F007000E
:108D700018BF05F049FA00991B20486005F5E0711D
:108D8000B1E80C500198A0E80C503461C6F814808A
:108D9000C6F81CB00198B061029800E08A4607222C
:108DA000CAF804200AF104010A1D82420BF1010BEA
:108DB000F4D3BBF1020FB8BF05F026FA0098B84211
:108DC00000F09980C01BC119C4084A6852085200BB
:108DD0004A6040F001017960C051202C20D205EB9F
:108DE000C40101F12806102838BF05F00DFA2868E3
:108DF00020FA04F1C907B04604D40121A140084378
:108E0000286006E0B068296988422CBF804605F0DA
:108E1000FBF9B760C8F80C70C7F80880FE606AE01C
:108E2000010A08BF002223D0B1F5803F28BF1F22CE
:108E30001ED2A1F58072120C02F008029140A1F539
:108E400080531B0C03F004039940A1F58044240CCB
:108E5000C2F10E0204F00204D21A121BA14002EB6E
:108E6000D131CA1D20FA02F303F0010202EB4102E4
:108E7000FA6100237B613B6105EB82016B6823FA99
:108E800002F4E40701F5987105D4012090401843DD
:108E900068600F601CE01F2A09680EBF002252089C
:108EA000C2F1190200FA02F200E019464B68DB0831
:108EB000DB00834210D0D30F01EB830303F11004D6
:108EC00052002368002BF0D12869844211D3276017
:108ED000B961FF60BF600EE02A698868914228BFCF
:108EE000904206D3C7608F60B860F9600020B86117
:108EF00001E005F089F9E8680499814211D2401A2D
:108F0000E860A969049A5218AA6140F00100506013
:108F1000049840F00300486006B001F10800BDE885
:108F2000F08D002006B0BDE8F08D0000FC6F002041
:108F3000E45D00206859883C2DE9F04D04468846E0
:108F400000265FEA1820C8F1000B08BF002123D0DB
:108F5000B0F5803F28BF1F211ED2A0F58071090CFB
:108F600001F008018840A0F58052120C02F00402C2
:108F70009040A0F580431B0CC1F10E0103F00203E9
:108F8000891AC91A984001EBD030C11D28FA01F2A4
:108F900002F0010101EB400104EB8100D0F8300147
:108FA00028B31F290EBF00224A08C2F1190208FA8D
:108FB00002F2002300E052004768FF08FF00A7EB21
:108FC00008075F4503D25FEA070B06460BD04769E7
:108FD000D50F00EB8500002F00691CBF87423B4680
:108FE0000028E8D1184600283CD1002E3CD10120B1
:108FF00088404000414208436168084000F06781B2
:1090000041420840411E080B00F0100021FA00F216
:10901000510901F0080122FA01F39A0802F004074D
:10902000FB405A0802F00205081823FA05F23844FA
:10903000C2F340032818181822FA03F1081804EBA9
:109040008000D0F830010DE008464168C908C90029
:10905000A1EB080159453CBF8B4606460169002932
:10906000F2D140690028F0D1002E00F03081A068D4
:10907000A0EB0800834580F02A8120698642C0F079
:1090800024817068C008C00008EB0B01884208EB1F
:10909000060518BF05F0B8F8AE4280F01681F768F3
:1090A000D6F818A0B7420CD0B0682169884223D303
:1090B000C168B14204BFB968B1421DD1C760B86090
:1090C0001CE006F11400076837B906F110000768C4
:1090D000A7B101E00846076807F114010A68002AF1
:1090E00002BF07F110010A68002AF3D12169884202
:1090F00002D30021016001E005F086F8BAF1000F0B
:1091000038D0F06904EB800000F5987001688E4259
:1091100009D10760380014D1F269606801219140DB
:109120008843606026E02069824508D3DAF81000A1
:10913000B04214BFCAF81470CAF8107001E005F00C
:1091400063F8BFB12069874212D3C7F818A030690D
:1091500030B12169884226BF3861876105F054F833
:10916000706938B12169884202D37861876101E072
:1091700005F04AF8BBF1100F0CD208EB0B0040F0E1
:109180000300706008EB0B008019416841F0010199
:10919000416096E048F0030070604BF001006860A9
:1091A0004FEADB004BF805B020281DD204EBC001CC
:1091B00001F12807216821FA00F2D207BB4605D445
:1091C000012202FA00F00843206006E0B868216935
:1091D00088422CBF834605F017F8BD60CBF80C50D1
:1091E000C5F808B0EF606CE05FEA1B2108BF002003
:1091F00023D0B1F5803F28BF1F201ED2A1F580707B
:10920000000C00F008008140A1F58052120C02F021
:1092100004029140A1F580431B0CC0F10E0003F045
:109220000203801AC01A994000EBD130C11D2BFAFD
:1092300001F202F0010101EB4000E86100226A61E5
:109240002A6104EB8001626822FA00F3DB0701F572
:10925000987106D4012303FA00F0104360600D609A
:109260001CE01F2809680EBF00204008C0F119004B
:109270000BFA00F000E011464A68D208D2005A45C5
:1092800010D0C20F01EB820202F1100340001A68F5
:10929000002AF0D12069834211D31D60A961ED60DD
:1092A000AD600EE022698868914228BF904206D3E3
:1092B000C5608D60A860E9600020A86101E004F04D
:1092C000A3FF06F10800BDE8F08D04F09DFF00202B
:1092D000BDE8F08D2DE9F84F0446884660684142AC
:1092E0000840411E080B00F0100021FA00F251095D
:1092F00001F0080122FA01F39A0802F0040223FAAD
:1093000002F56B0803F00203081825FA03F610189B
:10931000C6F340051818284426FA05F1081804EB8E
:109320008000D0F830014168C908C9000646A1EBA9
:10933000080A09E008464168C908C900A1EB08010C
:1093400051453CBF8A46064601690029F2D1406971
:109350000028F0D120698642C0F0C4807068C0083F
:1093600008EB0A09C000484508EB060B18BF04F0DB
:109370004BFF5E4580F0B680F768B569B7420CD008
:10938000B0682169884223D3C168B14204BFB9687B
:10939000B1421DD1C760B8601CE006F11400076837
:1093A00037B906F110000768A7B101E00846076861
:1093B00007F114010A68002A02BF07F110010A68C8
:1093C000002AF3D12169884202D30021016001E023
:1093D00004F01AFF002D34D0F06904EB800000F592
:1093E000987001688E4209D10760380011D1F26986
:1093F0006068012191408843606022E020698542D5
:1094000005D32869B04214BF6F612F6101E004F0F9
:10941000FBFEB7B12069874211D3BD61306930B11D
:109420002169884226BF3861876104F0EDFE7069CA
:1094300038B12169884202D37861876101E004F084
:10944000E3FEBAF1100F09D249F00300706009EB96
:109450000600416841F0010141603FE048F003002F
:1094600070604AF00100CBF804004AF80BA0D4F871
:1094700008804FEAD805202D28BF04F0C5FEB8F1BA
:10948000000F27D0D4F81490009504EBC50000F12C
:109490002805B8F1100F38BF04F0B6FE2068009917
:1094A00020FA01F2D1072F4605D4009A01219140FC
:1094B0000843206006E0A868216988422CBF07465F
:1094C00004F0A2FEC5F80890C7F80C90C9F808701F
:1094D000C9F80C50C4F808A0C4F814B006F108008C
:1094E000BDE8F28F04F090FE0020BDE8F28F2DE978
:1094F000F04F83B00546C046C046F52DDFF8C047A3
:1095000080F007810B2D31BF102705F10B00C0083B
:10951000C7002168FE0821FA06F010F0030F42D0C0
:10952000C04300F00100861904EBC60000F12808D2
:10953000F700D8F808506868C008C000B84218BFE3
:1095400004F062FED5F80890454508BF04F05CFEC3
:109550004D4508BF04F058FE6868C008C000B84216
:1095600018BF04F051FEC84505D120680121B14063
:10957000884320600DE02069814508D3D9F80C00AC
:10958000A84204D1C8F80890C9F80C8001E004F0A2
:109590003BFE47F00300686078190835416841F0E8
:1095A00001014160FDE0A168B94280F0C48000285B
:1095B00000F0A680012505FA06F149004A42B040B4
:1095C0001143084041420840411E080B00F01000C2
:1095D00021FA00F2510901F0080322FA03F18A0886
:1095E00002F0040221FA02F6710801F002081818CC
:1095F00026FA08F11018C1F340064044301821FA49
:1096000006F202EB000804EBC80000F128094FEA5B
:10961000C80AD9F808607068C008C000504518BF73
:1096200004F0F2FDD6F808B04E4508BF04F0ECFD9A
:109630005E4508BF04F0E8FD7068C008C0005045F2
:1096400018BF04F0E1FDD94505D1206805FA08F1FD
:10965000884320600DE02069834508D3DBF80C00C7
:10966000B04204D1C9F808B0CBF80C9001E004F086
:10967000CBFD47F003007060AAEB0708B819019012
:1096800048F0010001994860019848F80080A768F7
:109690004FEAD70ABAF1200F28BF04F0B5FD47B34F
:1096A000CDF800A004EBCA00D4F8149000F1280A09
:1096B000102F38BF04F0A8FD2068009920FA01F2AD
:1096C000D107D34605D4009905FA01F1084320607B
:1096D00007E0DAF80800216988422CBF834604F0CD
:1096E00093FDCAF80890CBF80C90C9F808B0C9F8F7
:1096F0000CA0C4F8088006F108050198606150E0EC
:109700006068C0B339462046FFF7E4FD050012D07B
:1097100047E015F1400F28BF4FF0FF370BD205F19E
:109720000B00C008C700606828B139462046FFF723
:1097300003FC050035D1A068B8421CD3C11B626987
:1097400010290AD3B8186061A16041F00103436099
:10975000095047F0030050600AE00021A1606161F8
:1097600040F0030151608018416841F001014160FF
:1097700002F1080515E0E06887420DD2C01BA1691F
:10978000E0607A18A26140F00100506001F1080524
:1097900047F00300486004E039462046FFF7FFF930
:1097A0000546C046C046284603B0BDE8F08F00B964
:1097B00070472DE9F047A0F10804C046C046DFF825
:1097C000005528698442C0F07482616801F0030288
:1097D000012A00F06E82CA084FEAC208CA0708EBE5
:1097E000040936D4226811F0030F00F06482A41A31
:1097F00084429044C0F05D8269698C4200F0D88058
:10980000D608202E70D2D4F80CA0A768544508BF03
:1098100004F0FAFCBC4208BF04F0F6FC6068C00823
:10982000C000B0EBC60F18BF04F0EEFC05EBC6009D
:1098300000F128018F4205D029698F4251D3F96880
:10984000A1424ED1BA453DD128680121B14088439B
:1098500028604C4580F02D82D9F80400C10740F102
:109860002882810700F17A81A969894540F0B58095
:10987000E868AC614044E86040F0010161606969FA
:109880008C4202D100216961A960E969814280F0BE
:109890001282DFF83004006808B9FEF796FFA96964
:1098A000002900F00882E868292824BF2846FEF72E
:1098B0007FFFE869E968884280F0FD814FF0FF3062
:1098C000E861F8E12830824506D02869824508D34E
:1098D000DAF80800A04204D1C7F80CA0CAF8087052
:1098E000B7E704F091FCB4E7E768A669A7420BD09C
:1098F000A168814222D3C868A04204BFB868A042D0
:109900001CD1CF60B9601BE004F114010F6837B9B6
:1099100004F110010F689FB101E011460F6807F1D3
:1099200014021368002B02BF07F110021368002B0A
:10993000F3D1814202D30020086001E004F064FC0E
:10994000002E86D0E06905EB800000F59870016874
:109950008C4209D10760380011D1E26968680121A1
:1099600091408843686074E72869864205D330696E
:10997000A04214BF7761376101E004F045FC002F7D
:109980003FF467AF28698742ABD3BE61216929B133
:10999000814226BF39618F6104F036FC606900287E
:1099A0003FF457AF296988429BD37861876150E7BC
:1099B00099F8040000F0030003287FF44AAFC5F8CB
:1099C0000880D9F8040040084000C9F8040048F0B5
:1099D0000100606048F804806DE16969894508D13B
:1099E000A8686C614044A86040F0010161600051CA
:1099F00061E1C008C0004FEAD00ABAF1200F8044EC
:109A000036D2D9F80C70D9F80860B94508BF04F00F
:109A1000FBFBB14508BF04F0F7FBD9F80400C00810
:109A2000C000B0EBCA0F18BF04F0EEFB05EBCA0094
:109A300000F128018E4206D029698E42C0F0818053
:109A4000F16849457DD1B74206D12868012101FA64
:109A50000AF18843286076E02830874205D02869DB
:109A600087426ED3B86848456BD1F760BE606AE044
:109A7000D9F80C70D9F818604F450DD0D9F8080006
:109A80002969884223D3C168494504BFB96849455B
:109A90001DD1C760B8601CE009F11400076837B930
:109AA00009F110000768A7B101E00846076807F14F
:109AB00014010A68002A02BF07F110010A68002A8F
:109AC000F3D12969884202D30021016001E004F04A
:109AD0009BFB002E37D0D9F81C0005EB800000F569
:109AE0009870016889450AD10760380012D1D9F809
:109AF0001C206868012191408843686023E0286940
:109B0000864205D33069484514BF7761376101E06B
:109B100004F07AFBBFB12869874212D3BE61D9F83D
:109B2000101029B1814226BF39618F6104F06CFBAE
:109B3000D9F8140038B12969884202D37861876165
:109B400001E004F061FB48F00100606048F8048027
:109B5000686984420BD1C5F80880ACE04008400039
:109B6000C9F8040048F00100606048F804804FEA3A
:109B7000D807202F22D205EBC70000F12809B8F141
:109B8000100F38BF04F040FB286820FA07F1C9071E
:109B90004E4604D40121B9400843286007E0D9F8B3
:109BA0000800296988422CBF064604F02DFBC9F83D
:109BB0000840F460A660C4F80C907CE05FEA1820CE
:109BC00008BF002123D0B0F5803F28BF1F211ED23F
:109BD000A0F58071090C01F008018840A0F58052C1
:109BE000120C02F004029040A0F580431B0CC1F15E
:109BF0000E0103F00203891AC91A984001EBD03014
:109C0000C11D28FA01F202F0010101EB4001E161FE
:109C100000226261226105EB81006A6822FA01F389
:109C2000DB0700F5987006D4012303FA01F1114314
:109C3000696004601CE01F2900680EBF002149080C
:109C4000C1F1190108FA01F100E010464268D2089A
:109C5000D200424510D0CA0F00EB820202F110037D
:109C600049001A68002AF0D129698B4211D31C607F
:109C7000A061E460A4600EE02A698168904228BF78
:109C8000914206D3CC608460A160E0600020A061B6
:109C900001E004F0B9FA286A401E28620BD1D5F819
:109CA000C80100E080680028FCD14FF0FF30286236
:109CB00001E004F0A9FAC046C046BDE8F087000004
:109CC000E45D0020FC6F002070B504460026DFF83C
:109CD0000854CA20E8615320E86100F018F8002811
:109CE00011D0286820F040002860286821680843C7
:109CF0002860A068A860A868616840EA0140A86080
:109D000000F024F80126FF20E861304670BD81B0E4
:109D100000200090DFF8C4030168490613D44FF017
:109D2000FF310160016801F04001009A521C00926D
:109D3000009AB2F5803F01D00029F3D00068800975
:109D400000F0010000E0012001B07047DFF88C0353
:109D5000016821F080010160704781B0002000900F
:109D6000DFF87813CA20886153208861086820F0E2
:109D7000A0000860086800F02000009A521C0092C1
:109D8000009AB2F5003F01D00028F3D008684009DE
:109D900000F00100FF228A6101B070472DE9F04117
:109DA00007460E460024DFF82C53002FA86804D184
:109DB00040060AD42046F07007E0400603D530780C
:109DC00000F0A5F901E02046F0703078002F09D0AE
:109DD0007178090241EA0040B1780843F17840EA1D
:109DE000014611E000F088F90746707800F084F928
:109DF0008046B07800F080F94FEA082141EA074137
:109E00000843F17840EA0146CA206862532068623C
:109E1000FFF77DFF00280FD0DFF8C4023040286034
:109E2000FFF794FFA868800605D4FFF796FF002887
:109E300002D0012400E00124FF2068622046BDE832
:109E4000F08110B50C46DFF88C120968DFF890221B
:109E500011400A0C02F03F0323700B0A03F07F034A
:109E6000637001F07F01A17002F04001E1700028F1
:109E70000BD1207800F04BF92070607800F047F9A2
:109E80006070A07800F043F9A07010BDDFF85412A4
:109E9000486A09687047F8B506460D460024002E4A
:109EA00006D16878C10603D500F0EF000A3068706B
:109EB000002E05D0687800F02AF9A87800F027F97C
:109EC000E878002E09D06978090241EA0040A978B3
:109ED0000843297840EA413610E000F00DF90646C3
:109EE000687800F009F90746A87800F005F939020A
:109EF00041EA06410843297840EA4136DFF8E45157
:109F0000CA20286253202862FFF701FF00280FD0E3
:109F1000DFF8D40130402860FFF718FF686880063A
:109F200005D4FFF71AFF002802D0012400E0012425
:109F3000FF2028622046F2BD10B50C46DFF8A411C0
:109F40000968DFF8A42111400A0CE2700A0A02F045
:109F50001F02627001F03F02A270490B01F007017D
:109F6000217000280BD1E07800F0D1F8E070607823
:109F700000F0CDF86070A07800F0C9F8A07010BDB6
:109F8000DFF85411CA22CA615322CA610A68D20892
:109F9000D2000A600A6810430860FF20C861704759
:109FA000DFF84811CA220A6153220A610860FF20C3
:109FB00008617047DFF83401006880B2704781B0F3
:109FC00000210091DFF81011CA22CA615322CA6130
:109FD0000028086804D040F480600860012012E086
:109FE00020F480600860486800F00400009A521C69
:109FF0000092009AB2F5803F01D00028F3D0486863
:10A00000800800F00100FF22CA6101B0704781B0F2
:10A0100000220092364A0092009A02EB80000090E3
:10A020000098016001B0704781B000210091304973
:10A030000091009901EB800000900098006801B049
:10A040007047254ACA23D3615323D36100F0040328
:10A0500020F004000029116805D008431060906BBF
:10A060001843906305E021EA00001060906B98436C
:10A070009063FF20D06170470021184A12681D4B81
:10A080001A40024200D001210846704730B4002136
:10A09000114A936B03F0040314680440050C45EA6D
:10A0A000D0352B402343526802EA101002D000043E
:10A0B00000D00121084630BC704708490003000C5D
:10A0C00040F080000A6802F0800262EA0000086046
:10A0D0007047000000280040082800400C2800407D
:10A0E0007F7F7F00042800403FFFFF0014280040CE
:10A0F000502800407F7F0100002101E0491C0A3800
:10A10000C0B20A28FADA40EA0110C0B27047010969
:10A1100001EB810200F00F0000EB4200C0B270477B
:10A120002DE9F04104460C21206990FBF1F202EB8D
:10A130004201B0EB810144BF0C31521E002A47D5C9
:10A140006069C2F1004398424ADB606915182846ED
:10A1500004F074F840F26D1808FB0500A168E5688A
:10A1600062682368DFF880C0DFF87CE018274FF4CE
:10A17000B46691FBF7F7281892FBF6F6381893FBB4
:10A18000FCFC30186044194D281807EB4705A1EB7B
:10A19000C5014FF4616569430EFB00104FF4B461D3
:10A1A00001FB1621C1EB011200EB820018180EFB17
:10A1B0001C05226A2946204604F05DF8206A012821
:10A1C000A8BFA5F5616504F0FDF8281ABDE8F08187
:10A1D000012ABADB6FF000406369801A9842B4DA52
:10A1E0004FF0FF30BDE8F08180510100209CFFFF5F
:10A1F00013F0004C03D55B42524263F100039CEA2A
:10A20000210C00F0178010B5644603D34942404248
:10A2100061F1000100F00EF8640004D349424042AD
:10A2200061F10001244203D55B42524263F1000315
:10A2300010BD00001B4213D1094236D12AB1844619
:10A24000B0FBF2F002FB10C2704704F009B9FCD376
:10A250000022002370470B000200002100207047FD
:10A26000904271EB030CF6D370B5B1FA81F4B3FAF6
:10A2700083F52C1BA340C4F1200532FA05F63343C5
:10A28000A2405FF00046E64002E05B085FEA32026F
:10A29000841A71EB030524BF204629467641F4D386
:10A2A00002000B003000002170BD012ACFD970B52B
:10A2B000140C20D0B1FA81F4B2FA82F5C4F1200472
:10A2C0006419B4F12006D6D3B2405FF00044F440E4
:10A2D000002502E052085FEA3303C61A71EB020E52
:10A2E00024BF3046714664416D41F3D302000B0038
:10A2F0002000290070BD0C46B1FBF2F102FB1145B4
:10A300002D0445EA1045B5FBF2F402FB145580B26A
:10A3100040EA0545B5FBF2F002FB105240EA04406A
:10A3200070BD000051EC100B00B500F003F841ECDB
:10A33000100B00BD40F2FF7C0B0D4DD0634566D283
:10A3400030B421EA035141F4801103F2FD3C5FEA8D
:10A350005C0C01D300184941890041EA90718000EA
:10A360004FF440140023E202D50AB1F5100107D4DE
:10A370006D081DD2091B641900184941491BF7D506
:10A380006D080AD20919641B00184941491BEFD511
:10A390006D08F7D301E0520817D0C01861419B1A2D
:10A3A000AC4100184941801AA941F4D452080AD09E
:10A3B000C01AA1419B186C4100184941801AA9415B
:10A3C000E9D45208F4D15B1C6C4161084FEA3300B8
:10A3D00001EB0C5130BC704750EA0103FBD030B4A4
:10A3E000B1FA81F311B9B0FA80F41B190B3BB3F148
:10A3F00020042FBF00FA04F19940C3F1200420FA91
:10A4000004F438BF21439840D3F101039DE763452D
:10A41000E1D011F5801FDED850EA4101DBD0D943ED
:10A4200004F020B8002061490860704738B52DED70
:10A43000068BB0EE408AF0EE608AB0EE419A044698
:10A4400020EE000A08EEA80A09EE090A10EE100A2A
:10A45000FBF752F841EC100BFFF764FF51EC100BC7
:10A46000FBF714FA09EE900A9FED4CABB0EE480AE8
:10A4700080EE290A10EE100AFBF73EF841EC100BB3
:10A4800000F036F953EC102B51EC1A0BFBF7B8F82F
:10A49000FBF7FCF908EE100A88EEA90A10EE100A84
:10A4A000FBF72AF841EC100B00F022F953EC102BCB
:10A4B00051EC1A0BFBF7A4F8FBF7E8F908EE900A49
:10A4C00089EE290A10EE100AFBF716F841EC100B82
:10A4D00000F00EF953EC102B51EC1A0BFBF790F82F
:10A4E000FBF7D4F909EE100A002C06D1B2EE040AEB
:10A4F000F0EE409A9FED2BAA05E0B3EE040AF0EED1
:10A50000409A9FED29AA10EE100AFAF7F5FF0246CD
:10A510000B4614461D4618EE100AFAF7EDFF21F01F
:10A52000004122462B46FBF753F82AD219EE900A37
:10A53000FAF7E2FF02460B4614461D4618EE900A53
:10A54000FAF7DAFF21F0004122462B46FBF740F8EC
:10A5500017D219EE100AFAF7CFFF21F00041024698
:10A560000B4614461D461AEE100AFAF7C5FF22469E
:10A570002B46FBF72DF804D20C480168491C0160FA
:10A5800002E000200949086008480068152801DB3E
:10A59000012000E00020BDEC068B32BD46DF617E6D
:10A5A000DCA54C400000A04200008C42C47000209A
:10A5B000B5EEC00AF1EE10FA02D4B1EEC00A70474F
:10A5C0006FF0004C00EE10CA03F04CBFD0B52DED7B
:10A5D000048B82B041EC180B8DED008BDDE900237C
:10A5E000C3F30A5140F2FF72914213D0002904BF15
:10A5F000190350EA113011D051EC180B002200233E
:10A60000FAF7E6FF3DBF81F0004141EC180B08244A
:10A61000002409E0190350EA1130EDD002B051ECEA
:10A62000180BBDEC048BD0BD51EC180B2B4A2C4BF6
:10A63000FAF7CEFF1CD29FED2C9B51EC190B53EC7B
:10A64000182BFDF735FF06460F4653EC182B51EC3F
:10A65000190BFBF7A7F832463B46FAF7D1FFFFF795
:10A6600069FE41EC100B51EC180B53EC102B1EE063
:10A6700001221C4BFAF7ACFF23D29FED1B9B51EC40
:10A68000190B53EC182BFDF713FF06460F4653EC3E
:10A69000182B51EC190BFBF785F832463B46FAF7BD
:10A6A000AFFFFFF747FE84F0020453EC182B03F0D2
:10A6B000DFFE02B02246BDEC048BBDE8D04003F0C3
:10A6C000FBBF04F0F1F82121016002B04FF0FF3030
:10A6D000BDEC048B6FF00041D0BD0000CE3B7F6627
:10A6E0009EA0E63F0000F03F000000000000F03FA9
:10A6F00080B551EC100BFFF769FF41EC100B01BD69
:10A70000002848BF40427047D54800F15C01016510
:10A7100000210162C1614162C16481628170017086
:10A720000121417000210B4603E000EB8102D3625E
:10A73000491C0729F9DB194641608160C16001614C
:10A7400041618161816441658165704738B500244C
:10A75000C34D2878012801D1204632BDE869072879
:10A7600006DBC01FE861A878002801D10120A8708D
:10A77000DFEDB41A9FEDB42A60EE022A95ED013A9E
:10A7800043EE212AC5ED042A20EE823AD5ED023AA5
:10A7900003EEA13A85ED053A61EE020A95ED030A52
:10A7A00040EE210AC5ED060AC5ED012A85ED023A03
:10A7B000C5ED030A22EEA20A03EE030A00EEA00A88
:10A7C000FFF7F6FEE86905EB800181ED0B0AA97839
:10A7D000002900F0CC80411C072291FBF2F2C2EB71
:10A7E000C202891A05EB8101D1ED0B0A70EE600AF5
:10A7F000B0EEE01ADFED951AB4EE611AF1EE10FA40
:10A8000003D5296A491C296206E021462962697834
:10A81000002901D101216970296A652906DB2146D9
:10A82000697029626962E9646965A965A96C002992
:10A830000CD1B1EE001AF4EE410AF1EE10FA41DB50
:10A840000121A964E96C491CE9643BE001290CD1B0
:10A85000E96C491CE9649FED7E1AF4EE410AF1EEC1
:10A8600010FA2FD50221A9642CE002290CD1E96C41
:10A87000491CE9649FED771AF4EE410AF1EE10FAF3
:10A8800020D50321A9641DE003291BD1E96C491CD3
:10A89000E964B9EE001AF4EE410AF1EE10FA11DBA8
:10A8A0001F290CDA696A491C6962022905DBAA6A58
:10A8B000142A02DA491E696201E02146A962214692
:10A8C000A964E964E96C652902DAA96A652903DBF0
:10A8D0002146E964A964A962696A012902DBAA6ABE
:10A8E000521CAA62142902DB012421462970801D12
:10A8F000072190FBF1F1C1EBC101401A05EB80008B
:10A90000D0ED0B0A30EE600A8DED000A032200A99B
:10A91000286D00F031F803221146286D00F040F850
:10A92000DFED4D0AB4EE600AF1EE10FA03D5686D62
:10A93000401C686501E000206865686DC92801DB7E
:10A940000020A865B4EE600AF1EE10FA09DBDFED35
:10A95000400AB4EE600AF1EE10FA02D5A86D401C70
:10A96000A865A86DC92802DB012420462870E86983
:10A97000401CE861204632BD0388934201D3002386
:10A98000038003885B1C03809BB2934201D30022A7
:10A990000280028800EB8200096841600120704754
:10A9A0002DE9F0412DED028B04460D4616469FED34
:10A9B0002B8A0027B4F9008000EE105AF8EEC08A06
:10A9C00000F022F880EE280A04E0A6F101080FFA50
:10A9D00088F87F1C3FB2AF420FDA04EB8800D0ED5D
:10A9E000010A70EEC00A00EEA08AB8F1010FECDB9C
:10A9F000A8F101080FFA88F8EBE788EE280ABDEC09
:10AA0000028BBDE8F081000030B49FED140A0023F2
:10AA1000B0F900400EE024B2250006D400EB850515
:10AA2000D5ED010A30EE200A641E24B2002C00D5B8
:10AA3000541E5B1C1BB28B42EDDB30BC70470848D8
:10AA400040787047D0CCCC3D6666663FCDCCCC3DDF
:10AA500001008040FEFF7FC0CDCCCC3E0000000056
:10AA6000206D002010B50FF2EC40F9F741FEDFF841
:10AA7000DC440022E4212046F7F7B0FC502060605F
:10AA800010BD000030B4DFF8C42492F8D83002EBD7
:10AA90008303C3F8981090ED000A82ED200A0C2180
:10AAA00092F8D83011FB032383ED020A90ED010ADE
:10AAB00002F1800383ED010A92F8D84011FB0424CF
:10AAC00084ED030A90ED020A83ED020A92F8D800A1
:10AAD00011FB002080ED040A92F8D800401C82F897
:10AAE000D80002F1D804C0B20A2804DB002082F8A2
:10AAF000D800012060709FEDD10ADFEDD00A9FEDF4
:10AB0000CF1A00206478012C2ED1044613E011FBEB
:10AB10000425D5ED021A30EE210AD5ED031A70EEA8
:10AB2000A10AD5ED041A31EE211A02EB8405D5F8FD
:10AB300098502818641C0A2CE9DBF2EE041A80EE07
:10AB4000210A83ED030AB2EE040A80EE800A83ED47
:10AB5000040AB2EE040A81EE000A83ED050A0A2116
:10AB6000B0FBF1F0186403E0D86018615861186414
:10AB700030BC7047DFF8D40390F8D900704700006C
:10AB800030B400219FEDAD0ADFEDAC0A9FEDAB1AAA
:10AB90000A46DFF8B83303F18C051CE002EB4204EF
:10ABA00003EB8404D4ED021A93ED232A71EEC21A4A
:10ABB00001EEA10AD4ED031A95ED012A71EEC21A35
:10ABC00041EEA10AD4ED041A95ED022A71EEC21AE3
:10ABD00001EEA11A521C0A2AE0DBF2EE041A81EE01
:10ABE000211ADFEDC51AB2EE042A80EE020AB4EE95
:10ABF000610AF1EE10FA19D5B2EE040A80EE800A6D
:10AC0000B4EE610AF1EE10FA10D5B4EE611AF1EE6D
:10AC100010FA0BD5A96B5A685118A963814203D366
:10AC20000020A863022104E0012102E008462A4630
:10AC30009063084630BC7047C44800F18001D0F8EA
:10AC4000800088644868C8648868086570470000A8
:10AC500010B52DED048B0024BC4901F1800090ED6E
:10AC6000120AD1ED200A30EE608A90ED130AD0ED81
:10AC7000010A70EE608A90ED140AD0ED020A30EEFF
:10AC8000609A00F02FF8DFEDA80A20EE200ADFED31
:10AC9000A70AC0EE209A28EE080A08EEA80A09EED4
:10ACA000090A10EE100AFAF727FC41EC100BFFF727
:10ACB00039FB51EC100BFAF7E9FD00EE100ADFED5D
:10ACC0009C0AB4EE600AF1EE10FA07DB9FED990AD8
:10ACD000F4EE409AF1EE10FA00DB01242046BDECC0
:10ACE000048B10BD10B52DED068B04469FED538AE5
:10ACF000964800F1C801D1ED028A91ED019AD0ED9C
:10AD0000329A29EEA90A09EE090A08EEA80AFFF705
:10AD10004FFCB0EE40AAD4ED020A94ED011A94ED76
:10AD2000000A20EE000A01EE010A00EEA00AFFF779
:10AD30003FFCD4ED000A69EEA00A94ED011A49EE39
:10AD4000010A94ED021A48EE810A2AEE000A80EE0A
:10AD5000800ADFED790AB4EE600AF1EE10FA1EDA2D
:10AD6000DFED760AB4EE600AF1EE10FA02D59FED3F
:10AD7000748A14E0DFED730AB4EE600AF1EE10FAA3
:10AD80000DDAFFEE000AB4EE600AF1EE10FA02D519
:10AD90009FED6B8A03E003F08DFDB0EE408AB0EECC
:10ADA000480ABDEC068B10BD80B52DED028B6748BF
:10ADB00000F1800191ED028AD1ED010A90ED200AA7
:10ADC00020EE000A00EEA00A08EE080AFFF7F0FBEA
:10ADD00088EE000A03F0A0FDDFED5B0A20EE200AFA
:10ADE000BDEEC00A10EE100ABDEC028B02BD80B5AC
:10ADF000FFF7DAFF10F1460F03DA5449086001202B
:10AE000002BD002002BD80B5FFF7CEFF4F490968A3
:10AE10000A1A00D5421A4E48282A03DB0168491C49
:10AE2000016001E0002101600168032903DB0021CA
:10AE30000160012002BD002002BD000000000000F2
:10AE4000F0B58BB000A80FF218112822F7F704FB19
:10AE500000243E4D05F1C006707E002801D164201B
:10AE600048E0012000E0401C05280DDAD5F8C010AC
:10AE700000AA52F830209142F5D300AA02EBC0029A
:10AE800052688A42EFD3044695F8E00005F1E007E6
:10AE9000E4B2A04207D17978A14204D0F069696890
:10AEA0000818F06114E0A04212D0042C02D1797885
:10AEB0008C4201D1002807D1D5F8C02079780FF253
:10AEC000C800F9F715FC7C700020F06185F8E040BF
:10AED000F06947F23051884209D395F8E02079783B
:10AEE0000FF2BC00F9F704FC0020F0617C70787868
:10AEF0006430C0B20BB0F0BD9A99993E002013495E
:10AF000001F1C002D1F8C0300A2B04D3536949685B
:10AF1000C918516101E0014651615169B1F57A7F6B
:10AF200001D35061012070470000B443D80FC940DD
:10AF30000100E040010070416766663F666666BFDB
:10AF4000D80F49400100803FE42E6542AC690020E3
:10AF5000C0700020234450434D20494E4954000006
:10AF60009CFFFFFFFFFFFFFF00000000020000004A
:10AF70000300000032000000330000006400000005
:10AF800065000000FFFFFF7F4450434D206272695F
:10AF90006768742075702025642025640000000017
:10AFA0004450434D204C7578206368616E6765643A
:10AFB0002025642D3E2564001EF0040F0CBFEFF326
:10AFC0000880EFF3098000F03DB870471EF0040FD1
:10AFD0000CBFEFF30880EFF3098000F033B8FEE711
:10AFE0001EF0040F0CBFEFF30880EFF3098000F0B0
:10AFF00029B870471EF0040F0CBFEFF30880EFF381
:10B00000098000F01FB870471EF0040F0CBFEFF36B
:10B010000880EFF3098000F015B870471EF0040FA8
:10B020000CBFEFF30880EFF3098000F00BB8704716
:10B030001EF0040F0CBFEFF30880EFF3098000F05F
:10B0400001B87047F9F715BB38B50C46DFF8AC55B9
:10B050002968C90706D5296849084900296029686F
:10B06000C907FCD400220146284600F0D5FCDFF8D1
:10B070009015284600F0EDFC214628464160C04668
:10B0800001212846BDE8344000F0B0BCF8B5DFF837
:10B0900074452078401C2070DFF86C552878401CDF
:10B0A0002870FCF72DFD6878F021084202D0992025
:10B0B000FCF7E2F9FCF756FA6878401C687002F079
:10B0C000CFFE6878F021084202D09920FCF7D4F92D
:10B0D0006878401E6870C0B2002801D1FCF73CFAC5
:10B0E000012003F07FFC012840F08E80012003F056
:10B0F00081FCDFF81805007800281CD1FCF732FA33
:10B100002078411E2170002802D19820FCF7B4F964
:10B110002878012804D16868002801D0FCF718FAC3
:10B120002878401E2870FCF717FA0FF20450BDE88B
:10B13000F240F9F72EB900260121DFF8D40400F01F
:10B140007BFB002855D0DFF8CC64DFF8B0743846BC
:10B1500000F068FC002826D03046461E0028F6D1B4
:10B160000021DFF8B40400F041FC0021384600F073
:10B170003DFC0FF2C440F9F7BBFA0120FDF776F968
:10B18000FCF7F0F92078411E2170002802D19820A8
:10B19000FCF772F92878012848D16868002845D062
:10B1A000FCF7D6F942E04FF48051DFF8700400F06C
:10B1B00043FB002812D0FCF7D5F92078411E2170FE
:10B1C000002802D19820FCF757F9287801282DD1C2
:10B1D000686800282AD0FCF7BBF927E0DFF84014A4
:10B1E000DFF8400403F00EFC06460120FDF73EF9AF
:10B1F00004E0DFF834140220FAF7FCFD002E03D03F
:10B200000FF23C40F9F7C5F8FCF7ACF92078411E85
:10B210002170002802D19820FCF72EF92878012807
:10B2200004D16868002801D0FCF792F92878401E04
:10B230002870BDE8F140FCF78FB938B5DFF8C4439A
:10B240002078401C2070DFF8C0532878401C2870FC
:10B25000FCF756FC6878F021084202D09920FCF7F0
:10B260000BF9FCF77FF96878401C687002F0F8FD74
:10B270006878F021084202D09920FCF7FDF8687840
:10B28000401E6870C0B2002801D1FCF765F90420A7
:10B2900003F0A8FB002827D0042003F0ABFBDB4819
:10B2A000007800281CD1FCF75DF92078411E217040
:10B2B000002802D19820FCF7DFF82878012804D173
:10B2C0006868002801D0FCF743F92878401E2870F0
:10B2D000FCF742F90FF27830BDE83240F9F759B87F
:10B2E000D2491020FAF786FDFCF73CF92078411E80
:10B2F0002170002802D19820FCF7BEF82878012898
:10B3000004D16868002801D0FCF722F92878401E93
:10B310002870BDE83140FCF71FB938B5B94C20782A
:10B32000401C2070B84D2878401C2870FCF7E8FBC2
:10B330006878F021084202D09920FCF79DF8FCF7CC
:10B3400011F96878401C687002F08AFD6878F02175
:10B35000084202D09920FCF78FF86878401E687088
:10B36000C0B2002801D1FCF7F7F8082003F03AFB3F
:10B37000002827D0082003F03DFBA44800780028CF
:10B380001CD1FCF7EFF82078411E2170002802D173
:10B390009820FCF771F82878012804D16868002803
:10B3A00001D0FCF7D5F82878401E2870FCF7D4F8B7
:10B3B0000FF2A420BDE83240F8F7EBBF9B4908200C
:10B3C000FAF718FDFCF7CEF82078411E217000280E
:10B3D00002D19820FCF750F82878012804D1686839
:10B3E000002801D0FCF7B4F82878401E2870BDE88A
:10B3F0003140FCF7B1B838B5824C2078401C207041
:10B40000814D2878401C2870FCF77AFB6878F02181
:10B41000084202D09920FCF72FF8FCF7A3F86878CF
:10B42000401C687002F01CFD6878F021084202D0D0
:10B430009920FCF721F86878401E6870C0B2002897
:10B4400001D1FCF789F84FF48050FEF71FFE002869
:10B450002ED06E48007800284FF4805022D1FEF79D
:10B460002CFE4FF4003003F0C5FAFCF77BF820788F
:10B47000411E2170002802D19820FBF7FDFF28789B
:10B48000012804D16868002801D0FCF761F8287809
:10B49000401E2870FCF760F80FF2C410BDE832407F
:10B4A000F8F777BFFEF709FE4FF4003003F0A2FA79
:10B4B000FCF758F82078411E2170002802D198200E
:10B4C000FBF7DAFF2878012804D16868002801D04A
:10B4D000FCF73EF82878401E2870BDE83140FCF7A4
:10B4E0003BB8F0B585B0474C2078401C2070464DE5
:10B4F0002878401C2870FCF703FB022003F090FB27
:10B50000002862D00021022003F06DFB022003F02E
:10B510008FFB002003F0BCFA00A90020FEF791FC8D
:10B52000012003F0B1FB01214FF4802003F019FB4F
:10B530000F20FEF779FD06461020FEF775FD074641
:10B54000012003F00BFB002003F008FB31460F2025
:10B55000FEF75DFD39461020FEF759FD00214FF43E
:10B56000802003F0FEFA012003F082FA01214FF05F
:10B57000805003F001FB4FF4807003F0D9FA3F20B4
:10B58000029040F2FF1003900020019001A8FEF706
:10B590009BFB00A90020FEF701FC012003F0DBFA71
:10B5A000FEF7DBFB0320FEF7EBFC4FF48040FEF7D9
:10B5B00084FD4FF4800003F01DFA01214FF4804018
:10B5C000FEF73FFD022003F033FBFBF7CBFF2078B3
:10B5D000411E2170002802D19820FBF74DFF2878EA
:10B5E000012804D16868002801D0FBF7B1FF287852
:10B5F000401E2870FBF7B0FF05B0F0BD106402409C
:10B600002000001009710020081F00200771002091
:10B6100000000240809698005864024000040240F6
:10B62000646E0020083F0020404A002018370020A8
:10B6300045585449302D52004558544930000000B7
:10B640004D534720426F782046756C6C0000000017
:10B6500045585449352D520045585449322D520011
:10B66000525443414C2D520080B54B49884209D178
:10B670000121084603F096FA00210120BDE80440AC
:10B6800003F090BA4549884209D10121022003F014
:10B6900089FA00210220BDE8044003F083BA404942
:10B6A000884209D10121042003F07CFA0021042002
:10B6B000BDE8044003F076BA3A49884209D1012135
:10B6C000082003F06FFA00210820BDE8044003F0D1
:10B6D00069BA3549884209D10121102003F062FA84
:10B6E00000211020BDE8044003F05CBA2F498842D5
:10B6F00009D10121202003F055FA00212020BDE8C6
:10B70000044003F04FBA2A49884209D10121402060
:10B7100003F048FA00214020BDE8044003F042BA9B
:10B720002449884209D10121802003F03BFA0021FD
:10B730008020BDE8044003F035BA1F4988420BD190
:10B7400001214FF4807003F02DFA00214FF4807036
:10B75000BDE8044003F026BA184988420BD1012104
:10B760004FF4007003F01EFA00214FF40070BDE8A2
:10B77000044003F017BA124988420BD101214FF45B
:10B78000806003F00FFA00214FF48060BDE80440B0
:10B7900003F008BA01BD00000000024000040240AE
:10B7A00000080240000C0240001002400014024059
:10B7B00000180240001C0240002002400024024009
:10B7C00000280240F0B4002232E0012393400C68CC
:10B7D0001C409C422BD154000325A540ED43066834
:10B7E0002E40066006680F79A7403E4306600E793A
:10B7F000012E01D0022E11D186682E408660866807
:10B800004F79A7403E438660466826EA03034360BB
:10B8100043688E799640B6B233434360C3682B4089
:10B82000C360C368CD7905FA04F42343C360521C96
:10B83000102ACAD3F0BC704700220069084200D029
:10B84000012210467047018370474183704710B44E
:10B85000CB1000EB830001F007018900036A0F247D
:10B860008C40A3430362036A02FA01F119430162A7
:10B8700010BC70470168490849000160002101605F
:10B8800041608160C1600161212141619D4988421F
:10B8900003D13D209C49086070479C49884204D1EF
:10B8A0004FF474609849086070479949884204D100
:10B8B0004FF474109449086070479649884204D147
:10B8C0004FF074609049086070479349884203D1F3
:10B8D00092488D49486070479149884203D1914808
:10B8E0008949486070479049884203D18F4886490A
:10B8F000486070478E49884204D14FF03D508249DC
:10B90000486070478B49884203D13D208A490860CE
:10B9100070478A49884204D14FF4746086490860B0
:10B9200070478749884204D14FF4741082490860F7
:10B9300070478449884204D14FF074607E490860A2
:10B9400070478149884203D174487B4948607047F9
:10B950007E49884203D173487749486070477C49E3
:10B96000884203D1714874494860704779498842D8
:10B9700003D14FF03D507049486070470268764BE4
:10B980001A400B681A43CB681A434B691A438B69F8
:10B990001A43CB691A430B6A1A434B6A1A438B6AE0
:10B9A0001A434B6B1A438B6B1A4302604269D208ED
:10B9B000CB6A53EAC2020B6B1A4342610A694260C6
:10B9C0004A6882608968C1607047002101604160F7
:10B9D0008160C160016141618161C1610162416257
:10B9E0008162C1620163416381637047002901681C
:10B9F00003D041F00101016070474908490001602E
:10BA000070470029016803D041F48021016070472C
:10BA100021F4802101607047002A01D00161704744
:10BA2000C1607047006800F0010070470022414B80
:10BA3000984201D2494800E049488B0001D540684E
:10BA400000E0006808404749084200D00122104643
:10BA50007047384A904201D2404800E04048414A8D
:10BA60000A40890001D5C2607047826070470B06AA
:10BA700009D5002A436903D043F08003436102E003
:10BA800023F08003436180290AD001F01E01002ABF
:10BA9000026802D011430160704722EA010101608F
:10BAA000704710B40022234B984201D22B4B00E088
:10BAB0002B4B2D4C214205D0006800EAD12000F02C
:10BAC0001E0002E0406900F080008C0001D55B6838
:10BAD00000E01B681940234B194202D0002800D017
:10BAE0000122104610BC7047124A904201D21B48F6
:10BAF00000E01B481B4A0A40890001D5C26070471C
:10BB00008260704710600240086002402860024076
:10BB10004060024058600240706002403D000020DA
:10BB200088600240400F0020A060024000003D20DD
:10BB3000B860024010640240086402402864024079
:10BB400040640240586402407064024088640240CD
:10BB5000A0640240B86402403F801CF000600240D4
:10BB6000006402407D0F7D0F3C0F3C0F38B5040090
:10BB70000D0017480078401C1549087015480078DA
:10BB8000002802D0A120FBF777FCFBF794FFA07EF2
:10BB9000662802D08220FBF76FFC802080F311889A
:10BBA00000BF00BF08E03821200002F009FB802020
:10BBB00080F3118800BF00BFE06821698842F2D09D
:10BBC0002900200003F06AF8FBF7B6FF31BD00BF83
:10BBD000081F00200B71002010B504001F480078DA
:10BBE000002802D0A120FBF747FCFBF764FF1C48AC
:10BBF0000078401C1A490870802080F3118800BF2B
:10BC000000BF174880688069204209D114488068C5
:10BC1000C46113488068082101741148FBF785FC52
:10BC20000F48806884690E488068002181610C4853
:10BC30000078401E0A49087009484078F0210842FF
:10BC400002D09920FBF718FC05484078002802D163
:10BC5000002080F31188200010BD00BF0B71002070
:10BC6000081F002038B504000D0016480078401C5D
:10BC70001449087014480078002802D0A120FBF76E
:10BC8000FBFBFBF718FFA07E662802D08220FBF7A3
:10BC9000F3FB802080F3118800BF00BF08E0402143
:10BCA000200002F08DFA802080F3118800BF00BFD1
:10BCB000E0680028F3D02900200003F01AF8FBF711
:10BCC0003BFF31BD081F00200B7100202DE9F04122
:10BCD00004000D0016001F00802080F3118800BFB3
:10BCE00000BF2248D0F8008006E0A04502D1AC2079
:10BCF000FBF7C2FBD8F80480B8F1000FF5D11C485F
:10BD00004078F021084202D09920FBF7B5FB184893
:10BD10004078002802D1002080F31188FBF7A3FEB1
:10BD20001C220021200001F043F9A7602661258331
:10BD30006620A076802080F3118800BF00BF0B48EA
:10BD4000006860600948046009484078F0210842B2
:10BD500002D09920FBF790FB05484078002802D1DB
:10BD6000002080F31188BDE8F0810000E870002019
:10BD7000081F00202DE9F84304000E0017001D00E5
:10BD8000DDF828802E480078002802D1A520FBF796
:10BD900073FBFBF790FE2B48D0F80C9006E0A14512
:10BDA00002D1AA20FBF768FBD9F80090B9F1000F87
:10BDB000F5D154220021200001F0FAF8642084F823
:10BDC00050006761207C204909780843207484F87A
:10BDD0004580002E00D06662089EE662099FA76239
:10BDE0003A00CD21300001F0E3F8BE19F608F60064
:10BDF000503E002030605FF0807070641348306403
:10BE0000F5647FF0020070621148F06211483063FF
:10BE100011487063114870601148B0601148F060BB
:10BE200011483061114870611148B0611148F061EA
:10BE30001148306266602000FBF71BFFBDE8F1830C
:10BE40000C710020081F002008710020F774000802
:10BE50000100CCCC0200CCCC0300CCCC0400CCCC78
:10BE60000500CCCC0600CCCC0700CCCC0800CCCC58
:10BE70000900CCCC0A00CCCC0B00CCCC80B53B4923
:10BE800088420BD101214FF4805002F0A1FE002125
:10BE90004FF48050BDE8044002F09ABE3449884215
:10BEA0000BD101214FF4804002F087FE00214FF4B6
:10BEB0008040BDE8044002F080BE2E4988420BD18C
:10BEC00001214FF4004002F078FE00214FF40040C1
:10BED000BDE8044002F071BE274988420BD1012120
:10BEE0004FF4005002F074FE00214FF40050BDE802
:10BEF000044002F06DBE214988420BD101214FF46C
:10BF0000801002F065FE00214FF48010BDE804406F
:10BF100002F05EBE1A4988420BD101214FF4001095
:10BF200002F056FE00214FF40010BDE8044002F07C
:10BF30004FBE01BD028802F441520B881A434B8860
:10BF40001A438B881A43CB881A430B891A434B89AF
:10BF50001A438B891A43CB891A430280828B4FF292
:10BF6000FF731A408283098A0182704700300140C2
:10BF700000380040003C00400034014000500140C7
:10BF8000005401400029018803D041F040010180A4
:10BF900070474FF6BF72114001807047002A8288B7
:10BFA00002D011438180704722EA010181807047ED
:10BFB00000220089084200D001221046704700008C
:10BFC0002DE9F04FA1B08246002017461D46029190
:10BFD0000B900DF1440B6FF000490AE017F8011BBC
:10BFE0000298D0470290002800F0A8820B98401CCD
:10BFF0000B90387808B90B98A2E22528EED10020E2
:10C00000059006900790089009900A9001E040F092
:10C01000010017F8011F2029F9D023290DD02B2961
:10C0200004D02D2906D030290AD00CE040F00200BF
:10C0300080B2EEE740F00400FAE740F00800F7E7CE
:10C0400040F01000F4E72A290ED12968296051F840
:10C05000042B2960002A0D9204D5514240F00400BF
:10C060000D9180B27F1C11E000210D9109E00D9926
:10C07000494505D001EB810302EB430130390D91B5
:10C080007F1C3A78A2F130010A29F0D339782E29A1
:10C0900003D04FF0FF310C911DE017F8011F2A2942
:10C0A00007D1296829607F1C51F8042B29600C9264
:10C0B00011E000210C9109E00C99494505D001EBF4
:10C0C000810302EB430130390C917F1C3A78A2F1D5
:10C0D00030010A29F0D3ADF838000FF674403978F2
:10C0E00002F048FE08B117F8010B8DF83A009DF8F0
:10C0F0003A00682802BF39786829622005D06C2888
:10C1000004BF38786C2803D171208DF83A007F1C69
:10C1100011A8049017F8014BB4F125002AD01C385F
:10C1200000F0CC80001F022840F2C880133800F0D5
:10C13000EE80093800F0C280801E00F04F81401E62
:10C1400000F02481401E022840F2B880001F00F059
:10C150001D81401F00F08380401E00F0D880401EEB
:10C1600029D0C01E0CD0801E00F0D180C01E00F06F
:10C17000CE803DE10120059025208DF8440043E16B
:10C180002868286050F8044B28600394DDF830805C
:10C19000B8F1000F04D52046FBF752F9804607E0BE
:10C1A00042460021204602F0F1FD08B1A0EB040850
:10C1B000CDF8188028E1296829604FF03C0851F833
:10C1C000040B29600021CDE9000111A80390DDE9ED
:10C1D0000001049C11B908B90C9AC2B10206120FF1
:10C1E000A0EB02123032D2B23A2AA8BF273200099D
:10C1F000A8F1010340EA017009091A5508BF002897
:10C20000984604D0039A08EB04039A42E6D308EB5D
:10C2100004000390C8F13C010C980691814209DAB0
:10C22000401A08904FF6EF71BDF838000840ADF89D
:10C230003800E9E0002840F1E7809DF8380000F080
:10C240001400102840F0E0800D98059A801A089A92
:10C25000801A401A0128C0F2D7800890D4E09DF8D7
:10C260003A0062281AD0682806D06A280CD06C28B8
:10C270001CD0712808D019E02868286050F8041BE9
:10C2800028600B980880BFE02868286050F8042BCD
:10C2900028600B98C117C2E90001B5E02868286042
:10C2A00050F8041B28600B980870ADE028682860DF
:10C2B00050F8041B28600B980860A5E02868C01D92
:10C2C00020F007022A60D2E9000108322A60CDE995
:10C2D0000001002903D5012005902D200CE0BDF8B8
:10C2E0003800810703D5012005902B2004E0C0070A
:10C2F00004D50120059020208DF84400059911A84F
:10C3000008180390214600A800F0D8F97CE09DF8B9
:10C310003A206C2A0DD0712A18BF6A2A09D12868E0
:10C32000C01D20F007032B60D3E9000108332B6008
:10C3300005E02968296051F8040B29600021CDE946
:10C340000001682A08BF80B207D0622A08BFC0B2C5
:10C3500003D0742A18BF7A2A02D10021CDE9000146
:10C360009DF83800000730D5DDE90001002908BF3D
:10C3700000282AD044F02000782826D130208DF8DB
:10C3800044008BF80140022005901EE09DF83A0021
:10C39000294600F0D8F8CDE90001002904DA059813
:10C3A000411C05912D210EE0BDF83800810704D510
:10C3B0000598411C05912B2105E0C00705D505987E
:10C3C000411C0591202100F80B10059911A80818AF
:10C3D0000390214600A800F0EDF815E0012005903B
:10C3E0002868286050F8041B28608DF844100BE082
:10C3F000012005902520002C8DF8440004D00598DC
:10C40000411C059100F80B400D980599401A0899B8
:10C41000401A0699401A0999401A0799401A0A9930
:10C42000A0EB01089DF8380040070FD420208DF8BC
:10C430004000002408E0012310AA00A9504600F0A3
:10C4400070FC00287AD1641C4445F4DB059C11AED5
:10C450000AE016F8011B0298D047029000286DD020
:10C460000B98401C0B90641E002CF2D130208DF8EC
:10C4700040000026089C08E0012310AA00A95046AD
:10C4800000F04FFC002859D1761CA642F4DB069C34
:10C49000039E0AE016F8011B0298D047029000287C
:10C4A0004CD00B98401C0B90641E002CF2D1302015
:10C4B0008DF840000026099C07E0012310AA00A97E
:10C4C000504600F02EFCC8BB761CA642F5DB039854
:10C4D0000699079C0E1809E016F8011B0298D04730
:10C4E000029058B30B98401C0B90641E002CF3D1A3
:10C4F00030208DF8400000260A9C07E0012310AA96
:10C5000000A9504600F00DFCC0B9761CA642F5DB30
:10C510009DF8380040077FF56CAD20208DF8400075
:10C52000002400E0641C4445BFF663AD012310AA5B
:10C5300000A9504600F0F5FB0028F3D04FF0FF3083
:10C5400021B0BDE8F08F622826D068281DD06A2867
:10C5500008D06C2827D0712804D0742823D07A28DA
:10C560000CD020E00868C01D20F007000860D0E96A
:10C570000023083008601946104670470A680A60B0
:10C5800052F8040B0A60002170470A680A6052F8EA
:10C59000040B0A6000B20BE00A680A6052F8040B50
:10C5A0000A6040B204E00A680A6052F8040B0A60AC
:10C5B000C11770472DE9FA4E05460A462F696F2AC2
:10C5C00008BF082405D041F02000782814BF0A24B1
:10C5D00010243C26D5E90001642A18BF692A814647
:10C5E0008A4605D1002903DAD9F100096AEB4A0A23
:10C5F000BAF1000F08BFB9F1000F0CD1286B50B988
:10C60000082C36D195F83800000732D530203B266B
:10C6100087F83B002DE0E317484651462246FDF7D8
:10C6200009FEA4FB0023A9EB02023032D2B2A6F12C
:10C63000010B3A2A5E4603DB9DF80030513B9A1805
:10C6400081465FEA010A0BF8072008BFB9F1000F25
:10C6500003D0E868F1198842DDD3082C09D195F898
:10C660003800000705D5F05D302802D0761E302056
:10C67000F055C6F13C00A861F119E960296B8842C8
:10C6800008DA081A28624FF6EF71288F08402887C9
:10C69000BDE8F38E00290ED595F8381001F014018D
:10C6A000102908D1696B6A69891A2A6A891A081AD5
:10C6B0000128A8BF2862BDE8F38E00002DE9F24FE3
:10C6C00004468EB0D4E90001CDE9020104AF9DF823
:10C6D000380040F0200BBBF1610F0AD0206B00281E
:10C6E00048BF062004D408BFBBF1670F01D1012069
:10C6F00020636168C1F30A5040F2FF7290421CD17E
:10C70000080304BF2068002809D10320A0619DF818
:10C71000380061381A2836D30FF2486108E0032048
:10C72000A0619DF8380061381A2829D30FF22C61D6
:10C73000E0680322F5F780FEBEE1012816DA204604
:10C7400002F050FB012811DB00250020BBF1610F36
:10C7500020D1E168302201F8012B4A1CE2609DF8EB
:10C760003820612A0CBF782258220FE0626840F21C
:10C77000FE3161F31E52451A62604FF0FF30E5E76B
:10C780000FF2D451D4E70FF2D851D1E70A706169A2
:10C79000891C616110B90026002584E1BBF1610F9D
:10C7A00040F09780206B00284CBF2126461CDDE915
:10C7B0000201D4E900AB00220023F8F709FF36B2EA
:10C7C0003ABF8BF00040CDE902A0CDE902AB06F103
:10C7D00001082D1F8DF810200DF1110700E0C71D75
:10C7E000B8F1010F33DBDDE9020100220023F9F784
:10C7F00095F82CD21C2102A802F016FBDDE90201FB
:10C80000F8F7BAFEA8F10708B8F1010F814609DB75
:10C81000F8F79AFE02460B46DDE90201FBF748FEF7
:10C82000CDE90201F81D072105E009F00F0200F82B
:10C83000012D4FEA2919B9F1010F01DB491EF4D589
:10C84000491E5CBF002200F8012DF9D5C7E70DF1A4
:10C850001100391AB142B8BF0E4636B230000DF1A0
:10C8600011072FD4884206DA04A94118497808290B
:10C87000A8BF0F2100DA002104AA821800E0761E6A
:10C8800012F80139401E8B42F9D00F2904D104A9B6
:10C8900041184A78521C4A70002802D504AF761C11
:10C8A0002D1D36B2701E0DD4C1190A783032D2B2A5
:10C8B0003A2A03DB9DF838303A3B9A18401E01F8BB
:10C8C0000129F2D5206B002840F1ED80701E206315
:10C8D000E9E0DDE9020100220023F8F779FE3CBF20
:10C8E00081F00041CDE902012DB247F29750684333
:10C8F0004B49DFF8309190FBF1F52DB2C5F1070AF5
:10C90000BAF1010F90461CDBDDE902675FEACA70ED
:10C9100007D542464B4630463946F8F771FE064683
:10C920000F464FEA6A0A4046494642464B46F8F7E8
:10C9300067FEBAF1000F80468946E7D1CDE902676C
:10C9400024E0CAF1000A0026374F14E05FEACA70FB
:10C9500007D542464B4630463946F8F751FE064663
:10C960000F464FEA6A0A4046494642464B46F8F7A8
:10C9700047FE80468946BAF1000FE7D1DDE90201A2
:10C9800032463B4601F074FDCDE90201BBF1660F72
:10C99000216BDFF898900CBF05F10A0006204618BD
:10C9A000142EA8BF132630208DF810000DF11107AA
:10C9B000012E3DDBDDE90201F8F7F4FD07F1080186
:10C9C00004220A23B0FBF3F303EB8307A0EB470039
:10C9D000303001F8010D0A20B3FBF0F000EB8007C6
:10C9E000A3EB47033033521E01F8013DE9D1083E65
:10C9F000012E01F10807DBDBDDE90201F8F7D2FDCA
:10CA0000F8F7ACFD02460B46DDE90201FBF750FDED
:10CA100000224B46F8F7F4FDCDE90201CAE700BF5A
:10CA2000A0860100000024400000F03F84D7974119
:10CA30000DF11100381A0DF1110702E0401E6D1EB4
:10CA40007F1C39783029F9D0BBF1660F02D12DB2A5
:10CA5000691C04E0BBF1650F0CBF01210021226BB2
:10CA60008E1836B2B042B8BF064636B231001AD47C
:10CA7000814204DAC85D3528A8BF392000DA3020A9
:10CA8000CA19521E00E0761E12F80139491E83426F
:10CA9000F9D0392802D1C85D401CC855002902D5FB
:10CAA0007F1E761C6D1C2DB29DF83810009533B298
:10CAB0003A46204600F003F80FB0BDE8F08F2DE9AC
:10CAC000F043054685B01E46D5F83080012E8946D4
:10CAD000174602DA01260FF2902749F02000BDF92F
:10CAE0003040662808BF641C17D0672840F0828059
:10CAF00014F1040FC0F28480444580F2818095F8DF
:10CB00003800641C000702D44645B8BFB04624B2C2
:10CB1000B8EB040848BF4FF0000824B2E868A969E0
:10CB2000012C25DA4A1C30230B54B8F1010F03DA2B
:10CB300095F83810090702D52E211154521C18EB14
:10CB4000040FB8BFC8F1000424B26142A044B0454C
:10CB5000AA61B8BF4646696236B2EE613246AB6939
:10CB600039461818F5F768FCA8EB0600A862C1E082
:10CB70000818A64218DA32463946F5F75DFCA9696D
:10CB80007118A01BA961B8F1010F686203DA95F86A
:10CB90003800000705D5EA682E208854E869401C53
:10CBA000E861C5F82880A5E022463946F5F744FC3F
:10CBB000A8692018361BB8F1010F03DA95F8381070
:10CBC000090703D5EA682E218154401CA86136B2BA
:10CBD000B045B8BF4646E868AB6936B23246E1199F
:10CBE0001818F5F729FCA8693018A861A8EB060009
:10CBF00068627FE0B9F1610F16D14FF0700918E05B
:10CC0000464504DA95F83810090758BFB046B8F120
:10CC1000010848BF4FF00008B9F1670F14BF4FF08B
:10CC200045094FF0650904E0B9F1410F08BF4FF025
:10CC30005009A969E86817F8013B0B544A1CB8F180
:10CC4000010F05DA95F83810090758BFAA6117D502
:10CC50002E211154531CB8F1010FAB6110DB761E6D
:10CC600036B2B045B8BF464636B2324639461818D5
:10CC7000F5F7E2FBA8693018A861A8EB0600686226
:10CC8000E868A9690F18200007F8019B03D42B203E
:10CC900007F8010B03E02D2107F8011B6442002671
:10CCA0000DF1080808E00A2200A802F049F90198ED
:10CCB00008F8010B761C009C21B20129F3DA022E40
:10CCC00006DA49F02000652804BF302007F8010B80
:10CCD0004EB9302007F8010B07E0761E02A8305C41
:10CCE000303007F8010B012EF7DAE868A969081857
:10CCF000381AE86195F8380000F0140010280DD1BA
:10CD00006869A9690818696A0818E9690818A96AA8
:10CD10000818696B8842BCBF081A286205B0BDE8D4
:10CD2000F083F8B504460D4616461F46002004E081
:10CD3000E86A401CE8627F1E002047B116F8011B1C
:10CD4000A868A047A8600028F2D14FF0FF30F2BDDC
:10CD5000686A6C747A4C00006E616E004E414E0041
:10CD6000696E6600494E4600300000000CB41CB5E8
:10CD7000044604A801900A46009401AB00A90748A4
:10CD800078441830FFF71CF9009A00211170002830
:10CD90005CBF0098001B16BC5DF80CFB3357FFFF0F
:10CDA0000901002806D55C4A00F00F00801800F841
:10CDB000041C7047594A8154704710B5401EB0F1A9
:10CDC000807F01D3012010BD554C60600F214FF0D2
:10CDD000FF30FFF7E5FF0020A06007202060002063
:10CDE00010BD5048006870474F48006800F08060F0
:10CDF000704738B54D4D2878401C28704C4C207831
:10CE0000401C2070FAF77CFE02F0A2F8FAF7AAFBA9
:10CE10002878411E2970002802D19820FAF72CFBAF
:10CE20002078012804D16068002801D0FAF790FB2F
:10CE30002078401E2070BDE83140FAF78DBB30B538
:10CE400085B000A80FF200111422F5F705FB394D4B
:10CE500028680090364C6078F021084202D0992072
:10CE6000FAF70AFBFAF77EFB6078401C607002F06C
:10CE700003F928684FF47A71B0FBF1F0FFF79DFFDA
:10CE8000002800D0FEE72C482C4908600E214FF006
:10CE9000FF30FFF785FF2868009000A802F060F9D6
:10CEA0002748016841F0404101606078F021084264
:10CEB00002D09920FAF7E0FA6078401E6070C0B2A4
:10CEC000002801D1FAF748FB05B030BD80B501E07C
:10CED000FBF7C4FA1B4841680029FBD10068002811
:10CEE000F6D1FBF7B9FAF5E710B41148006A114919
:10CEF00009684FF47A72B1FBF2F10A4A1368CB1A4F
:10CF0000094C2468640102D512688B1A401C00FB8E
:10CF1000013010BC7047000018ED00E000E400E0B4
:10CF200010E000E018E000E004ED00E009710020EE
:10CF3000081F0020282500200000000808ED00E060
:10CF400034EF00E0B470002000000000E8030000AF
:10CF500000000000E3CD0008E9CD0008EFF30580F4
:10CF6000002842F01F81704780B5EFF3108072B641
:10CF70000B49096851F47F01094A116080F3108858
:10CF80000848006810F4700F02D1A720FAF774FA6D
:10CF900005485FF00071016004480021016001BD97
:10CFA00020ED00E088ED00E03CEF00E034EF00E031
:10CFB00010B5040010000A0001002000F5F78CFAFB
:10CFC000200010BD0901002807D5DFF8302B00F044
:10CFD0000F00801800F8041C7047DFF8842C81547F
:10CFE000704710B5401EB0F1807F01D3012010BD05
:10CFF000DFF8704C60600F214FF0FF30FFF7E2FF69
:10D000000020A06007202060002010BDDFF8582C11
:10D01000002803D040211046FEF715BC40211046E1
:10D02000FEF713BCDFF8402C00284FF48051104667
:10D0300001D0FEF708BCFEF708BC1CB5DFF82C4C8D
:10D040002046FEF711FB0121084601F08AFD012070
:10D050008DF8040000208DF80500ADF806004FF4AF
:10D06000807120460183C0464FF48070009000A973
:10D070002046FEF7A7FB4FF480710020FBF7F0F984
:10D0800013BDF0B583B0DFF8E04B2046FEF7ECFAB5
:10D09000DFF8DC5B2846FEF7E7FADFF8D86B3046AE
:10D0A000FEF7E2FA0121084601F05BFD01210220B2
:10D0B00001F057FD0121042001F053FD01218020E2
:10D0C00001F04FFD03208DF8040001208DF80600CB
:10D0D00000208DF807008DF8050049F6FF600090EC
:10D0E000DFF8887B00A93846FEF76CFB4FF6FF702F
:10D0F000009000A92046FEF765FB00A92846FEF730
:10D1000061FB00A93046FEF75DFB0021012001F024
:10D1100028FD0021022001F024FD0021042001F05F
:10D1200020FD0021802001F01CFD0121032001F0E1
:10D1300018FD01208DF8040000208DF80500ADF8E1
:10D1400006000121022001F00CFD40212046018350
:10D15000C0464020009000A92046FEF733FB4FF464
:10D16000805120460183C0464FF48055009500A9A8
:10D170002046FEF727FB294638464183C0460095E6
:10D1800000A93846FEF71EFB04220A212046FEF7BE
:10D190005EFB092203212046FEF759FB02208DF891
:10D1A000040001208DF805008DF8060000208DF8A0
:10D1B00007004FF48060009000A92046FEF702FBB4
:10D1C0000820009000A92046FEF7FCFA042208215E
:10D1D0002046FEF73CFB042207212046FEF737FBE2
:10D1E00002208DF8040001208DF805008DF806005E
:10D1F00000208DF807004FF48070009000A92046B1
:10D20000FEF7E0FA8020009000A92046FEF7DAFA47
:10D21000F7BD30B585B0DFF8401C884235D0DFF867
:10D220003C1C88422FD14FF480050C460121284632
:10D2300001F0A2FC0121022001F093FC012128460B
:10D2400001F0BBFC0021284601F0B7FC0020ADF83E
:10D2500004004BF6FF70ADF806004FF48060ADF8A7
:10D260000A004FF48040ADF80C000A20ADF8080029
:10D27000DFF8AC0C009000A9204601F0DCFF012192
:10D28000204602F03BF805B030BD4FF400150C46C7
:10D29000CCE72DE9F04192B001214FF4805001F02C
:10D2A00076FC0121032001F05CFC01214FF4800099
:10D2B00001F057FCDFF8B449052211462046FEF77D
:10D2C000C6FADFF8A459052211462846FEF7BFFA30
:10D2D000052204212846FEF7BAFA05220F2120462E
:10D2E000FEF7B5FA02208DF8040001208DF8050044
:10D2F0000020ADF806002020009000A92046FEF78F
:10D3000061FA2020009000A92846FEF75BFA102061
:10D31000009000A92846FEF755FA4FF4004000900F
:10D3200000A92046FEF74EFADFF8F84B2046FEF73C
:10D33000A5FDDFF8F45B00202880686001202881CB
:10D3400000206881E8600720288200206880DFF8DC
:10D35000DC6B3046FEF78EFADFF8D47B3846FEF7FA
:10D3600089FA4FF48060069000210D9103210E91FF
:10D3700000210F910A910890DFF8380C03900846BD
:10D380001090099007904FF400300C9008460B90D5
:10D390004FF0C068CDF80880402005900846049002
:10D3A00002A93046FEF7EAFA00200B90CDF808807B
:10D3B000059005F11400049002A93846FEF7DEFA44
:10D3C0000020688029462046FEF7B4FD0122022194
:10D3D0002046FEF7E3FD012211462046FEF7DEFD62
:10D3E00001212046FEF7CEFD00213046FEF7FEFA71
:10D3F00000213846FEF7FAFA12B0BDE8F08130B5E8
:10D4000089B001214FF0805001F0B6FB012001F0FE
:10D410003BFC01214FF4802001F0A3FB0F20FCF71F
:10D4200003FE04461020FCF7FFFD0546012001F035
:10D4300095FB002001F092FB21460F20FCF7E7FD51
:10D4400029461020FCF7E3FD00214FF4802001F075
:10D4500088FB042001F00CFB412001F0CFFB0028E9
:10D46000FAD04FF4807001F063FB012001F000FB63
:10D47000012001F070FBFCF770FC0120069043F6E0
:10D48000FF7007900020059005A8FCF71DFC002008
:10D49000029002A9FCF782FC00208DF80700012011
:10D4A0008DF804008DF805008DF8060001A9002014
:10D4B000FCF7F1FC4FF4800001F09CFA4FF480007F
:10D4C000039000208DF8100008208DF81100012035
:10D4D0008DF8120003A801F04FFA03208DF8000028
:10D4E0000D208DF8010000208DF8020001208DF83C
:10D4F000030000A801F069FF0320FCF741FD4FF491
:10D500008040FCF7DAFD4FF4800001F073FA01214E
:10D510004FF48040FCF795FD012009B030BD1FB5E8
:10D520000121084601F01DFB01214FF4804001F06C
:10D530002EFB00208DF80C008DF80F0001200290CA
:10D54000DFF89C4A02A92046FEF73CF9042002902D
:10D5500002A92046FEF736F90820029002A92046CB
:10D56000FEF730F90021084601F068FF0221002093
:10D5700001F064FF0321002001F060FF00208DF81E
:10D58000040001208DF8060000900C208DF80500A5
:10D5900000A801F0F1F9042000900C208DF805009E
:10D5A00000A801F0E9F9082000908DF8050000A816
:10D5B00001F0E2F9012001F01DFA042001F01AFA4D
:10D5C000082001F017FA1FBD00B585B001210846FB
:10D5D00001F0C7FA01214FF4804001F0D8FA002091
:10D5E0008DF810008DF813000820039003A9DFF8D0
:10D5F000F009FEF7E7F80321002001F01FFF0020EB
:10D600008DF8080001208DF80A00082001908DF89F
:10D61000090001A801F0B0F9082001F0EBF9092098
:10D620008DF800000E208DF8010000208DF802001A
:10D6300001208DF8030000A801F0C7FE05B000BD71
:10D6400000B585B00121084601F08BFA01214FF4A5
:10D65000804001F09CFA00208DF810008DF8130036
:10D660000420039003A9DFF87809FEF7ABF8022144
:10D67000002001F0E3FE00208DF8080001208DF865
:10D680000A00042001900C208DF8090001A801F087
:10D6900073F9042001F0AEF908208DF800000E2087
:10D6A0008DF8010000208DF8020001208DF80300A4
:10D6B00000A801F08AFE05B000BD38B5DFF82449A6
:10D6C0002078401C2070DFF820592878401C2870F2
:10D6D000FAF716FA6878F021084202D09920F9F793
:10D6E000CBFEF9F73FFF6878401C687000F0B8FB8C
:10D6F0006878F021084202D09920F9F7BDFE6878D9
:10D70000401E6870C0B2002801D1F9F725FF4FF420
:10D710008040FCF7BBFC002814D04FF48040FCF79D
:10D72000CCFC4FF4800001F065F9F8F7BFFA0090E7
:10D7300000A9DFF8B80801F065F9DFF8B418042093
:10D74000F8F758FBF9F70EFF2078411E21700028EA
:10D7500002D19820F9F790FE2878012804D1686852
:10D76000002801D0F9F7F4FE2878401E2870F9F758
:10D77000F3FE31BDDFF87C080068704738B5044619
:10D78000012C38DB012001F07FFA0020FCF717FCA8
:10D790004FF400550420FCF76FFC012804D1284603
:10D7A000451E80B20028F5D100EE104AB8EEC00A3E
:10D7B000DFEDB50A80EE800AF0EE000A20EE200AC6
:10D7C000DFEDC20A80EE800ABDEEC00A10EE100A3C
:10D7D000401E80B2FCF7E4FB4FF48040FCF76DFC88
:10D7E0004FF4800001F006F90120FCF7E8FBDFF8B8
:10D7F0000408046031BD0020DFF8F817086001203C
:10D8000001F042FA0020BDE83240FCF7D8BB00002E
:10D8100070B501240023DFF8E0171A468A608A6891
:10D8200012F00C0FFBD1DFF8D42705460C2D4BD896
:10D83000DFE805F01D4A4A4A07181D2C31363B40E7
:10D8400045008D6845F080058D604FF4C065DFF8B8
:10D85000B06735600D6825F080750D60DFF8A4575E
:10D86000156032E02346DFF8A05715602DE08D6883
:10D870008D604FF4C065DFF8886735600D6825F06E
:10D8800080750D60DFF8845715601EE00223DFF815
:10D890008057156019E00323DFF87857156014E00E
:10D8A0000423DFF8745715600FE00523DFF86C5789
:10D8B00015600AE00623DFF86857156005E00723C6
:10D8C000DFF86057156000E01C46002B4AD00FF6C9
:10D8D000640503EBC3035B198D688D600D6825F04B
:10D8E00080750D600D6825F080650D609D781E883F
:10D8F00045EA8615DE787608761E45EA06451E79E5
:10D9000045EA06654D60DD881E7A360746EA8515CC
:10D91000DFF8146735600D6845F080750D600D689F
:10D92000AD01FCD55B7943F4C063DFF8D4562B60BE
:10D930008B688B608B688B60052804D1886840F009
:10D940009000886005E00B2803D1886840F480507F
:10D950008860886840F002008860886800F00C00E9
:10D960000828FAD11068DFF8C416884207D2DFF819
:10D97000C006016821F4404141F480410160106813
:10D980004FF47A71B0FBF1F0FFF72BFB204670BD2E
:10D990003EE7002800E0401EFDD17047F0B583B09F
:10D9A0000727DFF8B414884203D14FF48074802530
:10D9B00002E04FF48064082501208DF804008DF802
:10D9C00005008DF8060000208DF807000094DFF8B0
:10D9D000646600A93046FDF7F5FE009500A93046C3
:10D9E000FDF7F0FE214630464183C0460F20FFF789
:10D9F000D0FF214630460183C0460F20FFF7C9FF04
:10DA00003846471E80B20028ECD1009500A9304668
:10DA1000FDF7D8FE214630464183C0460520FFF77A
:10DA2000B8FF294630460183C0460520FFF7B1FF05
:10DA3000214630460183C0460A20FFF7AAFF21464F
:10DA400030464183C0460520FFF7A3FF29463046F4
:10DA50004183C0460520FFF79CFF02208DF804009B
:10DA600001208DF805008DF8060000208DF80700D4
:10DA7000009400A93046FDF7A5FE009500A93046A8
:10DA8000FDF7A0FEF7BD000000007A4438B5002481
:10DA9000DFF8A4550121286801F069FC286801F02D
:10DAA0009BFB2868FFF7B5FB05E02868FFF776FFCA
:10DAB0002868FFF7AEFB4FF40031286801F062FCE4
:10DAC000002802D0641C032CEFDB31BD00000047AE
:10DAD00030B40022838A008BDFF85C45656843EA36
:10DAE00000400840000255EA10206060084088426B
:10DAF00000D10122104630BC7047000018ED00E054
:10DB00002DE9F84F04460D4616464FF080091F7860
:10DB1000DFF824854FF40031D8F8000001F032FC22
:10DB2000002808D04846A0F101090028F2D1FFF7EB
:10DB3000ADFF00203EE0D8F8000001884FF6FF520C
:10DB4000114001800121D8F8000001F0E3FB4FF4FF
:10DB5000007AD1460020C8F80400D8F800B0DFF8F9
:10DB6000DC145846FFF7B4FF002806D14846A0F160
:10DB700001090028F1D100201CE0D14600222146F5
:10DB8000584601F0DFFB0020C8F80400D8F8004038
:10DB9000DFF8AC142046FFF79BFF00280CD1484665
:10DBA000A0F101090028F1D10121D8F8000001F00D
:10DBB000BDFB0020BDE8F28F3146C9B2204601828C
:10DBC000C046D1460020C8F80400D8F80040DFF86D
:10DBD00074142046FFF77CFF002805D14846A0F1C9
:10DBE00001090028F1D1DFE7012F15D1297820465E
:10DBF0000182C046D1460020C8F80400DFF848146E
:10DC0000D8F80000FFF764FF002822D14846A0F1B1
:10DC100001090028F2D1C7E73846471EC0B20028E4
:10DC200017D015F8011BD8F800000182C046D14674
:10DC30000020C8F80400DFF81014D8F80000FFF73F
:10DC400047FF0028E8D14846A0F101090028F2D199
:10DC5000AAE70121D8F8000001F068FB0120A9E73C
:10DC600000E400E010E000E0000402400000024098
:10DC700000080240001C02402DE9F54F81B00D461E
:10DC80001E464FF080083778DFF8AC434FF4003180
:10DC9000206801F077FB002808D04046A0F1010879
:10DCA0000028F3D1FFF7F2FE002039E02068018858
:10DCB0004FF6FF52114001800121206801F02AFB3C
:10DCC0004FF40079C84600206060DFF870A3D4F8F4
:10DCD00000B051465846FFF7FBFE002805D14046EC
:10DCE000A0F101080028F2D16EE000229DF8041096
:10DCF000584601F027FBC84600206060D4F800B009
:10DD0000CF495846FFF7E4FE00280BD14046A0F16A
:10DD100001080028F2D10121206801F007FB002052
:10DD2000BDE8FE8FBDF80810C9B258460182C04652
:10DD3000C846C649206801F025FB002805D14046A9
:10DD4000A0F101080028F4D1E5E70121206801F0E5
:10DD5000E1FAC84600206060D4F800B05146584649
:10DD6000FFF7B6FE002805D14046A0F101080028C3
:10DD7000F2D129E001229DF80410584601F0E2FAA0
:10DD8000022FC84638DAB249206801F0FBFA0028B1
:10DD900005D14046A0F101080028F4D1BBE70021DD
:10DDA000206801F0D8FA2068018B012101F0BEFA49
:10DDB000C846A849206801F0E5FA002806D1404687
:10DDC000A0F101080028F4D10020A9E72068008A0A
:10DDD000C0B228703078401E3070C8462068018874
:10DDE000890505D54046A0F101080028F6D192E743
:10DDF000012101F0B0FA29E0002060609649206816
:10DE0000FFF766FE002805D14046A0F10108002872
:10DE1000F4D180E7012616E0012F0CD1012E0AD1A2
:10DE200000263146206801F096FA2068818A018B2D
:10DE3000012101F07BFA2068818A490603D5008A16
:10DE400005F8010B7F1EFFB2002FE5D101212068EC
:10DE500001F081FA012063E70054004000580040BF
:10DE60007E48016808292FD163490A6842F0807210
:10DE70000A604268B2F1806F03D10A6842F08062A2
:10DE80000A600A689201FCD58A6842F002028A6040
:10DE90008A6802F00C02082AFAD14268B2F1806F57
:10DEA00002D10A681201FCD5544909685F4A9142BF
:10DEB00006D25F490A6822F4404242F480420A6076
:10DEC00000210160416070474168B1F1806F09D164
:10DED00049490A6842F080620A600A681201FCD56A
:10DEE0000021416070475E48016841F08051016047
:10DEF0004F4801688908890041F0010101600FF273
:10DF000035005849086070475748016821F00401FE
:10DF1000016030BF016841F00401016070470000FA
:10DF200070F3050000300140506E0020586402403C
:10DF30001064024010B5F7F7A4F9012803D10120BD
:10DF400000F0A5FE02E0002000F0A1FE464C80217A
:10DF50004648FEF72DF800281FD172B626483F49E3
:10DF6000826802F00C020A60006800F0806048607D
:10DF7000206840F004002060FCF71CF8B0F5704FFA
:10DF800002D90220FCF70CF830BF62B6206820F0FE
:10DF900004002060BDE8104062E7206820F0040023
:10DFA000206030BF206840F00400206010BD2D4884
:10DFB000006800470C3001400949401E05280DD873
:10DFC000DFE800F0030507090C0B1A4906E02849B1
:10DFD00004E0284902E0284900E028490846704743
:10DFE0000000024009710020081F0020DC2E0020E4
:10DFF00018370020CC70002000380240282500206F
:10E00000003C024000127A00809698000024F40040
:10E0100000366E010048E801005A6202006CDC0222
:10E0200080F0FA0200BD0105843802400190D0035F
:10E030000070004000040240A825002001000300F9
:10E040008200070080000700840007000400001021
:10E050000200001040000010020003009470002035
:10E0600040380240D070002010ED00E00030014048
:10E0700000080240000C024000100240001C024058
:10E0800010B50C46FFF798FF214689B2BDE8104055
:10E09000FDF7D9BB10B50C46FFF78EFF214689B2BC
:10E0A000BDE81040FDF7D1BBE0B5002A03D10C223A
:10E0B0008DF8092002E008228DF8092000281CD0E4
:10E0C000012802D0032821D007BD01200190102093
:10E0D0008DF8090006208DF800000E208DF8010053
:10E0E00000208DF808008DF80200002917D00120CB
:10E0F0008DF80A008DF8030015E004200190082037
:10E100008DF800000E208DF80100E9E7082001904D
:10E1100009208DF800000E208DF80100E0E78DF851
:10E120000A008DF8030001A800F026FC00A801F009
:10E130004CF907BD200110040F03020103F0001089
:10E14000060F01020103C00010080F01020103C005
:10E150000010060F01020103F00010060F0102017A
:10E1600003600008040F02020103C80010040F023C
:10E17000020103A80010020F0302010310B50400FE
:10E1800003E02068C068F9F717FD802080F311884C
:10E1900000BF00BF20680028F3D108484078F02174
:10E1A000084202D09920F9F767F90448407800281E
:10E1B00002D1002080F3118810BD00BF081F00208D
:10E1C00000B585B0029001900E4A926803928022B9
:10E1D00082F3118800BF00BF0268009200AA0260AB
:10E1E0000098002802D0009800AA42600548806884
:10E1F00000AA8260034880680174F9F77DFD05B0CC
:10E2000000BD00BF081F0020012001F02BB9000055
:10E210000749086808B1002070470648C008C000D8
:10E2200008600549C908C900091A0160704700BFA4
:10E23000FC7000204F08002048180020012804DB53
:10E24000421E531002EB937205E010F1030F04DA43
:10E25000421000EB9272921000E0002210F0030FC7
:10E2600000D110B90FF2441001E00FF2281030F97C
:10E270001100801870472DE9F84F044642484018B5
:10E28000154600901CB9414801F0F6F80446256295
:10E290004FF461650098DFF8F8A00FF210160FF246
:10E2A000F4076FF0020840F26D1902E0009800F5E3
:10E2B00061605146B0FBF1F14B1C4FF0070C93FB32
:10E2C000FCFCCCEBCC0CA3EB0C03A3614B4691FB09
:10E2D000F3F300E05B1E012B05DB5A1E4FEA620ED2
:10E2E00002EB9E7204E0434505DA5A1003EB92728A
:10E2F0004FEAA20C01E04FF0000C13F0030F02D123
:10E300000BB1BE4600E0B646BEF90020944409FBBE
:10E3100003CC6145DEDBA1EB0C02636113F0030F5C
:10E32000E26100D10BB9334600E03B464FF00C0CE4
:10E3300003F1180E3EF902BD5A45ACF1010CF9DBB0
:10E34000C4F810C00AFB110033F91C30D21A521C59
:10E350002946E260B0FBF1F1A16005FB11003C2110
:10E36000B0FBF1F1C1EB01126160A0EB8200206013
:10E37000206A002805D5204601F08CF8012820628B
:10E3800094DA2046BDE8F28F807EAA830C0000203C
:10E390008051010000001F003C005B0079009800E4
:10E3A000B600D500F400120131014F0100001F003A
:10E3B0003B005A0078009700B500D400F30011012B
:10E3C00030014E01F0B5244E83B0304601F054F8D0
:10E3D0000446224D284601F04FF8006808B901F0C4
:10E3E000F3F8284601F048F80546301D01F044F8DE
:10E3F000064628682168814228D0007810B901F0CB
:10E40000F9F82860286800AA022101F0F8F8074608
:10E4100000230A2201A901F013F930600199009A42
:10E42000C91B914205D100F2135040F627218842C2
:10E4300001D3002030606421306890FBF1F101EBE2
:10E440008102C0EBC2003060286820603068A0EB19
:10E450000011880003B0F0BD040000203C00002043
:10E46000704700001FB500F01FFA212101601FBD99
:10E47000F0B540F2FF7581EA030C0CF0004C15EA90
:10E4800011541DBF15EA1357AC42AF42E5E0BC4141
:10E49000C1F31301C3F31303801A994143F48013AA
:10E4A00004D2641E4000494180185941C90241EA22
:10E4B0005051B1FBF3F603FB1611A2FB0675D7EB27
:10E4C000C020A94102D2761E80185941C90241EAF2
:10E4D0005051B1FBF3FE03FB1E11A2FB0E75D7EBEF
:10E4E000C020A94103D2AEF1010E80185941890222
:10E4F00041EA9051760546EA8E2EB1FBF3F603FB16
:10E500001611A2FB0675D7EB8020A94102D2761E18
:10E5100080185941C90241EA50514EEA060EB1FB3A
:10E52000F3F603FB1611A2FB0675D7EBC020A94139
:10E5300002D2761E80185941C90241EA5051B1FBFE
:10E54000F3F703FB1711A2FB0735D3EBC020A9415A
:10E5500067F100070CBF004247F0010766F3D527BB
:10E560004FEA1E31B80814F5806412DDBD0775F15D
:10E57000004250EB0E5051EB045111F5801F5CBF6F
:10E5800041EA0C01F0BD4CF07F6141F0E041002018
:10E59000F0BDBD076D0840EA0E5041F48011D4F182
:10E5A0000104B4F120060ADAC4F120060200E040BA
:10E5B00001FA06F3E1401843B24015430EE0342C53
:10E5C00013DCC6F1200445EA40056D0820FA06F286
:10E5D000154321FA06F0A1400D43002175F10042D8
:10E5E00050F1000051EB0C01F0BD00205FEA0C017E
:10E5F000F0BDCFB992185B41B3FA83F704BFB2FA0A
:10E6000082F6BF190B3FB7F120062FBF02FA06F3BF
:10E61000BB40C7F1200622FA06F638BF3343BA40A2
:10E620001CB1E419641E33E77F4231F00041B1FAB6
:10E6300081F404BFB0FA80F6A4190B3CB4F12006B3
:10E640002FBF00FA06F1A140C4F1200620FA06F619
:10E6500038BF3143A0403C1B1AE7AC421ABF05EA61
:10E660001357AF4212E050EA41061CBF52EA43067C
:10E67000BFE750EA4107304661461CBF41EA0551F9
:10E68000F0BD52EA430C08BFC143F0BD00204FF477
:10E69000001616EB410F98BF16EB430F08BF16EBA1
:10E6A000410F24BFC14305E016EB430F0CBF614689
:10E6B0004CEA0551F0BD0000D0B51446544A554B04
:10E6C000F7F72CF92DED048B41EC180B1DD89FEDBD
:10E6D000529B53EC182B51EC190BF6F791FF0022CB
:10E6E0004F4BF7F75FF806460F4653EC182B51ECEB
:10E6F000190BF7F757F802460B4630463946FFF735
:10E70000B7FE41EC180B44F0010451EC180B002249
:10E71000444BF6F75DFF05D301224FF07953F7F72D
:10E72000FDF851D853EC182BF6F76AFF41EC190BA2
:10E7300053EC182BF6F764FF06460F4653EC192BE3
:10E7400039483A49F6F75CFF394A3A4BF7F72AF865
:10E7500053EC192BF6F754FF374A384BF7F722F8EA
:10E7600032463B46F6F74CFF53EC182BF7F71AF8F6
:10E7700006460F4653EC192B31483249F6F740FF55
:10E78000314A324BF7F70EF853EC192BF6F738FFF6
:10E790002F4A304BF7F706F853EC192BF6F730FFFA
:10E7A0002D4A2E4BF6F7FEFF53EC192BF6F728FFF8
:10E7B0002B4B0022F6F7F6FF02460B463046394651
:10E7C000FFF756FE41EC180BA00705D551EC180BCE
:10E7D00081F0004141EC180B14F007020BD00FF24E
:10E7E000880303EBC20251EC180B53681268F6F76A
:10E7F000D9FF41EC180B200705D551EC180B81F01F
:10E80000004141EC180B51EC180BBDEC048BD0BD52
:10E8100057CD9E5E1426D13FAA4C58E87AB6FB3FEE
:10E820000000F0BF000040BE845D57134B57B03F5F
:10E83000B2934C19ED5EE43FBEDE02B90240F83FF0
:10E84000DE39028FC7C0743F8AAB1283000CC83F09
:10E8500024D7E508B6D8F03F0F34580E5895FD3F41
:10E860000000F03F00000000000000000000000079
:10E8700066732D3852C1E03F182D4454FB21F93FF7
:10E8800066732D3852C1F03F182D4454FB21F93FD7
:10E8900066732D3852C10040182D4454FB210940A5
:10E8A0003FD038C6A6F10440014800F0E5BD0000A5
:10E8B0000000002010EE101A04204FF07E5C01EEE4
:10E8C00090CA49004FEA510100EE101A88BF082093
:10E8D000B1F17E5F13D871EEC00ADFF838C031EEB7
:10E8E000801A61EE200AF1EEE00A614586BF80F0F1
:10E8F000040080EE800A80EE200A00F0E5BE4900A8
:10E9000011F1807F9CBF6FF0004100EE101A7FF67E
:10E91000A9AD7047F404353F10EE101A4FF07E5C3D
:10E9200001EE90CAC80F31F0004122D000EE101A5B
:10E93000B1F17E5F13D871EEC00ADFF838C031EE56
:10E94000801A61EE200AF1EEE00A614586BF80F090
:10E95000040080EE800A80EE200A00F0B5BE490077
:10E9600011F1807F9CBF6FF0004100EE101A7FF61E
:10E9700079AD7047F404353F30B40168CB431F498B
:10E980008279002A27D00A4614682340136053680E
:10E990000468A34353600379CC18236805682B43AC
:10E9A000236093680468A3439360D3680468A34317
:10E9B000D36043790568102B07D191682943916092
:10E9C000D16800680843D0600AE051FA83F42068F7
:10E9D0002843206004E000790C182068184020606B
:10E9E00030BC70470021064A1268024200D0012163
:10E9F000084670470249086070470000003C01402B
:10EA0000143C014070B504000D000126A07E66286C
:10EA100002D08220F8F730FDF9F725F81348007886
:10EA2000401C12490870802080F3118800BF00BF8D
:10EA3000E0682169884204D22900200000F02EF904
:10EA400000260A484078F021084202D09920F8F7C1
:10EA500013FD06484078002802D1002080F3118879
:10EA6000F9F76AF83000C0B270BD00BF081F00207F
:10EA7000DFF8C81100220A700A70012802D00428A9
:10EA800003D0704701200870704705200870704758
:10EA9000DFF8AC110860704730B46A494A6802F088
:10EAA0000C02042A02D0082A03D022E0674A02603E
:10EAB00021E00A68C2F380520B6803F03F03002A8A
:10EAC00007D0624AB2FBF3F20B68C3F388135A43D0
:10EAD00006E05F4AB2FBF3F20B68C3F388135A43B4
:10EAE0000B68C3F301435B1C5B00B2FBF3F20260F3
:10EAF00001E0574A02604A6802F0F003554A1B09D8
:10EB00009B5C05682C46DC4044604B6803F4E05392
:10EB10009B0A9B5C2546DD408560496801F46041A5
:10EB2000490B895C42681346CB40C36030BC7047D8
:10EB3000454900F44072B2F5407F06D10A6822F4DC
:10EB4000F812454B03401A430A608A6E000552EAE8
:10EB50001050886670474149086070474049086016
:10EB60007047404A0029116802D00843106070477E
:10EB700021EA0000106070473B4A0029116802D06A
:10EB800008431060704721EA000010607047374A60
:10EB90000029116802D008431060704721EA000084
:10EBA00010607047324A0029116802D00843106093
:10EBB000704721EA0000106070472E4A0029116852
:10EBC00002D008431060704721EA000010607047CF
:10EBD000294A0029116802D008431060704721EAD1
:10EBE000000010607047254A0029117802D00843C0
:10EBF0001070704721EA00001070704741090E4AFA
:10EC0000012901D1116804E0022901D1116F00E04E
:10EC1000516F00F01F000A46C24002F00100704729
:10EC20000021174A1268024200D0012108467047AD
:10EC300014490870704700000038024070380240E4
:10EC4000800E4742043802400838024040787D0177
:10EC50000024F4004C250020FFFCFF0F3C0E47422F
:10EC6000400E4742303802404038024044380240AB
:10EC70001038024020380240243802400D3802404B
:10EC80000C3802400E3802400249086070470249C1
:10EC90000860704720000E4224000E4238B5028BF7
:10ECA000C3684469E3180469A34201D304691B1BC8
:10ECB000534384680D781D55491C5B1C521E002A65
:10ECC000F7D1C168491CC160012902D1FFF756FA8A
:10ECD0000EE027484078F021084202D09920F8F74A
:10ECE000CBFB23484078002802D1002080F3118814
:10ECF00031BD10B50400208B62694243A368D35C28
:10ED00000B70521C491C401E0028F7D16069401C42
:10ED100060612169884201D300206061E068411E82
:10ED2000E1602169884212D111484078F0210842FF
:10ED300002D09920F8F7A0FB0D484078002802D1B6
:10ED4000002080F311882000FFF718FA0EE0084831
:10ED50004078F021084202D09920F8F78DFB044852
:10ED60004078002802D1002080F3118810BD0000F7
:10ED7000081F00200278C9B28A421AB11CBF10F8DD
:10ED8000012FF9E718BF002070470000C9B28307C0
:10ED900006D0521E22D310F8013B9942F7D11FE052
:10EDA000083A13D302F1040241EA012141EA014188
:10EDB00050F8043B121F21BF4B40A3F1013C2CEA49
:10EDC000030C1CF0803FF3D0C9B2001F083210F8CA
:10EDD000013B521E28BF91EA030FF8D818BF01204B
:10EDE000401E704730B4436803F0004201211B030A
:10EDF0001B0B436004BF0368002B08D10DE00368C0
:10EE0000DD0F45EA440444605B000360491E44682A
:10EE1000E302F4D523031B0B436043681A434260AB
:10EE2000084630BC7047000070B504460D46606867
:10EE3000C0F30A5040F2FF71884207D160680003B6
:10EE400004BF2068002817D0022070BD20B92046DA
:10EE5000FFF7C8FF012868DA012D0FDB40F2FF71D0
:10EE6000091A8D420AD3606800284CBF9FED300B11
:10EE70009FED310B84ED000B012070BD4142A94292
:10EE8000616806DA6FF31E51401941EA0050606074
:10EE900042E0401E63684519012205F1350062F326
:10EEA0001F53352801F00041636003D361600020E7
:10EEB000206070BD002215F11F0F04DA2268236064
:10EEC000002020356060684214D0521E25689241AF
:10EED000C0F12003D2439D4045EAD272256825FA4D
:10EEE00000F6656805FA03F333432360636823FA89
:10EEF00000F5656060680843B2F1004F606003D8B8
:10EF00000DD12078C0070AD52068401C20602068F9
:10EF100028B96068401C60604FF0FF3070BD6068C9
:10EF2000884204BF20680028F6D1002070BD00BFD1
:10EF3000000000000000F0FF000000000000F07F73
:10EF400091FBF2F303FB1211C0E90031704700009E
:10EF500010B522480078002802D1A220F8F78CFAD8
:10EF60001F48406B002807D01D48012180F8381049
:10EF70001B480121417127E01948006A401C1849CB
:10EF800008621749D1E90A23521C53F100031449BE
:10EF9000C1E90A231249496A401A002802D41048DC
:10EFA000012141710E4890F8300000280CD00C4827
:10EFB00090F83000401E0A4981F83000C0B20028A5
:10EFC00002D10748012101710648046802E0606827
:10EFD00080472468002CFAD110BD00BF09710020C1
:10EFE000081F0020EC700020BFF34F8F49480168D4
:10EFF00001F4E061484A11430160BFF34F8F00BF45
:10F00000FDE710B5454C606C40F4804060644448B6
:10F01000016801F0070101290CD10168C908C90084
:10F020000160006800F00700012803D1FFF7DCFF52
:10F0300000BFFDE74FF4407000F0C2F939480168A5
:10F0400041F470010160206840F001002060002060
:10F05000A06020683449084020603448606020681F
:10F0600020F4802020600020E06000F039F84FF0AC
:10F0700000602F49086010BD00212E48426802F050
:10F080000C02042A02D0082A04D01CE02A492B4A88
:10F0900011611BE00268C2F38052036803F03F0372
:10F0A000002A06D12649B1FBF3F10268C2F38812A7
:10F0B00051430268C2F30142521C5200B1FBF2F10B
:10F0C0001E4A116102E01E491C4A11614068114646
:10F0D000C0F30310405C0A691346C3400B617047DC
:10F0E0001448C16B41F08051C16316490A6822F48B
:10F0F000404242F480420A60416841604168416098
:10F1000041684160082101604FF4C0600E49086009
:10F11000704700000CED00E00400FA0500380240E2
:10F120000038014088ED00E0FFFFF6FE10300024BB
:10F1300008ED00E00438024040787D0118250020E9
:10F140000024F40000700040003C024005E0B0FBE9
:10F15000F1F201FB1202080011000029F7D17047FB
:10F1600038B501000E481422F3F776F90C48006810
:10F170000B494968B0FBF1F0094948614FF47A74D2
:10F180000748456929002000FFF7E0FFB4FBF0F1D4
:10F19000034A9161B5FBF0F00149C86131BD00003F
:10F1A0007C6F00200021102806DB103800F1604140
:10F1B00011F56441097806E00E2801D1042007E02A
:10F1C0000449001F415C802901DA022000E001208F
:10F1D000704700BF18ED00E080B5434988420BD16D
:10F1E00001214FF40010FFF7E8FC00214FF400105C
:10F1F000BDE80440FFF7E1BC3C4988420BD1012146
:10F200004FF48000FFF7D9FC00214FF48000BDE8E7
:10F210000440FFF7D2BC364988420BD101214FF49C
:10F220000000FFF7CAFC00214FF40000BDE80440D5
:10F23000FFF7C3BC01BD7FB504460D46A68800A8F4
:10F24000FFF72AFC02992B48B1FBF0F04FF6C07291
:10F2500032400243A28022884FF6FE731A40228079
:10F260002A68254B9A420AD25200B1FBF2F10A46B3
:10F2700092B2042A00DA0421401C208421E0EB88A9
:10F280004BF6FF76B34204D102EB4202B1FBF2F13E
:10F2900006E019235A43B1FBF2F141F4804189B2EF
:10F2A0000A0502D141F0010189B241F4004180B266
:10F2B0004FF4967250434FF47A7290FBF2F0401C78
:10F2C0002084A183208840F00100208020884FF610
:10F2D000F5310840A9880843698908432080A88936
:10F2E0002989084320817FBD005400400058004018
:10F2F000005C004040420F00A18601000029018807
:10F3000003D041F00101018070474FF6FE721140B9
:10F31000018070470029018803D041F48071018089
:10F3200070474FF6FF621140018070470029018845
:10F3300003D041F40071018070474FF6FF52114035
:10F3400001807047002A02D041F0010101E001F084
:10F35000FE01018270470029018803D041F48061D9
:10F36000018070474FF6FF3211400180704700293D
:10F37000018803D041F40041018070474904490CE1
:10F380000180704782B0024600200346019300933B
:10F3900000920A0F01920902090A019A002A03D079
:10F3A000009A1432009203E0090C009A183200927D
:10F3B000009A12680A4200D0012002B07047000093
:10F3C00019490843194908607047F0B403781A4690
:10F3D0000121C478002C1DD0144B1B6803F4E0639A
:10F3E000C3F5E0631B0A4478C3F10405AC4085789B
:10F3F0000F2637461F4107EA050323431B010C4C28
:10F400001355007800F01F0291400A4A401142F85B
:10F41000201007E003F01F0001FA00F00649521126
:10F4200041F82200F0BC70470000FA050CED00E046
:10F4300000E400E000E100E080E100E030B401F031
:10F440000302920021F00301054BCC580F25954093
:10F45000AC43CC50CC5890402043C85030BC70478F
:10F460000838014080B5C046C046024A1100182045
:10F47000ABBEFBE72600020004490968002900D161
:10F480000349034A801A411808007047F0700020B1
:10F49000000000202DE9F84304464748FFF7ECFF41
:10F4A00080464648FFF7E8FF454F05463846FFF7D8
:10F4B000E3FF006808B900F087F83846FFF7DCFF83
:10F4C00006464048FFF7D8FFD8F8001007463868CE
:10F4D000814220D0007878B93068007810B900F007
:10F4E00089F83060306800AA032100F088F838609D
:10F4F000017809B1401E3860386800F04BF9060009
:10F5000008BF4FF0FF3054D02868FAF750F92E604A
:10F510003868C8F800004FF0000960690021FEF764
:10F520008DFE8046E169A0682D6801EB410200EB89
:10F53000C207606940F26D1101FB0080401C072189
:10F5400090FBF1F1C1EBC101401A00F10E0600E0A1
:10F550006D1D2878FF282BD0606929798842F7DB58
:10F56000E978FEF76BFEA978A0EB08000818297867
:10F5700071B13218521A072392FBF3F3C3EBC303A2
:10F58000D21A18BFC2F1070210180829B8BFC01F4D
:10F5900000EB4001687800EBC100874208DB287966
:10F5A000697A88420CBF89F001094FF00009CFE762
:10F5B0004846BDE8F28300BF440000203800002028
:10F5C0003C0000204000002038B5084C2046FFF7E2
:10F5D00053FF006848B90FF218052046FFF74CFFAB
:10F5E0000560201DFFF748FF056031BD3C0000208D
:10F5F000000000000FF20400704700003A00F8B568
:10F6000004460D462078002816460CBF002714F843
:10F61000017B01E06D1E441C39462046FFF7AAFB22
:10F6200018B92046F7F70CFF0019012D03DA001B6B
:10F6300030602046F2BD01780029EBD13160F2BD87
:10F640002DE9F04182B080460E001D4608BF00AE95
:10F65000474600E07F1C3878A0F109010529F9D35D
:10F660002028F7D02D2816BF2B2817F8014B2B2464
:10F670003146384600F02CF931688F4208BFC6F891
:10F6800000803168884514D120B92D2C16D1B0F1F5
:10F69000004F15D9FFF708F9222101600DB10120B3
:10F6A00028602D2C14BF6FF000404FF00040BDE8E3
:10F6B000F6812B2CE9D1B0F1004FEBD2BDE8F681F9
:10F6C0004042BDE8F68100001AA210EE101ADFF8E1
:10F6D00060C0F2EC060A614509DB00EE803A70EE8C
:10F6E000800A83EE200A40F0020010EE101A21F08A
:10F6F000004CDCF1665C0BD860EE000A20EE203A8C
:10F7000003EE010A01EEA02A42EE202A80EE220A30
:10F71000400810F0020F18BFB1EE400A02EB800261
:10F72000D2ED000A30EE200A28BFB1EE400A704741
:10F73000A430893ED7B3DD3F6AD5033F2B94A93D62
:10F74000B82A593F0000803F000080BF0000000041
:10F75000920A063FDB0FC93F920A863FDB0FC93F83
:10F76000920A0640DB0F4940368D274000220AE00E
:10F770000378303B0A2B09D202EB820310F8012BED
:10F7800002EB4302303A491EF2D501E04FF0FF325E
:10F79000104670472DE9F843054615F8018BB8F17E
:10F7A000000F00F092802846022601E0401C761CE3
:10F7B0004146FFF7DFFA0028F8D106EB8600F9F79B
:10F7C00096FE060000F08180002734464FF0FF3996
:10F7D00000E0641D287828280BD10421681CFFF75D
:10F7E000C5FFA0F26C77002F6CD46879292869D105
:10F7F000AD1D277102212846FFF7B8FF401EE070BB
:10F80000AD1C0220294600220AE00B78303B0A2B6F
:10F8100009D202EB820311F8012B02EB4302303ACA
:10F82000401EF2D500E04A46501EA07015F8021F97
:10F8300030390A2928BF002316D202212A46002384
:10F840000DE092F800C0ACF1300CBCF10A0F09D207
:10F8500003EB830C12F8013B03EB4C03303B491ED6
:10F86000EFD500E04B46AD1C6370E1780C29BFBFBB
:10F87000C0B264286078642824DA28782B2818BF5E
:10F880002D2802D00020207010E06878A0F130010F
:10F89000072917D230280CBF07203038207028786D
:10F8A0002B2802D12078C01D2070AD1C287828B9E3
:10F8B000FF20607167723046BDE8F28315F8010BD6
:10F8C000404586D03046F9F772FF0020BDE8F2834C
:10F8D0002DE9F04F85B004461E000D4690461CBF32
:10F8E00000203060A14601E009F1010999F800000B
:10F8F000A0F109010529F7D32028F5D02D2816BF3E
:10F900002B2819F8017B2B27B8F1000F57D4B8F139
:10F91000010F54D0B8F1250F51DAB8F1010F0DDB0A
:10F92000B8F1100F04BF99F80000302802BF99F811
:10F93000010040F02000782814D10EE099F8000072
:10F94000302818BF4FF00A080CD199F8010040F098
:10F950002000782804D14FF0100809F1020901E0D5
:10F960004FF00808CDF8109001E009F1010999F86D
:10F9700000003028F9D00FF2A00B4FF0000ACDF8AC
:10F980000C908DF808B00AE09DF80810CDF804A09E
:10F99000401AC0B2009008FB0A0A09F1010999F85F
:10F9A0000010A1F141001A2838BF203142465846C4
:10F9B000FFF7ECF90028E7D10498484503D105B1D9
:10F9C0002C60002025E00FF27801039818F8011050
:10F9D000A9EB0000401A14D4012808DA0098BAEB09
:10F9E000000004D30199B0FBF8F0884209D0FEF77B
:10F9F0005BFF222101600EB1012030604FF0FF3A21
:10FA000003E02D2F08BFCAF1000A0DB1C5F8009020
:10FA1000504605B0BDE8F08F3031323334353637DB
:10FA200038396162636465666768696A6B6C6D6EBC
:10FA30006F707172737475767778797A0000000050
:10FA400000002115110E0D0C0B0B0A0A09090909FA
:10FA5000090808080808080807070707070707072D
:10FA60000707070707000000F0B583B004460D46FE
:10FA700016461F460020ADF806008DF80400012050
:10FA8000009001AB2A467221204601F04AF901009C
:10FA900015D18DF806509DF80400B04338438DF819
:10FAA00004009DF804008DF8070002230DF1060202
:10FAB0007221204601F0D7F8010000D10020FEBDE0
:10FAC00070B582B004460020ADF80000DFF8805D1C
:10FAD0002878062818DB002600E0761C032E11D2B9
:10FAE000701900798DF800007019007A8DF8010006
:10FAF000022300AA7221204601F0B5F80100ECD0E3
:10FB0000297076BD0020287076BD1CB50446002003
:10FB1000ADF806008DF804002046012807D004281F
:10FB200005D0102803D0402801D0802846D10023DA
:10FB3000022280210520FFF797FF010047D1012015
:10FB4000009001AB90227221052001F0EAF801003B
:10FB50003DD19DF8040000F0FC008DF80400012C5C
:10FB60000AD0042C04D0102C1ED0402C21D025E02B
:10FB700040F001008DF8040090208DF806009DF8FB
:10FB800004008DF807009DF8040000F00300DFF882
:10FB9000C41C487002230DF106027221052001F0F9
:10FBA00062F801000CD016BD40F002008DF8040090
:10FBB000E2E740F003008DF80400DDE7012016BD08
:10FBC00002231A4680210520FFF74EFF002016BDB4
:10FBD00010B582B00020ADF8000082208DF8000042
:10FBE00000AC38206070022300AA7221082001F0C6
:10FBF0003AF801001FD18E208DF800009620607029
:10FC0000022300AA7221082001F02DF8010012D170
:10FC10008F208DF8000008206070022300AA722156
:10FC200001F021F8010006D108231A46D921104617
:10FC3000FFF71AFF002016BD38B50022ADF80020EE
:10FC4000DFF8104CA28A002902D01043A08202E003
:10FC500022EA0000A082A08A002805D002284BD00A
:10FC60001FD3032848D01AE0DD208DF8000000AD36
:10FC700000206870022300AA7221052000F0F3FF23
:10FC800001000DD180208DF8000000206870022353
:10FC900000AA7221052000F0E6FF010000D100203B
:10FCA00032BD81208DF8000000AD11206870022364
:10FCB00000AA7221052000F0D6FF0100F0D168787B
:10FCC0002070DD208DF8000000206870022300AA5B
:10FCD0007221052000F0C7FF0100E1D180208DF8DE
:10FCE000000003206870022300AA7221052000F0A2
:10FCF000BAFF0100D4D1D2E781208DF8000000AD19
:10FD000011206870022300AA7221052000F0ABFFC9
:10FD10000100C5D168782070FFF75AFF0100BED0FE
:10FD200032BD2DE9FE4F82468B4616461C46002703
:10FD3000B846DFF8205B0FF250106978085C29782C
:10FD4000491C10FB01F240F6DC235A43029289025F
:10FD5000B1F5803F01D34FF6FF71C9000A22B1FB14
:10FD6000F2F1102808D18C4206D34FF0010840462A
:10FD7000FFF7CBFE074619E0102808D1642C06DAFD
:10FD80004FF001084020FFF7C0FE07460EE0402874
:10FD900002D164398C4203D2012807D1642C05DAE0
:10FDA0004FF001081020FFF7B0FE0746B8F1000F32
:10FDB0000BD06A7839460FF63C30F4F799FC002FE7
:10FDC00001D101205EE038465CE0AA69D3172046E5
:10FDD000A0FB028900FB0399CDE90089E869C117FE
:10FDE000D046A8FB002308FB0133DDE900018018A1
:10FDF0005941CDE900012A6AD3175846A0FB028970
:10FE000000FB0399DDE9000110EB080841EB09094B
:10FE1000686AC117A6FB002306FB0133404649462A
:10FE20008018594132461AFA8BF3D3181B1B03EB87
:10FE3000D3735B101BB2AAEB0306D41A002903DCB0
:10FE400000DB01D200200146002E00D10126D5F8AA
:10FE500028804FEAE879A8FB002308FB013309FB5F
:10FE6000003310461946029AD317FAF7C1F90C99D4
:10FE70000860E86A604390FBF6F0296B08180D995A
:10FE800008600020BDE8FE8F0104104000B585B079
:10FE9000DFF8C019CA6902600A6A42604A6A826071
:10FEA0008A69C2608A6A0261CA6A4261096B8161B9
:10FEB00003914169029101690191C16800918368D0
:10FEC000426801680FF64420F4F712FC1C2005B0CC
:10FED00000BD00B585B01C2806D001460FF65020A5
:10FEE000F4F706FC01201FE0DFF868090A68C26128
:10FEF0004A6802628A684262CA6882610A698262EA
:10FF00004A69C2628A6902638869039048690290FB
:10FF100008690190C86800908B684A6809680FF604
:10FF20002C20F4F7E5FB002005B000BD1CB504460D
:10FF300000208DF80400ADF806000120009001AB10
:10FF400093227221082000F0ECFE002811D19320AA
:10FF50008DF806009DF8040020438DF80700022369
:10FF60000DF106027221082000F07DFE010000D193
:10FF7000002016BD10B582B00020ADF800000FF6CD
:10FF8000F010F4F7B5FBDFF8D0080221C1720021B0
:10FF900041730123072280210820FFF765FD002817
:10FFA00022D1DD208DF8000000AC08206070022313
:10FFB00000AA722100F057FE010015D16023E02253
:10FFC000D9210820FFF750FD00280DD1D7208DF84A
:10FFD000000001206070022300AA7221082000F0B6
:10FFE00042FE010000D1002016BD70B582B0002590
:10FFF0002C462146ADF80010042801DB012076BD17
:020000021000EC
:10000000002805D0022810D008D3032814D017E008
:10001000DFF8440801720478457811E0DFF8380809
:10002000012101728478C5780AE0DFF82C080221EA
:1000300001720479457903E06424DFF81C084579EE
:10004000224629460FF64410F4F752FB88208DF81B
:10005000000000AE7470022300AA7221082000F094
:1000600002FE01000CD18A208DF800007570022379
:1000700000AA7221082000F0F6FD010000D1002046
:1000800076BD00002DE9FC410446002001900646A3
:10009000DFF8C477787B002805D10FF60410F4F759
:1000A00027FB0320C4E00120009001AB9C227221B9
:1000B000082000F036FE002840F0BA809DF8048049
:1000C00040466070387A042800F2AC80DFE800F027
:1000D000030F2EAA400041460FF6D400F4F708FBA8
:1000E0000120FFF782FF010040F0A2807AE0F8785B
:1000F00040450BDA41460FF6C800F4F7F9FA022042
:10010000FFF773FF010040F093808BE0B8788045E3
:1001100080F2888041460FF6BC00F4F7E9FA3046D9
:10012000FFF763FF010040F083800DE041460FF6CA
:10013000B800F4F7DDFAFFF71DFF010078D1304673
:10014000FFF753FF010073D101260020207069E002
:1001500041460FF6A400F4F7CBFA0220009001AB61
:10016000C0227221082000F0DCFD002860D19DF83B
:1001700004309DF80520002A03D0184645422DB2D0
:1001800000E01D4629460FF68400F4F7B1FAFB2D76
:100190002CDBC0208DF806000DF106062846283815
:1001A000707002230DF106027221082000F05BFD41
:1001B00001003DD171780FF67000F4F799FAC12073
:1001C0008DF806000020707002230DF106027221E6
:1001D000082000F048FD01002AD10320FFF705FFA9
:1001E000010025D10126304620701BE0F8784045FB
:1001F00005DA0220FFF7F9FE010019D107E078784F
:10020000404507DA0120FFF7F0FE010010D1012080
:10021000207006E03046FFF7E8FE010008D13046C6
:1002200020700126A5712DB22812E07186F0010020
:10023000BDE8F68180B5042806D001460FF2FC70B7
:10024000F4F756FA012002BD0878002808D04A7851
:10025000002A05D08A78002A02D0CA78002A05D15F
:100260000FF2F470F4F744FA012002BDDFF8E8253C
:100270005070487890708878D070C8781071C878BD
:1002800000908B784A7809780FF2D870F4F730FA3A
:10029000002002BD1CB504460020ADF80400022079
:1002A000009001ABC0227221082000F03AFD002826
:1002B00001D0002016BD9DF8041001A84278002A44
:1002C00000D049429DF80420227043786370227860
:1002D00009B20FF2A870F4F70BFA022016BD70B540
:1002E00082B004465E25002600E040365E2E18DA15
:1002F000C6F15E00402801DB402000E080B2C0B2C1
:10030000009033193046A0F18002D2B27221082049
:1003100000F007FD0028E8D00FF27870F4F7E8F954
:100320000025284676BD38B50C460125012806D0A3
:1003300001460FF27070F4F7DBF9002032BD284659
:100340000090134622787221082000F0EAFC002871
:1003500005D021780FF26C70F4F7CAF90025284611
:1003600032BD80B5022806D001460FF27C70F4F74A
:10037000BFF9012002BD02230A467221082000F0C5
:1003800072FC010000D1002002BD00B583B0012144
:10039000009101AB9222722100F0C3FC01000AD14E
:1003A0009DF80410E42905D00FF25C70F4F7A0F971
:1003B00001200EBD00200EBD38B50020ADF80000B4
:1003C0000520FFF77DFB40B2014601292CDADFF85A
:1003D000844440F29D30A062DFF88004E06140F286
:1003E0004C402062DFF8780460624FF47A70A061BC
:1003F00040F6C150E06240F62F002063002500E087
:100400006D1C052D12D2281900798DF800002819CD
:10041000007B8DF80100022300AA7221052000F064
:1004200022FC40B20100EBD0C0B232BD002032BD90
:1004300080B50520FFF7A9FF4020FFF766FBDFF836
:100440001404002181700321C17001210846FFF7C7
:10045000F3FB40B2010001D0C0B202BD002002BDDA
:1004600080B500210120FFF7E7FB40B2010001D079
:10047000C0B202BD002002BD2DE9F04389B00446A0
:1004800007A800210A4606C00846059006900820E5
:10049000009007AB94227221052000F042FC002856
:1004A00053D19DF81C00A07307A84178E1738178AF
:1004B0002172C17861720179A1724079E0729DF870
:1004C000220020739DF823006073DFF8885328789A
:1004D000207468786074607A217A41EA0026E07AB4
:1004E000A17A41EA0027607B217B41EA0028E07B7A
:1004F000A17B41EA002906A8019005A800904B467F
:10050000424639463046FFF70CFC01001DD10598E4
:100510002060069860600120A870E878002813D059
:100520000120049005980390687802902878019043
:10053000CDF8009043463A4631460FF2EC50F4F7BE
:10054000D7F8E878401EE870002009B0BDE8F083D5
:1005500030B404460D4611461A4600201C2C06D025
:100560001D2C07D0222C08D1104630BC8EE410463A
:1005700030BCB4E6284630BCD5E630BC704780B508
:100580000B4611461D2805D0222806D11846FFF734
:10059000A0FC02E01846FFF7E4FE002002BD10B503
:1005A00082B00020ADF8000004460820FFF788FA6A
:1005B000010015D100E0641C032C10D2A948215C75
:1005C0008DF80010201800798DF80100022300AA90
:1005D0007221082000F047FB0100ECD016BD00207E
:1005E00016BD38B50020ADF800009B4C04202072E9
:1005F000002060738C208DF8000000AD3020687002
:10060000022300AA7221082000F02DFB01002BD14B
:100610000120207301460220FFF70EFB010023D1C9
:1006200088208DF80000FF206870022300AA722144
:10063000082000F018FB010016D18A208DF8000078
:1006400000206870022300AA7221082000F00BFB32
:10065000010009D1FFF78EFC010005D12020FFF732
:1006600065FC010000D1002032BD10B588B003A8A0
:1006700000210A4606C00FF2E8410CC90CC0002454
:10068000754821460173407B002822D100E0641C9C
:10069000062C0CDA0120009003A8231805A8225C80
:1006A0007221082000F03DFB0028F0D01DE003A8D7
:1006B0009DF8111002919DF8101001919DF80F10F6
:1006C0000091837842789DF80C100FF29C40F4F76B
:1006D0000FF800210220FFF7AFFA010005D120201A
:1006E000FFF724FC010000D1002008B010BDFEB5CA
:1006F000044600200190ADF808000646054601209A
:10070000009001AB93227221082000F00AFB002820
:1007100040F09D80012000900DF10503DC22722144
:10072000082000F0FEFA002840F09180FF20FFF73B
:10073000FDFB010040F08B80474F9DF8040040070F
:100740000CD5387B002809D00FF25C40F3F7D0FFBE
:10075000FFF710FC01007AD10120FEBD9DF80400D6
:10076000000747D5387B002844D001231A46DC21F6
:100770000820FFF779F9002869D106231A4680215D
:100780000820FFF771F9010061D1DD208DF8080024
:1007900024208DF80900022302AA7221082000F00B
:1007A00062FA010053D19DF805100FF21040F3F7E3
:1007B0009FFF0FF22040F3F79BFF01207873022088
:1007C00000900DF10603C0227221082000F0A9FA62
:1007D00000283CD19DF806109DF80720002A00D083
:1007E00049429DF8063009B20FF22020F3F780FF4E
:1007F0000120FEBD9DF80400800609D50126204693
:10080000FFF740FC002803D1387B002800D0354694
:100810009DF80400C021084200D00126002E09D115
:100820003869411C39619DF804200FF2C430F3F798
:100830005FFF01E00020386138691E2805D30FF200
:10084000C830F3F755FF0020386185F00100FEBD88
:10085000842500208020002004250020C2FCFFFF0A
:1008600064FBFFFFB02500201CB504460020ADF856
:1008700004000220009001ABC0227221082000F089
:1008800050FA00280DD10120009001AB9C2272216A
:10089000082000F046FA002803D19DF804002070DB
:1008A000002016BD30B404460D4611461A460020FD
:1008B0001C2C06D01D2C07D0212C08D1104630BC92
:1008C000E8E4104630BC0AE5284630BC2BE530BCD5
:1008D000704780B50B4611461D2805D01E2806D14D
:1008E0001846FFF7A7FC02E01846FFF73AFD002084
:1008F00002BD0000233E206761696E206368616766
:100900006E6564282564292025640000233E6C2040
:1009100067657420434F45462025642025642025C3
:1009200064202564202564202564202564000000BF
:10093000233E6C20636F6566206C656E677468206B
:100940006572726F7228256429000000233E6C20B6
:1009500073657420434F4546202564202564202577
:10096000642025642025642025642025640000007F
:10097000233E702063616C6962726174696F6E20DE
:10098000537461727420212121000000233E7020E5
:100990004849202564204C4F572025642000000042
:1009A000233E7020647572696E672063616C00007D
:1009B000233E7020444554454354202564000000E4
:1009C000233E70204445544543545F4849474820DE
:1009D00025640000233E702044482052454C454188
:1009E0005345202564000000233E702052454C45AD
:1009F0004153452025640000233E70204E4F4E4554
:100A00005F4D4F444520256400000000233E7020C8
:100A10006F666673657420256420307825782C20F5
:100A20003078257800000000233E702057726974EA
:100A300065206F666673657420256400233E702010
:100A4000746864206C656E677468206572726F727A
:100A50002825642900000000233E7020746864206B
:100A60003D203000233E7020746873657420257526
:100A7000202575202575202575000000233E702057
:100A80006F66667365742025642030782578203081
:100A900078257800233E2064756D70206661696C4E
:100AA00065640000233E20676574207265672076C8
:100AB000616C206C656E677468206572726F722855
:100AC00025642900233E20676574207265672076BF
:100AD000616C206661696C656428616464722030B1
:100AE0007825782900000000233E20736574207269
:100AF00065672076616C206C656E6774682065722E
:100B0000726F722825642900746D64333732352082
:100B100064657669636520696420283078257829C2
:100B2000206661696C656400233E723D2564206720
:100B30003D256420623D256420633D256420617469
:100B4000696D653D256420616761696E3D2564209E
:100B50006C75783D25752072656164793D2564006A
:100B600080888A93D7DD0000233E72454E41424C77
:100B7000453D2564207250494C543D2564207250F7
:100B80004948543D256420725354415455533D25E2
:100B900064207243414C49423D25642072494E54C1
:100BA000454E41423D256400233E702072656164DC
:100BB0002053545F5A494E5400000000233E7020D9
:100BC0007243414C494253544154203D20307825D2
:100BD00078000000233E702043616C69627261748A
:100BE000696F6E2046696E69736865642000000055
:100BF000233E20696E7620696E742025642073740C
:100C00006174757320257800233E207265736574C6
:100C100052510000052805D0082803D01D2801D016
:100C2000222803D17248734908607047724871499D
:100C30000860704710B5C0B2F3F715F900280DD061
:100C40006E4C2068401C20601E2807D30FF2B8109D
:100C5000F3F74EFDFCF71AFF0020206010BD0020C6
:100C60006649086070472DE9F84305460E46174669
:100C70004FF00208624C6078F021084202D09920BF
:100C8000F6F7FAFBF6F76EFC6078401C60709DF892
:100C90000000401E8DF8000017F9019B284640B265
:100CA000FFF7B8FF00AB4A4692B239463046FCF730
:100CB00027FF002812D06078F021084202D0992046
:100CC000F6F7DAFB6078401E6070C0B2002801D1F0
:100CD000F6F742FCFFF7C3FF002020E04FFA88F848
:100CE000424629460FF23410F3F702FD4046A0F1C8
:100CF00001080028D6D16078F021084202D099205E
:100D0000F6F7BAFB6078401E6070C0B2002801D1CF
:100D1000F6F722FC284640B2FFF78CFF0120BDE821
:100D2000F2832DE9F04704460D4616461F46DFF8CC
:100D3000D480089888F80000DFF8C49099F8010082
:100D4000F021084202D09920F6F796FBF6F70AFC4C
:100D500099F80100401C89F80100204640B2FFF7D5
:100D600059FF4FF0020A4346324639462846FCF7FF
:100D700083FF002815D099F80100F021084202D025
:100D80009920F6F779FB99F80100401E89F80100D7
:100D9000C0B2002801D1F6F7DFFBFFF760FF0020AB
:100DA00023E04FFA8AFA524621460FF27C00F3F70D
:100DB0009FFC5046A0F1010A0028D4D199F8010007
:100DC000F021084202D09920F6F756FB99F801006D
:100DD000401E89F80100C0B2002801D1F6F7BCFB23
:100DE000204640B2FFF726FF0120BDE8F087000053
:100DF00000540040A825002000580040C870002082
:100E0000081F002005710020233E496E6974696C3B
:100E100061697A6520493243000000004957452046
:100E200025642025640000004952452025642025C2
:100E30006400000080B500920B460246D6210120D6
:100E4000FFF76FFF02BD70B5A0B006460D46144611
:100E500000A88021F1F738FB2046802801DB012023
:100E600012E08DF80060002105E04A5D00ABCB1870
:100E70005A70491CC9B28142F7DB631CDBB200AA7D
:100E8000D6210120FFF7EFFE20B070BD80B50092A3
:100E90000B460246D6210420FFF743FF02BD70B582
:100EA000A0B006460D46144600A88021F1F70CFBC1
:100EB0002046802801DB012012E08DF8006000212F
:100EC00005E04A5D00ABCB185A70491CC9B281429B
:100ED000F7DB631CDBB200AAD6210420FFF7C3FEB8
:100EE00020B070BD70B582B004460D461646002095
:100EF000ADF80000012200A92046FFF7C7FF002837
:100F00000BD19DF80000A84330438DF80100012269
:100F10000DF101012046FFF7C2FF76BD80B5DFF875
:100F2000BC0A4178807840EA0102FE211120FFF7D7
:100F3000D9FF401E8041C043C00F00D1002002BD38
:100F400080B5DFF89C1A0A78521C0A7080B2F7F755
:100F50004BFABDE80140F6F7EFBD38B50420F2F7D3
:100F600082FF006A00284FD0C0684FF4C871002883
:100F700004D04FF47A7191FBF0F109B200254800DA
:100F8000DFF8584A00E06D1C082D05DA04EB450235
:100F9000B2F920209042F6DA082D00D10725281951
:100FA000007C6178884205D06070FFF7B7FF0028A9
:100FB0000AD031BD94F90C00002805D40FF6643036
:100FC000BDE83240F3F794BB6078402808D0502841
:100FD00006D0602807D0702805D0802803D005E00F
:100FE0000420207304E00820207301E00220207315
:100FF00094F90C2004EB4500B0F920100FF63430C2
:10100000BDE83840F3F774BB31BD80B500208DF8E2
:101010000000802211460920FFF764FF00283FD11D
:101020005C208DF800000246FE211120FFF75AFFD8
:10103000002835D1002240211220FFF753FF00285D
:101040002ED183208DF80000012200A90620FFF791
:1010500026FF002824D1012207210846FFF742FF7E
:1010600000281DD108208DF80000012200A9FFF7FB
:1010700016FF002814D100208DF80000012200A9DD
:101080000920FFF70CFF00280AD129208DF8000065
:10109000012200A90A20FFF702FF002800D100204A
:1010A00002BD2DE9F04788B005460E4604A8002190
:1010B00001600F4602A80A4606C000A806C005A89F
:1010C0000B460EC0FFF7A1FF8146B9F1000F05D016
:1010D0000FF67820F3F70CFB484608E1C820FFF72D
:1010E0002FFF4FF44070F4F731FC04000FD10220C1
:1010F000FDE001270020059005A84FF0000CC0F886
:1011000004C0C0F808C0ADF800E04A808B8000221F
:1011100007210A20FFF7E6FE8146B9F1000F04D04F
:101120000FF63020F3F7E4FADBE06420FFF708FF66
:10113000012207210A20FFF7D5FE8146B9F1000FF1
:1011400004D00FF61820F3F7D3FACAE06420FFF7B3
:10115000F7FE4FF4C0786420FFF7F2FE042204A9E2
:101160003A20FFF793FE002810D19DF811000006E9
:1011700002D54FF0000812E0A8F101080FFA88F834
:10118000B8F1000FE7D14FF00109AAE00FF6D41033
:10119000F3F7AEFA4FF00109A3E008F10108B8F542
:1011A000C07F0EDA022204EB48013E20FFF76EFEFC
:1011B0008146B9F1000FF0D00FF6B010F3F798FAAE
:1011C0008FE000203060804602A901E008F10308AA
:1011D000B8F5C07F3BDA3068401C306034F8180046
:1011E000ADF8080004EB4800B0F90290A1F80290B5
:1011F000B0F904A0A1F804A00598BDF9082000FAF0
:1012000082F0059005A8426802FA89F2426082687D
:1012100002FA8AF28260002000E0401C0328D5DA3E
:1012200002AA32F91020002A00D55242B2F50F6FFF
:10123000F3DD0FF64010F3F75BFABDF808002880E5
:10124000A5F80290A5F804A04FF0010949E04FF07D
:10125000000805A80CE050F8281040318A1101EB75
:101260005261C91140F8281025F8181008F101083A
:10127000B8F1030FEFDBB5F90430B5F90220B5F989
:1012800000E000A9012F7FF434AFBDF80000A0EB0F
:101290000E00ADF800004888801A48808888C01A7F
:1012A00088804FF0000801E008F10108B8F1030F51
:1012B0000EDA00A830F91800002800D5404249286D
:1012C000F2DB0FF6B800F3F713FA4FF0010908E06C
:1012D0000022FE211120FFF705FE8146B9F1000F23
:1012E00004D1002C02D02046F4F748FB484608B051
:1012F000BDE8F08710B584B000A80FF688011CC9BE
:101300001CC00A2200A91020FFF7C9FD002807D140
:10131000002207210A20FFF7E5FD002800D1002068
:1013200004B010BDF0B587B004460D4600208DF81E
:10133000000001A800210A4606C00E46084604E047
:1013400045F8260044F82600761C032EF8DBFFF74C
:10135000D1FF002840F0E780C820FFF7F1FD0A2701
:101360000520FFF7EDFD012200A91E20FFF78EFDED
:10137000002840F0D8807F1E03D09DF80000800731
:10138000EED5062201A92220FFF780FD002840F0BB
:10139000CA8000262DE00A270520FFF7D1FD012293
:1013A00000A91E20FFF772FD002840F0BC807F1EC0
:1013B00003D09DF800008007EED5062201A9222067
:1013C000FFF764FD002840F0AE80012E10DB20689E
:1013D000BDF9041000FA81F0206001A86168B0F93D
:1013E000022089186160A168B0F904000818A060A3
:1013F000761C062ECFDB2068052190FBF1F02060E3
:10140000606890FBF1F06060A06890FBF1F0A06074
:1014100004220C211420FFF765FD002840F0838092
:101420003220FFF78DFD0A270520FFF789FD0122F5
:1014300000A91E20FFF72AFD002874D17F1E03D0CB
:101440009DF800008007EFD5062201A92220FFF7B2
:101450001DFD002867D100262BE00A270520FFF795
:101460006FFD012200A91E20FFF710FD00285AD1B0
:101470007F1E03D09DF800008007EFD5062201A94A
:101480002220FFF703FD00284DD1012E10DB286834
:10149000BDF9041000FA81F0286001A86968B0F96C
:1014A000022089186960A968B0F904000818A860CA
:1014B000761C062ED1DB2868052190FBF1F0286010
:1014C000686890FBF1F06860A86890FBF1F0A86094
:1014D0000022FF211120FFF705FD002823D1002263
:1014E0000C211420FFF7FEFC00281CD100273E46EB
:1014F0000AE003A941F82600A0F65E0041F6B361B8
:10150000884200D37F1C761C032E07DA54F826206D
:1015100055F82610881AECD5501AEAE7012F01DB9E
:10152000012000E0002007B0F0BD70B594B0044683
:101530000020ADF814000FA800210A4606C00B4693
:101540000EC003A806C001A806C00CA80EC009A8BA
:101550000EC006A80EC008460090012205A90F2063
:10156000FFF794FC002840F0EC809DF814006A28F6
:1015700040F0E7800FF21860F3F7BAF805220FA9E0
:101580000620FFF783FC060006D10A2211A91020CD
:10159000FFF77CFC060005D00FF2FC50F3F7A8F82B
:1015A0003046D0E000A903A8FFF77BFD002821D03A
:1015B0000FF2EC50F3F79CF8BDF80C00ADF8040006
:1015C00001A803A94A8842808988818005220FA941
:1015D0000620FFF764FC060006D10A2211A910209C
:1015E000FFF75DFC060043D00FF2CC50F3F780F814
:1015F0003046A8E00A20FFF7A3FC00A903A8FFF7E4
:1016000050FD00280ED00FF2A050F3F771F8BDF88E
:101610000C00ADF8040001A803A94A88428089881B
:101620008180D3E709A90CA8FFF77CFE002805D02C
:101630000FF27C50F3F75CF8002500E00125002054
:101640000AE0891A01AA22F8101003A931F9101032
:1016500006AA42F82010401C0328B7DA0CA951F85A
:10166000202009A951F820108B1AEAD5511AE9E770
:1016700001202070BDF804006070BDF90400001264
:10168000A07001A8B0F90210E17009122171B0F93F
:10169000040060710012A071E5710098207200983A
:1016A0000012607200980014A07200980016E07298
:1016B0000698207306980012607306980014A073B1
:1016C00006980016E07306A8416821740A12627435
:1016D0000A14A2740916E1748068207501126175FC
:1016E0000114A1750016E0750C9820760CA8B0F9CD
:1016F0000000001260760CA94868A076B1F90400D9
:101700000012E07688682077B1F90800001260774F
:101710000998A07709A8B0F900000012E07709A99C
:10172000486884F82000B1F90400001284F8210010
:10173000886884F82200B1F90800001284F82300B8
:1017400000E00126304614B070BDF8B50446002014
:10175000ADF800000420F2F786FB054605F11C06F3
:10176000307B002806D10020E9694968884732208B
:10177000FFF7E6FB012200A91E20FFF787FB0028E8
:10178000F8D19DF800004007F4D5022200A92020DE
:10179000FFF77CFB0746307B002803D10020E96976
:1017A000C96888479DF801009DF8001041EA0020B3
:1017B00000B2C11000EB1170001119302070002030
:1017C00060703846F2BD8748704710B5834C0622DA
:1017D00004F118012220FFF759FB002805D00FF271
:1017E000E030F2F785FF012010BD1020F2F73BFB3F
:1017F000417804F1180000F059FA94F90C0001281E
:1018000009DB401E2073062204F1300104F11800A8
:10181000F0F722FE06E0062204F1180104F1300080
:10182000F0F71AFE002010BD10B50A46D2B20146EC
:101830000020FFF7FFFA040005D00FF28C30F2F71A
:1018400057FF204610BD0FF29030F2F751FF0020F5
:1018500010BD10B50122FFF7EDFA040005D00FF21C
:10186000A830F2F745FF204610BD40F232320FF2A9
:1018700078310FF2A030F2F73BFF002010BD10B519
:101880000122411C0078FFF7DEFA040005D00FF2B8
:10189000AC30F2F72DFF204610BD40F241320FF27E
:1018A0007C310FF27030F2F723FF002010BD10B52D
:1018B00082B00020ADF80000484C207060206070BD
:1018C0000820A070484860600020A060012200A9A4
:1018D0000F20FFF7DBFA002822D19DF800106A29BB
:1018E00005D00FF26430F2F703FF012016BD442249
:1018F00011461220FFF7F6FA002240211320FFF7CD
:10190000F1FA002280211620FFF7ECFAA0788DF87A
:10191000010001220DF101011120FFF7C0FA0020A2
:1019200016BD10B52D4CA06800060BD50022402135
:101930001320FFF7D7FA00280ED1A06820F080000E
:10194000A06008E04FF0FF302073FFF7E7FA0028AF
:1019500002D101202070002010BD10B586B00446D1
:1019600002A800210A460B460EC000A806C0FFF7D9
:101970002CFF02A94420F2F757FB1848018B029A6A
:10198000891AADF80010418B039A891AADF802103C
:10199000808B0499401AADF80400062200A9204665
:1019A000F0F74AFD002006B010BD10B5002240211E
:1019B0001320FFF797FA00280FD100F0C5FF074C5E
:1019C000A06820F08000A0600022F0211120FFF725
:1019D00089FA002801D10020207010BD14200020B9
:1019E000081F00202C200020295C0F3D70B5A8B0F6
:1019F00001A90FF2AC2370CB70C18DF80600002452
:101A0000182806D01C2829D01D2837D0262810D009
:101A100044E01EA82421F0F757FD1EA8FFF785FD1E
:101A200004462420ADF807001EA901A8F5F723FB02
:101A300034E02046ADF8000000A8FFF786FE04461B
:101A40009DF800100FF21820F2F752FE0220ADF8B8
:101A5000070000A901A8F5F70EFB1FE004A8682104
:101A6000F0F732FD652104A8FFF7DEFE6520ADF832
:101A7000070004A901A8F5F7FEFA0FE020468DF84B
:101A800002000DF102011078FFF7E3FE0120ADF82E
:101A900007000DF1020101A8F5F7EDFA204628B084
:101AA00070BD10B584B014461A2806D01D2830D059
:101AB000232812D02E2830D031E021780FF2B01038
:101AC000F2F716FE0420F2F7CEF9217841701020CB
:101AD000F2F7C9F92178417021E06078217841EA74
:101AE000002000B20090E078A17841EA002212B212
:101AF00001926079217941EA00231BB20293009997
:101B00000FF27C10F2F7F4FD00A94420F2F7B8F9C7
:101B100005E02046FFF7B3FE01E0FFF71EFA0020C4
:101B200004B010BD736B6970206779726F206F64A9
:101B3000722121006779726F206F64723A25642CDC
:101B400020736B69703A2564000000004746462DFB
:101B5000310000004746462D320000004746462D22
:101B6000330000004746462D340000004753462D01
:101B7000350000004753462D360000004753462DE0
:101B800037000000005C4400000000000038000046
:101B90004759524F2D5300004753462D3131000015
:101BA0004753462D464631004753462D46463200A0
:101BB0004753462D485700004753462D3132000009
:101BC00047462031000000004759524F2044554DF0
:101BD00050204621000000004759524F2044554DE7
:101BE00050205321000000006779726F5F6C736DA5
:101BF0003664736C5F6765745F726567697374657B
:101C0000725F76616C7565004759524F2047522DBF
